:020000040000FA
:1020000002A97402D9328F27AFA775A70F8FA77FB8
:10201000327E0012D132E52724FF92B47FE87E039E
:1020200002D13202D1F4D286D2872202D53C7D0180
:102030007F8012A70E901B9DE0FEA3E02400FFE42A
:102040003EFEC36480948050066307FF6306FF7CF6
:10205000007D021227FDE51B2FFFE51A3EFE7C00E6
:0A2060007D021227FD8E1A8F1B224D
:10206B0002D4FA7D1AAF16AE15129ACA12D5E97DB3
:10207B0018AF16AE15129ACA12D37F900968740363
:10208B00F09009677409F02202C68E8F27AFA775EF
:10209B00A70F8FA77F327E0012D132E52724FF9244
:1020AB00B57FC87E0002D13202D61CE590540C23BA
:1020BB00C0E074D6C0E0C082C08302D600E5905465
:1020CB000C23C0E074D6C0E0C082C08302D608E502
:1020DB0090540C23C0E074D6C0E0C082C08302D6FB
:1020EB0010E590540C23C0E074D6C0E0C082C083CE
:0A20FB0002D618EFC40390D600735C
:1021060002244EE86480F8E933E83360110460F095
:10211600ED33EC337009E8FCE9FDEAFEEBFF22043F
:1021260060DED3EB9FEA9EE99DE8C2E78CF0C2F73A
:1021360095F0400CE8CCF8E9CDF9EACEFAEBCFFB06
:1021460012241985D0F05804700320D5B3E8047022
:10215600075002B2D502245892D5EC0460F7E4CCBD
:10216600C0E0C398F8603B94186008400DD0E0FBCF
:10217600022430E4FBFAC9FC8028E830E406E4C90E
:10218600FBE4CAFCE830E305E4C9CACBFCE8540723
:102196006010F8C3E913F9EA13FAEB13FBEC13FC2E
:1021A600D8F130F52FC3E49CFCEF9BFFEE9AFEEDD1
:1021B60099FDD0E0FBEF4E4D4C701222DB0302245A
:1021C60055EC2CFCEF33FFEE33FEED33FDED30E73F
:1021D600EB022430EF2BFFEE3AFEED39FDD0E0FBAB
:1021E60050130BBB0003022458ED13FDEE13FEEF54
:1021F60013FFEC13FC022430EC4D6011E849701714
:10220600ED33EC3304600DE4FCFFFEFD22E933E818
:10221600330470F802244E12241958046009E4CCE1
:1022260024815006285009022458284003022455C8
:10223600C0E0EB4A7044B98006D0E0FB022444EFCC
:102246004E701CBD8008EBFFEAFEE9FD80EBE98DD0
:10225600F0A4FEE5F00222E7E9CDF9EAFEEBFFEF96
:1022660089F0A4FCE5F0CE89F0A42EFFE435F0CD8C
:1022760089F0A42DFEE435F08067EF4E7005BD8031
:10228600D780C3EF8BF0A4ACF0EE8BF0A42CFCE46B
:1022960035F0F8EF8AF0A42CE5F038FCE433CB8D6A
:1022A600F0A42CFCE5F03BF8EE8AF0A42CFCE5F05B
:1022B60038F8E433CF89F0A42CFCE5F038CF3400AD
:1022C600CE89F0A42FFFE5F03EFEE433C98DF0A4DD
:1022D6002EFEE5F039CD8AF0A42FFFE5F03EFEE4B0
:1022E6003DFD33D0E0FB50070BBB000F022458EC3A
:1022F6002CFCEF33FFEE33FEED33FD0224300224D7
:1023060058EC5D046005E85904700302244E12245B
:1023160019580460F6EC4860F2EC7004FDFEFF22EA
:10232600C860DB2481C85009C398600250060224A5
:10233600559850CAF582E9294B4A7005AB820224AA
:102346004475F0007C1A7880C3EF9BEE9AED9940B5
:102356000DC3EF9BFFEE9AFEED99FDE842F0DC23FC
:10236600ACF0D0E0FFD0E0FED0E0FDAB8220E7107D
:102376001BEB60BAEC2CFCEF33FFEE33FEED33FDC6
:10238600022430E803F830E705C0F075F000EF2FBF
:10239600FFEE33FEED33FD40B830E7C280AA75F09C
:1023A60020800E75F010800575F0087D007E007F98
:1023B600003392D530D5031229E1EC334010EF33C8
:1023C600FFEE33FEED33FDEC33FCD5F0ED22E5F008
:1023D600247EA2D513CC92E7CDCEFF22EDD2E7CD57
:1023E60033EC3392D524814006E4FFFEFDFC22FC4B
:1023F600E4CFCECDCC24E0501174FF80EDC3CC13D6
:10240600CCCD13CDCE13CECF13CF0470F030D5DEA6
:102416000229E1E9D2E7C933E833F892D5EDD2E7EC
:10242600CD33EC33FC5002B2D522EC30E7100FBFAF
:10243600000C0EBE00080DBD00040BEB6014A2D507
:10244600EB13FCED92E7FD2274FFFCFDFEFF22E498
:1024560080F8A2D574FF13FC7D80E480EFF920E7B5
:102466002824F950037907E4F42402FB18DBFDE67F
:1024760024FB5014E9600DE4F618E604F6B40A08E5
:10248600E4F6D9F57401F60A22C2D522ED33EC330F
:1024960092D5FA602AB4FF33EDC2E77BFF60067A75
:1024A6002479B7E4227A2479C020D5047A2479BB2A
:1024B600224E614E002B494E46002D494E4600E401
:1024C6007A08F608DAFC7B00740722E8C0E0ECC064
:1024D600E0EDC0E0EEC0E0EFC0E0EA75F010A4CA9F
:1024E600ABF075F04DA42BFBE435F0FCEA2410FAB2
:1024F600EB34C5FBEC34D9FCEDC2E7FF75F056A40E
:10250600F42411C5F0F434C58FF0A42AE5F03BE4B9
:102516003CF620E7141225C5D0E0FFD0E0FED0E05F
:10252600FDD0E0FC1223078014F4041225C5D0E088
:10253600FFD0E0FED0E0FDD0E0FC1221FED0E0F8B6
:10254600E6FAEDD2E7CD33EC332482FBE4C3CF3396
:10255600CFCE33CECD33CD33DBF37B0775F00A8494
:102566006004F6081B0AE5F0F6088FF0740AA4FF6B
:10257600ACF08EF0740AA42CFEACF050010C8DF079
:10258600740AA42CFDE435F0F608DBDE7407223F5E
:102596008000004120000042C80000447A00004646
:1025A6001C400047C35000497424004B1896804CC9
:1025B600BEBC205A0E1BCA6753C21C749DC5AEFB17
:1025C60060065407601C23231225F3EB5438600978
:1025D6001225DF1225EE1221FEECF8EDF9EEFAEFE8
:1025E600CB22EB1225EE80F1543803241C9025955E
:1025F600FE93FC0EEE93FD0EEE930ECE93FF22E7B6
:1026060009F608DFFA8046E709F208DFFA803E8815
:10261600828C83E709F0A3DFFA8032E309F608DF4C
:10262600FA8078E309F208DFFA807088828C83E307
:1026360009F0A3DFFA806489828A83E0A3F608DFC3
:10264600FA805889828A83E0A3F208DFFA804C80F8
:10265600D280FA80C680D4806980F2803380108070
:10266600A680EA809A80A880DA80E280CA803389D0
:10267600828A83ECFAE493A3C8C582C8CCC583CC0E
:10268600F0A3C8C582C8CCC583CCDFE9DEE7800DE0
:1026960089828A83E493A3F608DFF9ECFAA9F0EDC0
:1026A600FB2289828A83ECFAE0A3C8C582C8CCC51E
:1026B60083CCF0A3C8C582C8CCC583CCDFEADEE8EC
:1026C60080DB89828A83E493A3F208DFF980CC88D1
:1026D600F0EF60010E4E60C388F0ED2402B40400F2
:1026E60050B9F582EB2402B4040050AF232345828F
:1026F6002390265573BB010689828A83E022500205
:10270600E722BBFE02E32289828A83E49322BB018D
:102716000CE58229F582E5833AF583E0225006E945
:102726002582F8E622BBFE06E92582F8E222E5824A
:1027360029F582E5833AF583E49322BB010FF8E598
:102746008229F582E5833AF583E028F0225009C50F
:102756008229F8E58226F622BBFE09C58229F8E21F
:102766002582F222F8EA2583F583E9932822BB0124
:102776000689828A83F0225002F722BBFE01F322E9
:10278600F8BB010DE58229F582E5833AF583E8F089
:10279600225006E92582C8F622BBFE05E92582C835
:1027A600F222BC000BBE0029EF8DF084FFADF022B3
:1027B600E4CCF875F008EF2FFFEE33FEEC33FCEEB9
:1027C6009DEC984005FCEE9DFE0FD5F0E9E4CEFDAC
:1027D60022EDF8F5F0EE8420D21CFEADF075F0087F
:1027E600EF2FFFED33FD4007985006D5F0F222C3D8
:1027F60098FD0FD5F0EA22C2D5EC30E709B2D5E450
:10280600C39DFDE49CFCEE30E715B2D5E4C39FFF03
:10281600E49EFE1227A8C3E49DFDE49CFC800312FF
:1028260027A830D507C3E49FFFE49EFE22C5F0F833
:10283600A3E028F0C5F0F8E582158270021583E062
:1028460038F022A3F8E0C5F025F0F0E58215827095
:10285600021583E0C838F0E822BB0110E58229F5AD
:1028660082E5833AF583E0F5F0A3E0225009E925F5
:1028760082F886F008E622BBFE0AE92582F8E2F530
:10288600F008E222E5832AF583E993F5F0A3E993BC
:1028960022F8BB0111E58229F582E5833AF583E842
:1028A600F0E5F0A3F0225009E92582C8F608A6F063
:1028B60022BBFE09E92582C8F2E5F008F222E88F7C
:1028C600F0A4CC8BF0A42CFCE98EF0A42CFC8AF0AE
:1028D600EDA42CFCEA8EF0A4CDA8F08BF0A42DCCB0
:1028E6003825F0FDE98FF0A42CCD35F0FCEB8EF009
:1028F600A4FEA9F0EB8FF0A4CFC5F02ECD39FEE4EF
:102906003CFCEAA42DCE35F0FDE43CFC2275F00833
:10291600758200EF2FFFEE33FECD33CDCC33CCC521
:102926008233C5829BED9AEC99E58298400CF5823C
:10293600EE9BFEED9AFDEC99FC0FD5F0D6E4CEFBAE
:10294600E4CDFAE4CCF9A88222B800C1B90059BA9C
:10295600002DEC8BF084CFCECDFCE5F0CBF97818CA
:10296600EF2FFFEE33FEED33FDEC33FCEB33FB10C4
:10297600D703994004EB99FB0FD8E5E4F9FA2278DE
:1029860018EF2FFFEE33FEED33FDEC33FCC933C9F0
:1029960010D7059BE99A4007EC9BFCE99AF90FD8FA
:1029A600E0E4C9FAE4CCFB2275F010EF2FFFEE331A
:1029B600FEED33FDCC33CCC833C810D7079BEC9A59
:1029C600E899400AED9BFDEC9AFCE899F80FD5F0E2
:1029D600DAE4CDFBE4CCFAE4C8F922C3E49FFFE4D1
:1029E6009EFEE49DFDE49CFC22EB9FF5F0EA9E42F0
:1029F600F0E99D42F0EC6480C864809845F022EBD3
:102A06009FF5F0EA9E42F0E99D42F0E89C45F022EF
:102A1600E8600FECC313FCED13FDEE13FEEF13FF9E
:102A2600D8F122E8600FEFC333FFEE33FEED33FD3E
:102A3600EC33FCD8F1227401FF3395E0FEFDFC086F
:102A46000808E6CF2FF618E6CE3EF618E6CD3DF698
:102A560018E6CC3CF622ECF0A3EDF0A3EEF0A3EFE3
:102A6600F022A8828583F0D083D082122A7F122A90
:102A76007F122A7F122A7FE473E493A3C583C5F0ED
:102A8600C583C8C582C8F0A3C583C5F0C583C8C5BC
:102A960082C822A42582F582E5F03583F58322FAE1
:102AA600E6FB0808E6F925F0F618E6CA3AF622D05B
:102AB60083D082F8E4937012740193700DA3A393EC
:102AC600F8740193F5828883E4737402936860EF67
:102AD600A3A3A380DFD083D082E493701274019302
:102AE600700DA3A393F8740193F5828883E473743D
:102AF60002936C70127403936D700C7404936E7071
:102B0600067405936F60DDA3A3A3A3A3A380CAE302
:102B1600F5F009E208B5F06D606B80F3E3F5F009B6
:102B2600E608B5F060605E80F387F009E608B5F068
:102B360054605280F487F009E208B5F04860468098
:102B4600F488828C8387F009E0A3B5F0386036807C
:102B5600F488828C8387F009E493A3B5F027602577
:102B660080F388828C83E3F5F009E0A3B5F0166064
:102B76001480F388828C83E3F5F009E493A3B5F01F
:102B860004600280F2022C40808580E7808E80D22D
:102B9600803C8015806C807E809B80B5808B80A178
:102BA600804F8070803A022C4C89828A83ECFAE44A
:102BB60093F5F0A3C8C582C8CCC583CCE493A3C85B
:102BC600C582C8CCC583CCB5F070606E80E18982C1
:102BD6008A83E493F5F0A3E208B5F05E605C80F2C8
:102BE60089828A83E0F5F0A3E608B5F04D604B8054
:102BF600F389828A83E0F5F0A3E208B5F03C603AF7
:102C060080F389828A83E493F5F0A3E608B5F02A77
:102C1600602880F2805389828A83ECFAE493F5F087
:102C2600A3C8C582C8CCC583CCE0A3C8C582C8CC1E
:102C3600C583CCB5F004600280E27FFFB5F0020FD9
:102C46002240027F012289828A83ECFAE0F5F0A312
:102C5600C8C582C8CCC583CCE0A3C8C582C8CCC5CC
:102C660083CCB5F0D560D380E389828A83ECFAE021
:102C7600F5F0A3C8C582C8CCC583CCE493A3C8C568
:102C860082C8CCC583CCB5F0B160AF80E288F0EDE8
:102C96002402B4040050A3F582EB2402B4040050CD
:102CA600992323458223902B8E73E3F5F009E208DE
:102CB600B5F06BDFF58067E3F5F009E608B5F05E81
:102CC600DFF5805A87F009E608B5F052DFF6804E48
:102CD60087F009E208B5F046DFF6804288828C83E9
:102CE60087F009E0A3B5F036DFF6803288828C8360
:102CF60087F009E493A3B5F025DFF5802188828C5F
:102D060083E3F5F009E0A3B5F014DFF580108882BF
:102D16008C83E3F5F009E493A3B5F002DFF4022D0A
:102D2600DF808780E9809080D4803E8015806E8029
:102D36007E809D80B7808D80A380518074803C0208
:102D46002DEB89828A83ECFAE493F5F0A3C8C58259
:102D5600C8CCC583CCE493A3C8C582C8CCC583CCF4
:102D6600B5F076DFE3DEE1807089828A83E493F54D
:102D7600F0A3E208B5F062DFF4805E89828A83E020
:102D8600F5F0A3E608B5F051DFF5804D89828A8318
:102D9600E0F5F0A3E208B5F040DFF5803C89828AD1
:102DA60083E493F5F0A3E608B5F02EDFF4802A80DD
:102DB60002805789828A83ECFAE493F5F0A3C8C5AA
:102DC60082C8CCC583CCE0A3C8C582C8CCC583CC99
:102DD600B5F006DFE4DEE280007FFFB5F0020F22E9
:102DE60040027F012289828A83ECFAE0F5F0A3C8CB
:102DF600C582C8CCC583CCE0A3C8C582C8CCC58370
:102E0600CCB5F0D5DFE5DEE380CF89828A83ECFAA4
:102E1600E0F5F0A3C8C582C8CCC583CCE493A3C8AB
:102E2600C582C8CCC583CCB5F0AFDFE4DEE280A9AD
:102E360088F0EF60010E4E60ABED2402B404005042
:102E460098F582EB2402B40400508E232345822396
:102E5600902D2773EF4E6012EF60010EEDBB010B54
:102E660089828A83F0A3DFFCDEFA2289F05007F715
:102E760009DFFCA9F022BBFEFCF309DFFCA9F02266
:102E8600EF8DF0A4A8F0CF8CF0A428CE8DF0A42E60
:102E9600FE2278A37C097D017BFF7AE179AD122CB5
:102EA60093EF3395E04F700302C04678A37C097D0B
:102EB600017BFF7AE179B4122C93EF3395E04F70E2
:102EC60003024FEC78A37C097D017BFF7AE179C18F
:102ED600122C93EF3395E04F700302C7E178A37C81
:102EE600097D017BFF7AE179C6122C93EF3395E0D9
:102EF6004F70030291C878A37C097D017BFF7AE1BC
:102F060079CB122C93EF3395E04F700302ACD47853
:102F1600A37C097D017BFF7AE179D0122C93EF33F4
:102F260095E04F700302BB8E78A37C097D017BFF81
:102F36007AE179D8122C93EF3395E04F700302D9DA
:102F46004678A37C097D017BFF7AE179DC122C931C
:102F5600EF3395E04F700302D68F78A37C097D018D
:102F66007BFF7AE179E0122C93EF3395E04F700303
:102F760002652A78A37C097D017BFF7AE179EA1252
:102F86002C93EF3395E04F700302672E78A37C09EC
:102F96007D017BFF7AE179F2122C93EF3395E04FB6
:102FA60070030270B478A37C097D017BFF7AE17916
:102FB600F7122C93EF3395E04F700302631278A358
:102FC6007C097D017BFF7AE179FE122C93EF339524
:102FD600E04F70030275EC78A37C097D017BFF7AD4
:102FE600E27901122C93EF3395E04F70030235A777
:102FF60078A37C097D017BFF7AE27907122C93EF97
:103006003395E04F700302A5D078A37C097D017B40
:10301600FF7AE2790D122C93EF3395E04F7003029D
:10302600A66F78A37C097D017BFF7AE27913122CC7
:1030360093EF3395E04F700302BC0078A37C097DC3
:10304600017BFF7AE27919122C93EF3395E04F70EA
:1030560003026EDA78A37C097D017BFF7AE279238D
:10306600122C93EF3395E04F700302D96278A37C5C
:10307600097D017BFF7AE2792E122C93EF3395E0DE
:103086004F70030294F578A37C097D017BFF7AE2F9
:103096007938122C93EF3395E04F700302CC797890
:1030A600A37C097D017BFF7AE27944122C93EF33EE
:1030B60095E04F70030247B778A37C097D017BFF3B
:1030C6007AE2794A122C93EF3395E04F700302D9D6
:1030D6001078A37C097D017BFF7AE27951122C934B
:1030E600EF3395E04F700302D91978A37C097D016F
:1030F6007BFF7AE27957122C93EF3395E04F7003FA
:1031060002D6F678A37C097D017BFF7AE2795B1211
:103116002C93EF3395E04F700302D87778A37C09A0
:103126007D017BFF7AE27960122C93EF3395E04FB5
:10313600700302828078A37C097D017BFF7AE279A5
:1031460069122C93EF3395E04F7002801678A37CBA
:10315600097D017BFF7AE2796F122C93EF3395E0BC
:103166004F700302D30178A37C097D017BFF7AE2CD
:103176007975122C93EF3395E04F7002801678A381
:103186007C097D017BFF7AE2797A122C93EF3395E5
:10319600E04F700302591878A37C097D017BFF7A02
:1031A600E27983122C93EF3395E04F700280167804
:1031B600A37C097D017BFF7AE2798E122C93EF3393
:1031C60095E04F700302D3D078A37C097D017BFF85
:1031D6007AE27999122C93EF3395E04F700302A4AB
:1031E6009078A37C097D017BFF7AE279A4122C9367
:1031F600EF3395E04F700302A53078A37C097D017B
:103206007BFF7AE279B0122C93EF3395E04F70038F
:103216000288C878A37C097D017BFF7AE279C41213
:103226002C93EF3395E04F7003029CD778A37C096B
:103236007D017BFF7AE279D7122C93EF3395E04F2D
:10324600700302ABBA78A37C097D017BFF7AE27931
:10325600E3122C93EF3395E04F700302C83578A341
:103266007C097D017BFF7AE279F0122C93EF33958E
:10327600E04F700302D8AC78A37C097D017BFF7A0E
:10328600E279FA122C93EF3395E04F700302CD0AE0
:1032960078A37C097D017BFF7AE37909122C93EFF1
:1032A6003395E04F700302D89F78A37C097D017B9C
:1032B600FF7AE37913122C93EF3395E04F700302F4
:1032C600B7EB78A37C097D017BFF7AE37924122C86
:1032D60093EF3395E04F7003029B7A78A37C097DC8
:1032E600017BFF7AE37934122C93EF3395E04F702C
:1032F6000302D7B078A37C097D017BFF7AE3794C82
:10330600122C93EF3395E04F700302D7C178A37C5C
:10331600097D017BFF7AE37962122C93EF3395E006
:103326004F7003027AB278A37C097D017BFF7AE3B2
:10333600796E122C93EF3395E04F700302C58878AF
:10334600A37C097D017BFF7AE37980122C93EF330E
:1033560095E04F700302C8DB78A37C097D017BFFF3
:103366007AE3798C122C93EF3395E04F7003029D2C
:103376008478A37C097D017BFF7AE37999122C93EB
:10338600EF3395E04F7003028D6A78A37C097D01C7
:103396007BFF7AE379AA122C93EF3395E04F700303
:1033A60002AB2978A37C097D017BFF7AE379BA1207
:1033B6002C93EF3395E04F700302AC4778A37C095A
:1033C6007D017BFF7AE379C7122C93EF3395E04FAB
:1033D600700302B30E78A37C097D017BFF7AE37943
:1033E600CD122C93EF3395E04F700302B38C78A384
:1033F6007C097D017BFF7AE379DA122C93EF339512
:10340600E04F700302D46E78A37C097D017BFF7ABE
:10341600E379E9122C93EF3395E04F700302D70A54
:1034260078A37C097D017BFF7AE379FA122C93EF6E
:103436003395E04F700302CEA178A37C097D017B12
:10344600FF7AE47908122C93EF3395E04F7003026C
:10345600BCE178A37C097D017BFF7AE47910122C0C
:1034660093EF3395E04F7003029A1478A37C097D9D
:10347600017BFF7AE47918122C93EF3395E04F70B5
:103486000302A35078A37C097D017BFF7AE47921AE
:10349600122C93EF3395E04F700302A3F078A37CD0
:1034A600097D017BFF7AE4792A122C93EF3395E0AC
:1034B6004F700302D51B78A37C097D017BFF7AE45C
:1034C6007933122C93EF3395E04F700302D7D278FD
:1034D600A37C097D017BFF7AE47939122C93EF33C3
:1034E60095E04F700302B86578A37C097D017BFFE8
:1034F6007AE47941122C93EF3395E04F700302BDC5
:103506005078A37C097D017BFF7AE47949122C93DC
:10351600EF3395E04F700302D83C78A37C097D0118
:103526007BFF7AE47954122C93EF3395E04F7003C6
:10353600029F7F78A37C097D017BFF7AE479601284
:103546002C93EF3395E04F700302D03378A37C09B8
:103556007D017BFF7AE4796F122C93EF3395E04F70
:10356600700302D3F878A37C097D017BFF7AE479A6
:103576007A122C93EF3395E04F700302A84678A396
:103586007C097D017BFF7AE47982122C93EF3395D7
:10359600E04F700302B10C7BFF7AE4798A1243AAEA
:1035A60022901B47E0FCA3E0FDA3E0FEA3E024017C
:1035B600FFE43EFEE43DFDE43CFC901B47122A5C22
:1035C600901BA6122A6800000010E4901BA2F0A32C
:1035D600F0900987E070069009B374FFF0E4901B41
:1035E600A2F0A3F0900987E0FF901BA2E0FCA3E005
:1035F600FDC39FEC94004003023938901B6775F0B9
:1036060013ED122A99EC75F013A42583F583E0FED9
:10361600A3E024B3F58274093EAF82F5228F23908E
:103626001B5E75F013ED122A99EC75F013A4258331
:10363600F583E0FCA3E0FDA3E0FEA3E0F52F8E2ECC
:103646008D2D8C2C7F007E367D6E7C0112CF1B90DB
:103656001BA2E0FEA3E0FF901B6475F013122A99EB
:10366600EE75F013A42583F583E0FDD394017480F1
:10367600948050030238C77C00901B6975F013EFE5
:10368600122A99EE75F013A42583F583E0FEA3E0D4
:10369600FF1227A8901BA4ECF0A3EDF04C70369017
:1036A6001BA2E0FEA3E0FF901B6B75F013122A9994
:1036B600EE75F013A42583F583E07D0070027D018D
:1036C600901B6B75F013EF122A99EE75F013A42573
:1036D60083F583EDF0901BA2E0FEA3E0FF901B694B
:1036E60075F013122A99EE75F013A42583F583E479
:1036F60075F001122833901B5A75F013EF122A99B0
:10370600EE75F013A42583F583E0FCA3E0FDA3E0AA
:10371600FEA3E0FFE47BB0FAF9F8C3122A0570595C
:103726007F407E427D0FFC901BA2E0FAA3E0901B37
:103736005E75F013122A99EA75F013A42583F583B2
:10374600122A5C12D869901BA2E0FEA3E0901B6BC4
:1037560075F013122A99EE75F013A42583F583E00C
:10376600FF12D78E12D81E901BA4A3E0540F04900C
:103776001BAAF044B0F0023848901BA2E0FEA3E07A
:10378600901B5A75F013122A99EE75F013A425832F
:10379600F583E0FCA3E0FDA3E0FEA3E0FFE47BC02D
:1037A600FAF9F8C3122A057037901BA2E0FEA3E0CF
:1037B600901B6B75F013122A99EE75F013A42583EE
:1037C600F583E02482F582E43409F583E0FF901B5B
:1037D600A4A3E0FEEF4E04901BAAF044C0F0806262
:1037E600901BA2E0FEA3E0901B5A75F013122A99D3
:1037F600EE75F013A42583F583E0FCA3E0FDA3E0BA
:10380600FEA3E0FFE47BA17A16F9F8C3122A05703D
:1038160031901BA2E0FEA3E0901B6B75F013122AF9
:1038260099EE75F013A42583F583E02482F582E4EE
:103836003409F583E0FF901BA4A3E0FEEF4E901B36
:10384600AAF0901BA2E0FEA3E0901B5A75F013129B
:103856002A99EE75F013A42583F583E0FCA3E0FD19
:10386600A3E0FEA3E0540FFFE4FBFAF9F8C3122A23
:10387600057019E5232401FFE43522FE901BAAE01A
:10388600FB901BA2A3E0F52EE4FD8017E52324019F
:10389600FFE43522FE901BAAE0FB901BA2A3E0F5F5
:1038A6002E7D0112563F78AB7C1B7D017E007F0387
:1038B6001226D5901BAAE0852382852283A3F08059
:1038C60024E5232401FFE43522FE901BA2A3E0F5A4
:1038D6002E7B01E4FD12563F78AB7C1B7D017E00FA
:1038E6007F031226D5901BABE0852382852283F0C9
:1038F600901BA6E0F8A3E0F9A3E0FAA3E0FB901B77
:10390600ADE02401FF901BACE03400FEE4FCFDEBCF
:103916002FFFEA3EFEED39FDEC38FC901BA6122A7D
:103926005C901BA3E004F07006901BA2E004F0027A
:1039360035EA7E097FA3128021E4901BAAF0FF7E60
:103946000CFDFC901BA6E0F8A3E0F9A3E0FAA3E0C7
:10395600FBD3122A05400A7E097FA37D007C1080D6
:1039660046E4FF7E08FDFC901BA6E0F8A3E0F9A361
:10397600E0FAA3E0FBD3122A05400A7E097FA37D65
:10398600007C0C8022E4FF7E04FDFC901BA6E0F880
:10399600A3E0F9A3E0FAA3E0FBD3122A0540127EC6
:1039A600097FA37D007C0812D32C901BAAEFF08020
:1039B60005901BAAE4F012D832E4901BA2F0A3F003
:1039C600901BA2E0FEA3E0FFC3EE9404501F74A375
:1039D6002FF58274093EF583E0FF12D800901BA3F1
:1039E600E004F070DB901BA2E004F080D3E4FF7EDD
:1039F60004FDFC901BA6E0F8A3E0F9A3E0FAA3E01F
:103A0600FBC3122A055008901BAAE0FF12D800E457
:103A1600901BA2F0A3F0901BA2E0FEA3E0FFC3EE72
:103A26009404501C74A32FF58274093EF583E4F0C8
:103A3600901BA3E004F070DE901BA2E004F080D699
:103A46002212936A8F118E108D0F8C0E12C3C6EF41
:103A560060277D09AF16AE15129ACA7E087F007DD3
:103A6600007B017A007900122E5A74004400600926
:103A76007D12AF16AE15129ACAE4F522F52374002C
:103A86002523F58274003522F583E0FF74A22523F1
:103A9600F582741B3522F583EFF00523E5237002CA
:103AA60005226408452270D67E117F947D007B0135
:103AB6007A0979A3122E5A78A37C097D017B017AB3
:103AC6000079007E047F001226D5E4F52EF52F7FBF
:103AD600807E08FDFC1287CB7E097F607D007B011E
:103AE6007A007900122E5A12C3C6EF60097D09AF1B
:103AF60016AE15129ACA9000B8E09000CAF090006F
:103B0600B9E09000CBF09000BAE09000CCF09000C5
:103B1600BBE09000CDF09000BCE09000CEF09000AD
:103B2600BDE09000CFF09000BEE09000D0F090098C
:103B360091E0FF9000D3F0900992E0FE9000D4F05F
:103B4600900993E0FD9000D5F0900994E0FC900078
:103B5600D6F0900995E0FB9000D7F0900996E0F931
:103B66009000D8F0900997E0FA9000D9F0E4900020
:103B760031F0900025EFF0A3EEF0A3EDF0A3ECF00A
:103B8600A3EBF0A3E9F0A3EAF0900991E09000DC42
:103B9600F0900992E09000DDF0900993E09000DE4D
:103BA600F0900994E09000DFF0900995E09000E035
:103BB600F0A3E9F0900997E09000E2F07E087F001C
:103BC6007D007B017A0979A3122E5AE4F522F523AA
:103BD60074002523F58274003522F583E0FF74A373
:103BE6002523F58274093522F583EFF00523E523B5
:103BF60070020522B400D9E522B404D47E097FA35D
:103C06007DFE7C0312D32C900DA1EFF07B017A0987
:103C160079A37DFF7C0312CFFE900DA2EFF0E4FFA7
:103C2600FE12A2AFE4F52EF52F7F907E08FDFC1262
:103C360087CB7E087F007D007B017A0979A3122E4F
:103C46005AE5112470FFE51034F7FEE50F34FFFD49
:103C5600E50E34FFFCE4FB7A08F9F81228C48F2736
:103C66008E268D258C24780E122A3CE4F52EF52F0F
:103C76001287CBAF11AE10AD0FAC0EE4F52EF52FBB
:103C86001287CBAD19AC18AF16AE1512ADEBAD1948
:103C9600AC18AF16AE1512AE76900979E07E008E9E
:103CA60022F52375F020A4FF90097BE07C002FFD10
:103CB600EC35F0FC900978E02414FFEF7F0025E056
:103CC600FEEF2DFFEC3E901BCAF0A3EFF090097DAE
:103CD600E075F020A4FFA3E0C3137C002FFDEC35B4
:103CE600F0FC90097CE07F0033333354F8FEEF2D6F
:103CF600FFEC3E901BCCF0A3EFF078AA7C1B7D0175
:103D06007BFF7AE879A17E007F201226D5901BCC16
:103D1600E0FEA3E0F9901BB8F0EEFDA3F0901BCAFD
:103D2600E0FEA3E0901BBAF0EEFFFCA3F0901BCAE6
:103D3600A3E0FB901BBCF0A3ECF0901BC0E9F0A342
:103D4600EDF0A3EBF0A3EFF078A37C097D017B01F6
:103D56007A1B79AA7E007F201226D578AA7C1B7D45
:103D6600017BFF7AE879817E007F201226D5901BA1
:103D7600CCE0FEA3E0F9901BB8F0EEFDA3F0901B9B
:103D8600CAE0FEA3E0901BBAF0EEFFFCA3F0901B86
:103D9600CAA3E0FB901BBCF0A3ECF0901BC0E9F0BB
:103DA600A3EDF0A3EBF0A3EFF078C37C097D017BD4
:103DB600017A1B79AA7E007F201226D578AA7C1B61
:103DC6007D017BFF7AE879C17E007F201226D5909F
:103DD6001BCCE0FEA3E0F9901BB8F0EEFDA3F0903B
:103DE6001BCAE0FEA3E0901BBAF0EEFFFCA3F09026
:103DF6001BCAA3E0FB901BBCF0A3ECF0901BC0E930
:103E0600F0A3EDF0A3EBF0A3EFF078E37C097D01DE
:103E16007B017A1B79AA7E007F201226D59009FFA6
:103E2600E527F0FFAE26AD25AC247808122A16A3A6
:103E3600EFF0AF27AE26AD25AC247810122A16A3D4
:103E4600EFF0AF27AE26AD25AC247818122A16A3BC
:103E5600EFF0E4F522F52374A22523F582741B35D1
:103E660022F583E0700F74A22523F582741B352298
:103E7600F5837420F00523E52370020522640845C6
:103E86002270D4E4F522F52374A22523F582741B4F
:103E96003522F583E0FF74E32523F5827409352284
:103EA600F583EFF00523E523700205226408452219
:103EB60070D6E4F52EF52FFF7E08FDFC1287CB02A7
:103EC600CB9BC3E51C94085054901B47E0FCA3E031
:103ED600FDA3E0FEA3E02401FFE43EFEE43DFDE495
:103EE6003CFC901B47122A5C900981E0FBE4FAF93E
:103EF600F8901B47E0FCA3E0FDA3E0FEA3E0FF1261
:103F0600294FAC00AD01AE02AF03E4FBFAF9F8C3EA
:103F1600122A0570AD12728312815D80A512D968CE
:103F26007D02AF16AE15129ACA12C3C6E4FFFE741E
:103F3600002FF58274003EF583E0FD74A22FF58212
:103F4600741B3EF583EDF00FBF00010EEF64084EC3
:103F560070DD9000B8E09000CAF09000B9E09000E3
:103F6600CBF09000BAE09000CCF09000BBE090005F
:103F7600CDF09000BCE09000CEF09000BDE0900047
:103F8600CFF09000BEE09000D0F0900991E0FF9055
:103F960000D3F0900992E0FE9000D4F0900993E0EF
:103FA600FD9000D5F0900994E0F99000D6F09009C4
:103FB60095E09000D7F0900996E09000D8F090092F
:103FC60097E09000D9F0E4900031F0900025EFF0F2
:103FD600A3EEF0A3EDF0A3E9F0900995E0FF9000C1
:103FE60029F0900996E0FE90002AF0900997E0FDEE
:103FF60090002BF0900991E09000DCF0900992E09F
:104006009000DDF0900993E09000DEF0A3E9F0A3C4
:10401600EFF0A3EEF0A3EDF07E087F007D007B01BC
:104026007A0979A3122E5AE4FEFF74002FF58274E2
:10403600003EF583E0FD74A32FF58274093EF583F7
:10404600EDF00FBF00010EE4B507DFEEB404DB7E32
:10405600097FA37DFE7C0312D32C900DA1EFF07B8C
:10406600017A0979A37DFF7C0312CFFE900DA2EFA2
:10407600F0E4FFFE12A2AF12BA38E4F52EF52F7F58
:10408600907E08FDFC1287CB12C1E27B017A09798A
:10409600A312743AE4F52EF52F7F407E08FDFC123C
:1040A60087CB752E08752F007F417E087D007C002A
:1040B6001287CB7E087F007D007B017A0979A312E7
:1040C6002E5AE5112470FFE51034F7FEE50F34FF94
:1040D600FDE50E34FFFCE4FB7A08F9F81228C48FDC
:1040E600268E258D248C23E5112401F511E4351047
:1040F600F510E4350FF50FE4350EF50E12C245AD99
:1041060019AC18AF16AE1512ADEBAD19AC18AF164B
:10411600AE1512AE76900979E075F020A4FF9009ED
:104126007BE07C002FFDEC35F0FC900978E0241450
:10413600FFEF7F0025E0FEEF2DFFEC3E901BCAF05F
:10414600A3EFF090097DE075F020A4FFA3E0C31370
:104156007C002FFDEC35F0FC90097CE07F003333CA
:104166003354F8FEEF2DFFEC3E901BCCF0A3EFF09E
:1041760078AA7C1B7D017BFF7AE879A17E007F20EF
:104186001226D5901BCCE0FEA3E0F9901BB8F0EE0A
:10419600FDA3F0901BCAA3E0901BBAF0901BCAE0E7
:1041A600FF901BBBF0901BCAA3E0FE901BBCF0A3C4
:1041B600EFF0901BC0E9F0A3EDF0A3EEF0901BCA60
:1041C600E0901BC3F078A37C097D017B017A1B7903
:1041D600AA7E007F201226D578AA7C1B7D017BFF54
:1041E6007AE879817E007F201226D5901BCCE0FEEE
:1041F600A3E0F9901BB8F0EEFDA3F0901BCAA3E074
:10420600901BBAF0901BCAE0FF901BBBF0901BCA34
:10421600A3E0FE901BBCF0A3EFF0901BC0E9F0A357
:10422600EDF0A3EEF0901BCAE0901BC3F078C37CC0
:10423600097D017B017A1B79AA7E007F201226D593
:1042460078AA7C1B7D017BFF7AE879C17E007F20FE
:104256001226D5901BCCE0FEA3E0F9901BB8F0EE39
:10426600FDA3F0901BCAA3E0901BBAF0901BCAE016
:10427600FF901BBBF0901BCAA3E0FE901BBCF0A3F3
:10428600EFF0901BC0E9F0A3EDF0A3EEF0901BCA8F
:10429600E0901BC3F078E37C097D017B017A1B79F2
:1042A600AA7E007F201226D59009FFE526F0FFAEF4
:1042B60025AD24AC237808122A16A3EFF0AF26AE5C
:1042C60025AD24AC237810122A16A3EFF0AF26AE44
:1042D60025AD24AC237818122A16A3EFF0E4FEFFCE
:1042E60074A22FF582741B3EF583E0700D74A22F25
:1042F600F582741B3EF5837420F00FBF00010EEFAC
:1043060064084E70DBE4FEFF74A22FF582741B3E38
:10431600F583E0FD74E32FF58274093EF583EDF035
:104326000FBF00010EEF64084E70DDE4F52EF52F89
:10433600FF7E08FDFC1287CB12D37F9009687403B9
:10434600F022E54A2436F8E6054A22783330070299
:104356007836E475F001122AA50226FB2000EB7FD1
:104366002ED2008018EF540F2490D43440D4FF305E
:10437600040BEF24BFB41A0050032461FFE54B6021
:1043860002154B054EE54E7002054D30070D78338C
:10439600E475F001122AA5EF02277402D80F740300
:1043A600D2078003E4C207F54A8B338A348935E4A1
:1043B600F54BF54DF54EE54B60077F2012438380A4
:1043C600F5754CFFC201C200C202C203C205C20695
:1043D600C208124351FF700D3007057F0012439447
:1043E600AF4EAE4D22B4255FC2D5C204124351FF73
:1043F60024D0B40A00501A75F00A784B30D5050857
:10440600B6FF0106C6A426F620D5047002D20380A4
:10441600D924CFB41A00EF5004C2E5D20402468173
:10442600D20180C6D20080C0D20280BCD2D580BA6A
:10443600D20580B47F201243832002077401B54B56
:104446000040F1124348FF1243830243BCD208D214
:10445600068095124348FB124348FA124348F94A2C
:104466004B700679787A477BFF20022EE54B602A4F
:104476007E008E8275830012271460060EEE654C50
:1044860070F0C2D5EBC0E0EAC0E0E9C0E0EE12464B
:10449600E1D0E0F9D0E0FAD0E0FB1226FBFF60AAFB
:1044A600EBC0E0EAC0E0E9C0E0124383D0E02401BB
:1044B600F9D0E03400FAD0E0FBE54C0460DCD54CE2
:1044C600D98087D20280A21246C460F7E54C7001FB
:1044D60004122463A94C600DE54C600914F54C12D6
:1044E600476BEF60F3EA30E702F404C3995077EACA
:1044F600F4254C0430E701E404F54C800D1246C463
:1045060060C1EA054C254C122463EA7849F630E787
:1045160001E4254C04D54C04200501141246E1E4BF
:10452600C0E012476B7849E6601320E70714F612DD
:10453600436B802204F6D0E014C0E07F0012436B88
:10454600E54C6007124362154C800B30050312439D
:1045560062D0E00243BCD0E00480C51246C460A02D
:10456600E54C041224637849EAF6E54C200502601E
:10457600010424041246E174FF04C0E012476B12E2
:10458600436BE54C2005026003124362D0E0B54C54
:10459600E87F451243757849E67F2B30E7047F2D87
:1045A600F404C0E0124383D0E075F00A84C0F01230
:1045B600436CD0E012436C0243BC79108002790848
:1045C600C206C2088008D2D5790A8004790AC2D503
:1045D600E54C047002F54CE4FAFDFEFF124348FC7C
:1045E6007B08200113124348FD7B1030000A12435A
:1045F60048FE124348FF7B20EC3382D592D55013F8
:10460600C3E43000069FFFE49EFEE42001039DFD07
:10461600E49CFCE4CBF8C201EC700CCFCECDCCE828
:1046260024F8F870F38017C3EF33FFEE33FEED3353
:10463600FDEC33FCEB33FB994002FB0FD8E9EB3082
:104646000105F8D0E0C448B201C0E00AEC4D4E4F77
:1046560078207B0070C2EAB54C0040BCC0E0124630
:10466600E3D0F0D0E0200104C4C0E0C4B201C0F041
:1046760012436CD0F0D5F0EB0243BC122AB5445974
:104686005345C058442A4C44264245C44F45CC4461
:1046960045CC49443F4345D25545034645614544CB
:1046A600CD47479850442E2D44322E44552B443640
:1046B6002344532047812A43EE480000444DE54CED
:1046C600B4FF03754C06124348FC124348FD1243DF
:1046D60048FE124348FF7842022492790AA2D52066
:1046E6000314300509B910020404B9080104A2D55F
:1046F6002006025001042002689202B54B00503495
:10470600C0E07F203003197F30A202720672055086
:104716000F12473AC202C206C205C2087F30800F96
:10472600300503E9C0E0124383300503D0E0F9D039
:10473600E0B54BCC3005177F30B9100C1243837FA0
:10474600583004077F788003B90803124383300288
:10475600057F2D0243837F202008F87F2B2006F358
:1047660022920280CF7F00B4070050052442F8E66B
:10477600FF22286E756C6C2900D201124348300165
:10478600F8C201784B30D50108F60243EE2D5043AE
:1047960049581243482403B405004001E490479366
:1047A60093124374743A124374D203754B04024550
:1047B600C0E4901BA2F0A3F0901BA2E0FEA3E024AD
:1047C600A3F58274093EF583E06010901BA3E00414
:1047D600F070E5901BA2E004F080DD901BA3E004DE
:1047E600F07006901BA2E004F0901BA2E0FEA3E08E
:1047F60024A3F974093EFA7B01129C29901BA6EEAC
:10480600F0A3EFF0EE6003024BF2EF14B40D00409C
:1048160003024BF290482875F003A4C58325F0C522
:10482600837302484F024889024A92024AA2024A08
:10483600C0024ADD024B5D024B87024B8B024B9056
:10484600024B94024BF2024B9A1297F090097EE0CB
:10485600FF901BA4E4F0A3EFF07FD07E0712D132C5
:10486600AD19AC18AF16AE1512AE7690097EE0FF04
:10487600901BA4E07003A3E06F7F317003024AD758
:10488600024B8D12D96890097CE0FFE4FCFDFE7BAB
:104896003CFAF9F81228C4A804A905AA06AB0790A1
:1048A600097DE0FFE4FCFDFEEB2FFFEE3AFEED395D
:1048B600FDEC38FC901BA8122A5C901BA8E0FCA318
:1048C600E0FDA3E0FEA3E0FFE47B3CFAF9F8122842
:1048D600C4901BA8122A5C901BA8E0F8A3E0F9A3D9
:1048E600E0FAA3E0FB90097EE0FFE4FCFDFEEB2F7F
:1048F600FFEE3AFEED39FDEC38FC901BA8122A5C5F
:10490600901BA8E0FCA3E0FDA3E0FEA3E02408FFC3
:10491600E43EFEE43DFDE43CFC901BA8122A5CE468
:104926007B3CFAF9F8901BA8E0FCA3E0FDA3E0FEAF
:10493600A3E0FF12294FAC00AD01AE02AF03901BFE
:10494600AC122A5C901BACA3A3A3E090098EF09056
:104956001BA8E0FCA3E0FDA3E0FEA3E0FFA3E0F8B4
:10496600A3E0F9A3E0FAA3E0FBC3EF9BFFEE9AFEF8
:10497600ED99FDEC98FC901BA8122A5C901BA8E010
:10498600FCA3E0FDA3E0FEA3E0FFE47B3CFAF9F81C
:1049960012294F901BA8122A5CE47B3CFAF9F89086
:1049A6001BA8E0FCA3E0FDA3E0FEA3E0FF12294F55
:1049B600AC00AD01AE02AF03901BAC122A5C901B9B
:1049C600ACA3A3A3E090098DF0901BA8E0FCA3E0A4
:1049D600FDA3E0FEA3E0FFA3E0F8A3E0F9A3E0FA5D
:1049E600A3E0FBC3EF9BFFEE9AFEED99FDEC98FC6E
:1049F600901BA8122A5C901BA8E0FCA3E0FDA3E094
:104A0600FEA3E0FFE47B3CFAF9F812294F901BA8BD
:104A1600122A5C901BA8A3A3A3E0FF90098CF0A325
:104A2600E0FDA3E0FB12CF8F900978E0FFA3E0FD45
:104A360090097BE0FB90097AE0F52512CC2F12D580
:104A4600D012D6E212D95112D744E47FF87E2AFD5D
:104A5600FCAB0DAA0CA90BA80AC3122A057F0050AD
:104A6600027F01E5147E0070027E01EF5E70DB12AC
:104A7600D8DC12D95512D5E9E51464017F327005E8
:104A860012D27E800312D2AAE4F5142212B6F6ECF4
:104A96004D4E4F7F337003024B8D803512BAAAEF0D
:104AA600701312BB1CEF700D12CA1CEF7F3470031B
:104AB600024B8D801C7F34024B5812BAAAEF70133A
:104AC60012BB1CEF700D12CA1CEF7F357003024B30
:104AD6008D807F7F35807BE4901BA2F0A3F0901B36
:104AE600AC122A6800000000E4FFFE7D0FFC901B5C
:104AF600ACE0F8A3E0F9A3E0FAA3E0FBC3122A05B1
:104B0600503F901BACE0FCA3E0FDA3E0FEA3E0FF5A
:104B1600129739901BA3E02FF0901BA2E03EF09075
:104B26001BACE0FCA3E0FDA3E0FEA3E02400FFEE47
:104B36003401FEE43DFDE43CFC901BAC122A5C8093
:104B4600A7C3901BA3E0945A901BA2E094007F3663
:104B5600400302D2AA8030E4901BA6F0A3F0FF1215
:104B6600D663E4752F80752E25F52DF52CFF7E3640
:104B76007D6E7C0112CF1B7F3712D27E7F0102D65B
:104B8600637F3880027F3902D27E7D3080027D319C
:104B96007F318052E4901BA2F0A3F0FF12D663127D
:104BA6007283D3901B3EE09488901B3DE0941340A3
:104BB60008901BA2E4F0A304F07F0112D6631272E0
:104BC60083C3901B3EE09488901B3DE094135008ED
:104BD600901BA2E4F0A304F0901BA2E07002A3E0F5
:104BE6007D337F31700302D16412D1942212C42125
:104BF600EF7003024C9012D96812C3C6EF60097DAC
:104C060009AF16AE15129ACA900991E09000CAF043
:104C1600900992E09000CBF0900993E09000CCF0E0
:104C2600900994E09000CDF0900995E09000CEF0C8
:104C3600900996E09000CFF0900997E09000D0F0B0
:104C46007E087F007D007B017A0979A3122E5A78AF
:104C5600A37C097D017B017A0079007E047F001226
:104C660026D57E097FA37DFE7C0312D32C900DA151
:104C7600EFF07B017A0979A37DFF7C0312CFFE90CA
:104C86000DA2EFF0E4FFFE12A20E12C3C6EF6009FA
:104C96007D09AF16AE15129ACA7B017A0079137D8B
:104CA6000412C368E47B7DFAF9F812294F90098152
:104CB600EFF0700F7D24AF16AE15129ACA900981D7
:104CC6007402F07B017A0079177D0212C36890099D
:104CD60085EEF0A3EFF09003BDE0900987F0D39442
:104CE6000374809480400F7D24AF16AE15129ACAC5
:104CF6009009877403F0E4F524F525900987E0FF11
:104D0600C3E5259FE52494004003024F24E525C40E
:104D1600F8540FC868FFE524C454F048FE74BE2F4B
:104D2600F974033EFA7B017D0412C368901B5A7521
:104D3600F013E525122A99E52475F013A42583F5C9
:104D460083122A5CE525C4F8540FC868FFE524C41D
:104D560054F048FE74C22FF974033EFA7B017D04B9
:104D660012C368901B5E75F013E525122A99E52497
:104D760075F013A42583F583122A5CE525C4F8543F
:104D86000FC868FFE524C454F048FE74C62FF974B2
:104D9600033EFA7B017D0212C368901B6275F01315
:104DA600E525122A99E52475F013A42583F583EEEB
:104DB600F0A3EFF0E525C4F8540FC868FFE524C456
:104DC60054F048FE74C82FF58274033EF583E0FD67
:104DD600901B6475F013E525122A99E52475F013E6
:104DE600A42583F583EDF074C92FF974033EFA7B8D
:104DF600017D0212C368E5252FFFE5243EFE901BC8
:104E06006775F013E525122A99E52475F013A42594
:104E160083F583EEF0A3EFF0901B6B75F013E52599
:104E2600122A99E52475F013A42583F5837401F0FD
:104E3600901B6975F013E525122A99E52475F01380
:104E4600A42583F583E4F0A3F0901B5A75F013E5CF
:104E560025122A99E52475F013A42583F583E0FC31
:104E6600A3E0FDA3E0FEA3E0FF122ADB4E880000CC
:104E760000B04EB9000000C04EFB000016A10000B5
:104E86004F199000A8E0FF7E00700790098274BC5D
:104E9600800BEF64014E700A90098274BDF0A3F096
:104EA6008071EF64024E706B90098274BCF0A304AB
:104EB600F080609000A8E0FD75F00A84FE25E025EC
:104EC600E0540C900982F0ED75F00A84AFF0EF25FE
:104ED600E025E0540CA3F09000B1E0FF901B6C7548
:104EE600F013E525122A99E52475F013A42583F518
:104EF60083EFF0801E9000A8E0FD75F00A84FEC4E2
:104F06005470900982F0ED75F00A84AFF0EFC45446
:104F160070A3F00525E52570020524024D01E4F590
:104F26001CF51D901B47122A680000000075080931
:104F36007509A3E4900975F0A3F0900974F0F524BF
:104F4600F525900987E0FFC3E5259FE524940040F9
:104F560003024FEB901B5A75F013E525122A99E5CB
:104F66002475F013A42583F583E0FCA3E0FDA3E0FC
:104F7600FEA3E0FFE47BC0FAF9F8C3122A05705AD3
:104F8600901B5E75F013E525122A99E52475F0133A
:104F9600A42583F583E0FCA3E0FDA3E0FEA3E0FFE8
:104FA600752F00752E36752D6E752C0112CF1B12BE
:104FB600D869901B6C75F013E525122A99E52475BE
:104FC600F013A42583F583E0FF12D78E12D81E7F37
:104FD600407E0D7D037C0012D55C0525E52570021B
:104FE6000524024F4822901BA5745FF0742E2409F5
:104FF600F582E434DEF583E493F9901BA6F0742E73
:10500600240AF582E434DEF583E493FF901BA7F0CF
:10501600A3742EF090DE2EE493FE644F6009EE64D6
:105026004E6004EEB444047E3180027E30901BA9AB
:10503600EEF090DE2EE493B44A17A3E493B4611124
:1050460015827583DEA3A3E493B46E057E31025107
:105056002C90DE2EE493FEB446057E3202512CEEF1
:10506600B44D1A90DE2EA3E493B4611115827583B4
:10507600DEA3A3E493B472057E3302512C90DE2E98
:10508600E493B4410BA3E493B470057E3402512C2F
:1050960090DE2EE493FEB44D16A3E493B46110158E
:1050A600827583DEA3A3E493B479047E358077EE1C
:1050B600B44A1990DE2EA3E493B475101582758355
:1050C600DEA3A3E493B46E047E36805A90DE2EE40B
:1050D60093B44A16A3E493B4751015827583DEA3C0
:1050E600A3E493B46C047E37803C90DE2EE493FEFA
:1050F600B4410AA3E493B475047E388029EEB45310
:10510600047E39802190DE2EE493FEB44F047E3077
:105116008014EEB44E047E31800C90DE2EE4937E35
:105126003FB444027E32901BAAEEF0742E2404F59E
:1051360082E434DEF583E493FEFD3395E0FCC3EDB3
:105146009430EC64809480400280027E30901BABE9
:10515600EEF0E4A3F0C3ED9430EC6480948040104C
:10516600742E2404F582E434DEF583E493FE800293
:105176007E30901BADEEF0742E2405F582E434DE0D
:10518600F583E493901BAEF0A3742EF090DE2EE42C
:1051960093FE644F6009EE644E6004EEB444047EF0
:1051A6003180027E30901BB0EEF090DE2EE493B498
:1051B6004A17A3E493B4611115827583DEA3A3E4B1
:1051C60093B46E057E310252A490DE2EE493FEB4B3
:1051D60046057E320252A4EEB44D1A90DE2EA3E4AA
:1051E60093B4611115827583DEA3A3E493B47205AB
:1051F6007E330252A490DE2EE493B4410BA3E493D3
:10520600B470057E340252A490DE2EE493FEB44DB3
:1052160016A3E493B4611015827583DEA3A3E49309
:10522600B479047E358077EEB44A1990DE2EA3E475
:1052360093B4751015827583DEA3A3E493B46E044C
:105246007E36805A90DE2EE493B44A16A3E493B4D5
:10525600751015827583DEA3A3E493B46C047E37C0
:10526600803C90DE2EE493FEB4410AA3E493B47529
:10527600047E388029EEB453047E39802190DE2ED8
:10528600E493FEB44F047E308014EEB44E047E31B7
:10529600800C90DE2EE4937E3FB444027E32901B57
:1052A600B1EEF0A3742EF0A3E9F0A3EFF0E4A3F0BF
:1052B60078A37C097D017BFF7AE17988FE7F08125D
:1052C60026D578AB7C097D017B017A1B79AD7E0002
:1052D6007F091226D578B47C097D017BFF7AE179B6
:1052E600807E007F081226D5E4901BA4F07E097FFD
:1052F600A37D19FC12D32C901BA4EFF012D832E434
:10530600901BA2F0A3F0901BA2E0FEA3E0FFC394C3
:1053160019EE9400501F74A32FF58274093EF5838D
:10532600E0FF12D800901BA3E004F070D9901BA2F6
:10533600E004F080D1901BA4E0FF02D800E4F5223F
:10534600F523900987E0FFC3E5239FE522940040FB
:1053560003025639901B6775F013E523122A99E567
:105366002275F013A42583F583E0FEA3E0FF74B352
:10537600251DF5827409351CF583E5822FF582E536
:10538600833EAF82F5268F27901B5E75F013E523CB
:10539600122A99E52275F013A42583F583E0FCA370
:1053A600E0FDA3E0FEA3E0F52F8E2E8D2D8C2C7F45
:1053B600007E367D6E7C0112CF1B901B6475F01348
:1053C600E523122A99E52275F013A42583F583E0D7
:1053D600FFD39401748094805003025616EFFD7C2F
:1053E60000901B6975F013E523122A99E52275F0E2
:1053F60013A42583F583E0FEA3E0FF1227A88D24DE
:10540600E5247033901B6B75F013E523122A99E59A
:105416002275F013A42583F583E07F0070027F01D7
:10542600901B6B75F013E523122A99E52275F0138C
:10543600A42583F583EFF0901B6975F013E523121D
:105446002A99E52275F013A42583F583E475F00106
:10545600122833901B5A75F013E523122A99E52278
:1054660075F013A42583F583E0FCA3E0FDA3E0FE1D
:10547600A3E0FFE47BB0FAF9F8C3122A05602E9088
:105486001B5E75F013E523122A99E52275F013A425
:105496002583F583E0FCA3E0FDA3E0FEA3E0FF7B0C
:1054A600407A42790F7800C3122A05704612D869ED
:1054B600901B6B75F013E523122A99E52275F013FC
:1054C600A42583F583E02482F582E43409F583E09C
:1054D600FF12D78E12D81EE4FFFE0FBF00010EBECC
:1054E6001FF8BF40F5E524540F04F5254325B0E425
:1054F6000255A0901B5A75F013E523122A99E5224E
:1055060075F013A42583F583E0FCA3E0FDA3E0FE7C
:10551600A3E0FFE47BC0FAF9F8C3122A05702A90CB
:105526001B6B75F013E523122A99E52275F013A477
:105536002583F583E02482F582E43409F583E0458A
:105546002404F5254325C08051901B5A75F013E5B8
:1055560023122A99E52275F013A42583F583E0FC2E
:10556600A3E0FDA3E0FEA3E0FFE47BA17A16F9F831
:10557600C3122A057024901B6B75F013E523122ABB
:1055860099E52275F013A42583F583E02482F5823C
:10559600E43409F583E04524F525901B5A75F0138C
:1055A600E523122A99E52275F013A42583F583E0F5
:1055B600FCA3E0FDA3E0FEA3E0540FFFE4FBFAF931
:1055C600F8C3122A057012E5272401FFE43526FEEA
:1055D60085232EAB25E4FD8010E5272401FFE43565
:1055E60026FE85232EAB257D0112563F78A27C1B15
:1055F6007D017E007F031226D5852782852683A31B
:10560600E525F0901BA2E0852782852683F0801889
:10561600AD23AC22AF27AE2612D09B78A27C1B7D91
:10562600017E007F031226D50523E523700205229D
:10563600025348901BA2E0FF228E2A8F2B8D2C8BC3
:105646002D78B07C1B7D017BFF7AE979247E007F73
:10565600031226D5E4F52FE52E75F013A4245EF586
:1056660082E4341BF583E0FCA3E0FDA3E0FEA3E0A7
:10567600FF122ADB568400002580000056FFE52E27
:1056860075F013A4245EF582E4341BF583E0F8A3D9
:10569600E0F9A3E0FAA3E0FB7F807E967D987C008C
:1056A60012294FE47BFAFAF9F812294FE47B02FA41
:1056B600F9F8D3122A054008E47F02FEFDFC802E8D
:1056C600E52E75F013A4245EF582E4341BF583E021
:1056D600F8A3E0F9A3E0FAA3E0FB7F807E967D982D
:1056E6007C0012294FE47BFAFAF9F812294FEF24CD
:1056F6000AF531E43EF5308074E52E75F013A424E6
:105706005EF582E4341BF583E0F8A3E0F9A3E0FA42
:10571600A3E0FB7F807E967D987C0012294FE47B78
:10572600FAFAF9F812294FE47B02FAF9F8D3122AA9
:10573600054008E47F02FEFDFC802EE52E75F01381
:10574600A4245EF582E4341BF583E0F8A3E0F9A314
:10575600E0FAA3E0FB7F807E967D987C0012294FBD
:10576600E47BFAFAF9F812294F8E308F3112D86994
:10577600E52E75F013A4245AF582E4341BF583E074
:10578600FCA3E0FDA3E0FEA3E4FFE4FBFAF9F8C303
:10579600122A05704AE52E75F013A4245AF582E400
:1057A600341BF583A3A3A3E0FBEB452DFFE4901B7D
:1057B600B3EFF0E52E75F013A4245EF582E4341BF6
:1057C600F583E0FCA3E0FDA3E0FEA3E0FF7B407AC7
:1057D60042790F7800C3122A05901BB302587AE566
:1057E6002E75F013A4245AF582E4341BF583A3A383
:1057F600E0FEA3E4FFE4FDFC7808122A16901BB332
:10580600EFF0E52E75F013A4245AF582E4341BF567
:1058160083A3A3A3E0FFE4901BB4EFF0E52C603173
:10582600A3E52DF07E1B7FB37D037C0012D32C9065
:105836001BB6EFF0901BB3E0FF12D78E901BB4E0BF
:10584600FF12D78E901BB5E0FF12D78E901BB68045
:10585600237E1B7FB37D027C0012D32C901BB5EFF9
:10586600F0901BB3E0FF12D78E901BB4E0FF12D767
:105876008E901BB5E0FF12D78E12D81EAB2BAA2A2C
:10588600AD31AC307F647E0012C530901BB1EEF0B6
:10589600A3EFF04E7007901BB07403806DE52E7574
:1058A600F013A4245AF582E4341BF583E0FCA3E04C
:1058B600FDA3E0FEA3E4FFE4FBFAF9F8C3122A0510
:1058C600702CF52FFFFED3901BB2E09F901BB1E02A
:1058D6009E4016E52B2FF582E52A3EF583E0252F1F
:1058E600F52F0FBF00010E80DD532F7F8011901B17
:1058F600B1E0FCA3E0FDAF2BAE2A12D32C8F2FE52F
:105906002F7F017001FF901BB0EFF07B017A1B79AE
:10591600B022E4901BA2F0A3F0901BA2E475F00164
:10592600122849FE74A325F0F58274093EF583E03A
:1059360070E7901BA2E0FEA3E024A3F974093EFAE7
:105946007B01129013901BA4122A5CE4FFFEFDFC5F
:10595600901BA4E0F8A3E0F9A3E0FAA3E0FBC312CE
:105966002A05704A12CB4F7E097FA37D007C041264
:10597600D32C8F2212D832E4901BA2F0A3F0901BF6
:10598600A2E0FEA3E0FFC3EE9404501F74A32FF51C
:105996008274093EF583E0FF12D800901BA3E00451
:1059A600F070DB901BA2E004F080D3025BD7E47BAF
:1059B60002FAF9F8901BA4E0FCA3E0FDA3E0FEA325
:1059C600E0FF12294FEF24FFFFEE34FFFEED34FF18
:1059D600FDEC34FFFC901BA8122A5C90096CE06475
:1059E600017038FF7E08FDFC901BA8E0F8A3E0F9E3
:1059F600A3E0FAA3E0FBD3122A05401F901BA8E000
:105A0600FCA3E0FDA3E0FEA3E02470FFE43EFEE479
:105A16003DFDE43CFC901BA8122A5C901BA8E0FC10
:105A2600A3E0FDA3E0FEA3E0FF12B504EF600302CE
:105A36005BDC901BA8E0FCA3E0FDA3E0FEA3E0FF77
:105A4600122ADB5A5F000000005AA5000008005A1F
:105A5600DC0000089000005AE2E4901BA2F0A3F0DC
:105A6600901BA2E0FEA3E0FF2400F58274003EF541
:105A760083E0FD74A32FF58274093EF583EDF09063
:105A86001BA3E004F07006901BA2E004F0901BA29A
:105A9600E0B404CCA3E0B400C712D250025B93E496
:105AA600901BA2F0A3F0901BA2E0FEA3E0FFC3EEC2
:105AB6009404501C74A32FF58274093EF583E4F018
:105AC600901BA3E004F070DE901BA2E004F080D6E9
:105AD60012A0CA025B9312D1C4025B93901BA4A3CB
:105AE600A3A3E05401FFE4FEFDFCFBFAF9F8C312A0
:105AF6002A057041901BA2F0A3F0901BA2E0FEA322
:105B0600E0FF2400F58274003EF583E0FD74A32FC8
:105B1600F58274093EF583EDF0901BA3E004F07066
:105B260006901BA2E004F0901BA2E0B404CCA3E014
:105B3600B400C78058901BA4A3A3A3E05401FFE4BC
:105B4600FEFDFCFBFAF9F8C3122A056040E4901B3F
:105B5600A2F0A3F0901BA2E0FEA3E0FF2400F582D2
:105B660074043EF583E0FD74A32FF58274093EF5B7
:105B760083EDF0901BA3E004F07006901BA2E004F6
:105B8600F0901BA2E0B404CCA3E0B400C77E097F6A
:105B9600A37D007C0412D32C8F2212D832E4901BF2
:105BA600A2F0A3F0901BA2E0FEA3E0FFC3EE9404D4
:105BB600501F74A32FF58274093EF583E0FF12D8B7
:105BC60000901BA3E004F070DB901BA2E004F080C1
:105BD600D3AF2212D80022901CDEE0FF90097EE0AF
:105BE600FE6F7003025CB2901CDEEEF0901CC4E007
:105BF600FCA3E0FDA3E0FEA3E02401FFE43EFEE4F7
:105C06003DFDE43CFC901CC4122A5C901CC8E0FCE0
:105C1600A3E0FDA3E0FEA3E02401FFE43EFEE43D95
:105C2600FDE43CFC901CC8122A5C901CCCE0FCA352
:105C3600E0FDA3E0FEA3E02401FFE43EFEE43DFD1B
:105C4600E43CFC901CCC122A5C901CD0E0FCA3E047
:105C5600FDA3E0FEA3E02401FFE43EFEE43DFDE4F7
:105C66003CFC901CD0122A5C901CD4E0FCA3E0FD06
:105C7600A3E0FEA3E02401FFE43EFEE43DFDE43C98
:105C8600FC901CD4122A5C901CD8E0FCA3E0FDA377
:105C9600E0FEA3E02401FFE43EFEE43DFDE43CFC1F
:105CA600901CD8122A5C901CDDE004F0D3901B38BF
:105CB600E094E8901B37E09403403AE47F107E0EB0
:105CC600FDFC901CC8E0F8A3E0F9A3E0FAA3E0FB12
:105CD600D3122A05401F901CC8122A680000000033
:105CE6007527FF7528E87529E1901B37E0FAA3E0D0
:105CF600FB7D05804EC3901B3EE09488901B3DE0E3
:105D060094135051E47F107E0EFDFC901CD4E0F8F5
:105D1600A3E0F9A3E0FAA3E0FB122A054037901CA2
:105D2600D4122A6800000000901B3FE0FAA3E0FBB3
:105D3600C39488EA941350147527FF7528E87529CB
:105D4600E57D0EAF16AE1512793380097D0FAF16BD
:105D5600AE15129ACAC3901B38E0941E901B37E00A
:105D66009400503EE47F107E0EFDFC901CCCE0F8C3
:105D7600A3E0F9A3E0FAA3E0FB122A054024901C55
:105D8600CC122A68000000007527FF7528E87529DF
:105D9600E1901B37E0FAA3E0FB7D06AF16AE1512C5
:105DA6007933901B55E06403702D7F107E0EFDFC49
:105DB600901CC4E0F8A3E0F9A3E0FAA3E0FBD31239
:105DC6002A054013901CC4122A68000000007D04B6
:105DD600AF16AE15129ACA901B55E06401702D7F5E
:105DE600107E0EFDFC901CD0E0F8A3E0F9A3E0FACB
:105DF600A3E0FBD3122A054013901CD0122A680098
:105E06000000007D07AF16AE15129ACAC3901B3A62
:105E1600E094E0901B39E0942E503EE47F087E0724
:105E2600FDFC901CD8E0F8A3E0F9A3E0FAA3E0FBA0
:105E3600122A054024901CD8122A6800000000751A
:105E460027FF7528E87529E5901B39E0FAA3E0FBE2
:105E56007D10AF16AE15127933C3901B40E09488BF
:105E6600901B3FE094135026901CDCE0700804F071
:105E7600E4A3F0FF8015901CDDE0D39402748094B7
:105E860080400BE4F0901CDCF07F0112D66322E523
:105E960063656270030260DAAF62056274002FF513
:105EA60082E43400F583E0F522E55E600302605C7F
:105EB600E52224F6606424FD7003025FCA24ED60C7
:105EC6004024F5601D24F17003025FDA24FD606949
:105ED60024CA6058246B6003026042E4F558F55901
:105EE60080AD0559E559AE58700205581424A3F53E
:105EF6008274093EF583E4F0F55CF55D755E01801C
:105F06008E0559E559AE58700205581424A3F5823A
:105F160074093EF583E4F0025E9574A32559F58273
:105F260074093558F583E4F0F55EFF220559E55905
:105F3600AE587002055802604C0559E559AE5870C6
:105F46000205581424A3F58274093EF583E4F0751E
:105F56005E01755F01F55AF55BF55CF55D74A32589
:105F66005BF5827409355AF583E0600A055BE55BEB
:105F760070EB055A80E7055BE55B7002055A74A372
:105F8600255BF5827409355AF583E0600A055BE501
:105F96005B70EB055A80E7055BE55B7002055A749A
:105FA600A3255BF5827409355AF583E0600A055B23
:105FB600E55B70EB055A80E7055BE55B7002055A09
:105FC60024A3806674A32559F58274093558F58390
:105FD600E4F0FF220559E559AE587002055814241D
:105FE600A3F58274093EF583E4F0755E01755F01E1
:105FF600F55AF55BF55CF55D055BE55BAE5A70023F
:10600600055A1424A3F58274093EF583E070E90568
:106016005BE55BAE5A7002055A1424A3F582740937
:106026003EF583E070E974A3255BF97409355AFAE5
:106036007B01129C298E608F61025E950559E55998
:10604600AE58700205581424A3F58274093EF583F0
:10605600E522F0025E95E55F6034055DE55D700260
:10606600055C0559E559AE58700205581424A3F588
:106076008274093EF583E522F0C3E55D9561E55C32
:1060860095605003025E95E4F55EF55F8030055D30
:10609600E55D7002055C0559E559AE587002055874
:1060A6001424A3F58274093EF583E522F0C3E55D69
:1060B6009401E55C94045003025E95E4F55E74A3D6
:1060C6002559F58274093558F583E522F0E4F5582B
:1060D600F559FF227F01228E2F8F308D318A328B28
:1060E6003312AF808F3A8E398D388C377F007E40E1
:1060F6007D017C00AB3AAA39A938A837C3122A0514
:1061060040030263117E007F407D007B017A1C798B
:1061160022122E5A7E007F0C7D007B017A1C791696
:10612600122E5A853082852F83A3A3A3E0C3940A37
:1061360074809480500D7E1C7F227BFF7ADD79FF70
:1061460012A7B5853082852F83A3A3A3E0FF7E0027
:106156007B017A1C7916127D8112A7AB12C9CE85F6
:106166003082852F83A3E0C3940A74809480500DF7
:106176007E1C7F227BFF7ADD79FF12A7B5853082F0
:10618600852F83A3E0FF7E007B017A1C7916127DA2
:106196008112A7AB12C9CE853082852F83E0FF7EA0
:1061A600007B017A1C7916127D8112A7AB7E1C7FBB
:1061B600227B2012C9D4E5302404F582E4352FF57C
:1061C60083E0C3940A74809480500D7E1C7F227BEA
:1061D600FF7ADD79FF12A7B5E5302404F582E435B0
:1061E6002FF583E0FF7E007B017A1C7916127D81F4
:1061F60012A7AB7E1C7F227B3A12C9D4E530240558
:10620600F582E4352FF583E0C3940A7480948050B8
:106216000D7E1C7F227BFF7ADD79FF12A7B5E53064
:106226002405F582E4352FF583E0FF7E007B017AB5
:106236001C7916127D8112A7AB7E1C7F227B3A1237
:10624600C9D4E5302406F582E4352FF583E0C394FE
:106256000A74809480500D7E1C7F227BFF7ADD7944
:10626600FF12A7B5E5302406F582E4352FF583E065
:10627600FF7E007B017A1C7916127D8112A7ABAFD7
:1062860031126CF97E007F0C7D007B017A1C791639
:10629600122E5AAE32AF33E4FCFD7B017A1C79161E
:1062A60012692312A7AB7E1C7F227B2012C9D4E57C
:1062B6003645354534600D7E1C7F22AB34AA35A9A0
:1062C6003612A7B57B017A1C792212D6A5C3EF94A4
:1062D6003EEE9400501474222FF582741C3EF58312
:1062E6007420F00FBF00010E80E3901C60740DF067
:1062F600A3740AF0AF3AAE39AD38AC377B017A1CDD
:10630600792275420075434012BE9A22E4901BA280
:10631600F0A3F0901BA2E0FEA3E024A3F58274098B
:106326003EF583E06010901BA3E004F070E5901B3F
:10633600A2E004F080DD901BA2E475F0011228496A
:10634600FE74A325F0F58274093EF583742BF09054
:106356001BA2E0FEA3E024A3F58274093EAF82FEF1
:106366007D017C0412D32C901BA4EFF0901BA2E0BD
:10637600FEA3E024A3F58274093EF583E090098725
:10638600F0E4901BA5F0900987E0FF901BA5E0FEC6
:10639600C39F4003026516EE75F010A424A4F97499
:1063A6000935F0FA7B01901BA2E0FEA3E029F9EA89
:1063B6003EFA7D0412C368901BA5E0FB75F013A49A
:1063C600245AF582E4341BF583122A5CEB75F0102F
:1063D600A424A8F9740935F0FA7B01901BA2E0FE0B
:1063E600A3E029F9EA3EFA7D0412C368901BA5E0F2
:1063F600FB75F013A4245EF582E4341BF583122AA0
:106406005CEB75F010A424ACF9740935F0FA7B0145
:10641600901BA2E0FEA3E029F9EA3EFA7D0212C330
:1064260068901BA5E0FD75F013A42462F582E434A0
:106436001BF583EEF0A3EFF0901BA2E0FEA3E0FFB6
:1064460075F010EDA42FF582E5F03EF583E5822484
:10645600AEF582E5833409F583E0FFED75F013A40C
:106466002464F582E4341BF583EFF0ED75F010A497
:1064760024AFF9740935F0FA7B01901BA2E0FEA364
:10648600E029F9EA3EFA7D0212C368901BA5E0FDF9
:106496007A002FFFEA3EFEED75F013A42467F5821D
:1064A600E4341BF583EEF0A3EFF0901BA5E0FF7537
:1064B600F013A4246BF582E4341BF5837401F09089
:1064C6001BA2E0FCA3E0901B6975F013122A99EC5D
:1064D60075F013A42583F583E4F0A3F0EF75F013AC
:1064E600A42462F582E4341BF583E0FEA3E04E703B
:1064F60016901BA5E075F013A42462F582E4341B04
:10650600F583E4F0A304F0901BA5E004F002638C8D
:10651600E4900982F0A3F0900985740FF0A374FF4C
:10652600F002D76AE4901BA2F0A3F0901BA2E475D8
:10653600F001122849FE74A325F0F58274093EF590
:1065460083E070E7901BA2E475F001122849FE74FF
:10655600A325F0F58274093EF583E070E7901BA24F
:1065660075F001122849FE74A325F0F58274093EE0
:10657600F583E075F00AA4FF901BA2E475F0011202
:106586002849FC74A325F0F58274093CF583E02FB5
:1065960024F0900988F0901BA2E475F001122849B6
:1065A600FE74A325F0F58274093EF583E075F00AC2
:1065B600A4FF901BA2E475F001122849FC74A325E0
:1065C600F0F58274093CF583E02F24F0900989F0F8
:1065D600901BA2E475F001122849FE74A325F0F57C
:1065E6008274093EF583E075F00AA4FF901BA2E4CD
:1065F60075F001122849FC74A325F0F58274093C54
:10660600F583E02F24F090098AF0901BA2E475F040
:1066160001122849FE74A325F0F58274093EF5831C
:10662600E075F00AA4FF901BA2E475F00112284958
:10663600FC74A325F0F58274093CF583E02F24F061
:1066460090098BF0901BA2E475F001122849FE74A4
:10665600A325F0F58274093EF583E075F00AA4FFE0
:10666600901BA2E475F001122849FC74A325F0F5ED
:106676008274093CF583E02F24F090098CF0901B7E
:10668600A2E475F001122849FE74A325F0F5827480
:10669600093EF583E075F00AA4FF901BA2E475F0AD
:1066A60001122849FC74A325F0F58274093CF58390
:1066B600E02F24F090098DF0901BA2E475F00112F2
:1066C6002849FE74A325F0F58274093EF583E0752A
:1066D600F00AA4FF901BA2E475F001122849FC748D
:1066E600A325F0F58274093CF583E02F24F0900988
:1066F6008EF090098CE0FFA3E0FDA3E0FB12CF8FA4
:10670600900988E0FFA3E0FD90098BE0FB90098AE1
:10671600E0F52512CC2F12D5D012D7F1EF64017017
:106726000302D76A12D77C22E4901BA2F0A3F09052
:106736001BA2E475F001122849FE74A325F0F58228
:1067460074093EF583E070E7901BA2E475F0011230
:106756002849FE74A325F0F58274093EF583E0709E
:10676600E7901BA275F001122849FE74A325F0F5E7
:106776008274093EF583E075F00AA4FF901BA2E43B
:1067860075F001122849FC74A325F0F58274093CC2
:10679600F583E02F24F0900978F0901BA2E475F0C1
:1067A60001122849FE74A325F0F58274093EF5838B
:1067B600E075F00AA4FF901BA2E475F001122849C7
:1067C600FC74A325F0F58274093CF583E02F24F0D0
:1067D600900979F0901BA2E475F001122849FE7425
:1067E600A325F0F58274093EF583E075F00AA4FF4F
:1067F600901BA2E475F001122849FC74A325F0F55C
:106806008274093CF583E02F24F090097AF0901BFE
:10681600A2E475F001122849FE74A325F0F58274EE
:10682600093EF583E075F00AA4FF901BA2E475F01B
:1068360001122849FC74A325F0F58274093CF583FE
:10684600E02F24F090097BF0901BA2E475F0011272
:106856002849FE74A325F0F58274093EF583E07598
:10686600F00AA4FF901BA2E475F001122849FC74FB
:10687600A325F0F58274093CF583E02F24F09009F6
:106886007CF0901BA2E475F001122849FE74A32542
:10689600F0F58274093EF583E075F00AA4FF901BBB
:1068A600A2E475F001122849FC74A325F0F5827460
:1068B600093CF583E02F24F090097DF0901BA2E4BB
:1068C60075F001122849FE74A325F0F58274093E7D
:1068D600F583E075F00AA4FF901BA2E475F001129F
:1068E6002849FC74A325F0F58274093CF583E02F52
:1068F60024F090097EF090097CE0FFA3E0FDA3E080
:10690600FB12D0CE900978E0FFA3E0FD90097BE072
:10691600FB90097AE0F52512CDDC02D76A8F3E8E10
:106926003D8D3C8C3B8B3F8A408941901BD9740A34
:10693600F0E4A3F0EC3350257401F0253EFFE43576
:106946003DFEE4353CFDE4353BFC1229E1EF240134
:10695600FFE43EFEE43DFDE43CFCA3800BAF3EAE0F
:106966003DAD3CAC3B901BDB122A5CE4901BD7F0A0
:10697600901BD9E0FF901BD7E0C39F5065E47B0ACC
:10698600FAF9F8901BDBE0FCA3E0FDA3E0FEA3E030
:10699600FF12294FEB2430FF901BD9E024FFFDE4C2
:1069A60034FFFC901BD7E0FBC3ED9BFDEC9400ABE2
:1069B6003FAA40A9418D82F583EF122786901BDB03
:1069C600E0FCA3E0FDA3E0FEA3E0FFE47B0AFAF906
:1069D600F812294F901BDB122A5C901BD7E004F0BB
:1069E600808EE4901BD7F0901BD9E014FF901BD744
:1069F600E0FEC39F5019AB3FAA40A9418E82758322
:106A060000122714B43008901BD7E004F080D89009
:106A16001BDAE0607EE4901BD8F0901BD7E0FF9075
:106A26001BD9E0C39FFE901BD8E0FDC39E5028ED06
:106A36002FF582E433F583AB3FAA40A94112271410
:106A4600FF901BD8E0F582758300A3EF122786908E
:106A56001BD8E004F080C3AB3FAA40A941742D12B5
:106A66002774901BD7E0FF901BD9E0C39FFFE494E7
:106A760000CF2401CF3400AB3FAA40A9418F82F555
:106A860083E4122786901BD7E0FF901BD9E0C39FB3
:106A960004FF22901BD7E0D3940074809480404A70
:106AA600E4A3F0901BD7E0FF901BD9E0C39FFE90B4
:106AB6001BD8E0FDC39E5027ED2FF582E433F58306
:106AC600AB3FAA40A941122714FF901BD8E0F582DC
:106AD600758300EF122786901BD8E004F080C4ABC4
:106AE6003FAA40A941901BD88009AB3FAA40A941C3
:106AF600901BD9E0F582758300E4122786901BD798
:106B0600E0FF901BD9E0C39FFF228E2F8F308D317F
:106B160012AF808F358E348D338C327F007E407D70
:106B2600017C00AB35AA34A933A832C3122A05402A
:106B360003026CF87E007F407D007B017A1C79227F
:106B4600122E5A7E007F0C7D007B017A1C7916126C
:106B56002E5A853082852F83A3A3A3E0C3940A749B
:106B660080948050097BFF7ADD79FF12A7B18530CA
:106B760082852F83A3A3A3E0FF7E007B017A1C7985
:106B860016127D8112A7AB12C9CE853082852F835E
:106B9600A3E0C3940A74809480500D7E1C7F227BF0
:106BA600FF7ADD79FF12A7B5853082852F83A3E0B2
:106BB600FF7E007B017A1C7916127D8112A7AB122B
:106BC600C9CE853082852F83E0FF7E007B017A1C4B
:106BD6007916127D8112A7AB7B2012C9D0E530242D
:106BE60004F582E4352FF583E0C3940A748094801B
:106BF600500D7E1C7F227BFF7ADD79FF12A7B5E55B
:106C0600302404F582E4352FF583E0FF7E007B0116
:106C16007A1C7916127D8112A7AB7E1C7F227B3AE5
:106C260012C9D4E5302405F582E4352FF583E0C397
:106C3600940A74809480500D7E1C7F227BFF7ADD3F
:106C460079FF12A7B5E5302405F582E4352FF583E3
:106C5600E0FF7E007B017A1C7916127D8112A7ABBC
:106C66007E1C7F227B3A12C9D4E5302406F582E4E5
:106C7600352FF583E0C3940A74809480500D7E1CF2
:106C86007F227BFF7ADD79FF12A7B5E5302406F572
:106C960082E4352FF583E0FF7E007B017A1C7916AE
:106CA600127D8112A7ABAF31126CF97B017A1C7988
:106CB6002212D6A5C3EF943EEE9400501474222FF0
:106CC600F582741C3EF5837420F00FBF00010E8020
:106CD600E3901C60740DF0A3740AF0AF35AE34ADCA
:106CE60033AC327B017A1C7922754200754340121F
:106CF600BE9A227C1C7D227B407A008C3B8D3C8A8E
:106D06003D8B3EEFB426004003026EC8906D19F825
:106D1600282873026D8B026D94026D9D026DA6028A
:106D26006DAF026DB8026DC1026DCA026DD3026D00
:106D3600DC026DE5026DEE026DF7026EC8026E00B2
:106D4600026E09026E12026E1B026E24026E2D0284
:106D56006E36026E3F026E48026E50026E58026E2A
:106D660060026E68026E70026E78026E80026E8835
:106D7600026E90026E98026EA0026EA8026EB002BB
:106D86006EB8026EC07BFF7AD9796B026ECE7BFF3E
:106D96007AD97987026ECE7BFF7AD979A4026ECE34
:106DA6007BFF7AD979C4026ECE7BFF7AD979E60267
:106DB6006ECE7BFF7ADA7902026ECE7BFF7ADA79C3
:106DC6001E026ECE7BFF7ADA793A026ECE7BFF7AAE
:106DD600DA795F026ECE7BFF7ADA797C026ECE7B41
:106DE600FF7ADA799C026ECE7BFF7ADA79C3026E7D
:106DF600CE7BFF7ADA79DB026ECE7BFF7ADA79E92F
:106E0600026ECE7BFF7ADB7908026ECE7BFF7ADBE1
:106E16007927026ECE7BFF7ADB7949026ECE7BFF45
:106E26007ADB796A026ECE7BFF7ADB798B026ECED5
:106E36007BFF7ADB79A3026ECE7BFF7ADB79CC020D
:106E46006ECE7BFF7ADB79ED807E7BFF7ADC791173
:106E560080767BFF7ADC7934806E7BFF7ADC795D25
:106E660080667BFF7ADC796F805E7BFF7ADC7993C4
:106E760080567BFF7ADC79B4804E7BFF7ADC79D151
:106E860080467BFF7ADC79F7803E7BFF7ADD7915D9
:106E960080367BFF7ADD7931802E7BFF7ADD79576C
:106EA60080267BFF7ADD797A801E7BFF7ADD79A3E7
:106EB60080167BFF7ADD79B8800E7BFF7ADD79CD8F
:106EC60080067BFF7ADD79EDAD3EAC3DAF3CAE3B57
:106ED60012A7B922E4901BA2F0A3F0901BA2E0FE39
:106EE600A3E024A3F58274093EF583E06010901BAD
:106EF600A3E004F070E5901BA2E004F080DD901B97
:106F0600A3E004F07006901BA2E004F0901BA2E040
:106F1600FEA3E024A3F58274093EF583E0643160A4
:106F26000302701D901BA3E004F07006901BA2E004
:106F360004F0E47FC0FEFDFC901B5AE0F8A3E0F9E4
:106F4600A3E0FAA3E0FBC3122A05601AE47FC0FEA1
:106F5600FDFC901B6DE0F8A3E0F9A3E0FAA3E0FBCB
:106F6600C3122A05704A901BA2E0FEA3E024A3F9EF
:106F760074093EFA7B01129C297C007D0A1227FDCA
:106F8600EF25E025E0540C900982F0901BA2E0FE6C
:106F9600A3E024A3F974093EFA7B01129C297C0024
:106FA6007D0A1227FDAF05EF25E025E0540C806031
:106FB600E47FA17E16FDFC901B5AE0F8A3E0F9A33E
:106FC600E0FAA3E0FBC3122A0560030270B0901B2F
:106FD600A2E0FEA3E024A3F974093EFA7B01129C09
:106FE600297C007D0A1227FDEFC45470900982F0B7
:106FF600901BA2E0FEA3E024A3F974093EFA7B01EC
:10700600129C297C007D0A1227FDAF05EFC454703F
:10701600900983F00270B0901BA2E0FEA3E024A3C7
:10702600F58274093EF583E0B43225901BA3E00493
:10703600F07006901BA2E004F0901BA2E0FEA3E015
:1070460024A3F58274093EF583E0900984F0805A02
:10705600901BA2E0FEA3E024A3F58274093EF5830B
:10706600E064337048901BA3E004F07006901BA206
:10707600E004F0901BA2E0FEA3E024A3F5827409CD
:107086003EF583E0FFB4300790098274BC8009EFB7
:10709600B4310A90098274BDF0A3F0800DEFB432CA
:1070A6000990098274BCF0A304F012D76A22E49016
:1070B6001BA2F0A3F0901BA2E475F001122849FE72
:1070C60074A325F0F58274093EF583E070E7901B02
:1070D600A2E0FEA3E024A3F974093EFA7B01129014
:1070E60013901B5A122A5C901BA2E0FEA3E024A375
:1070F600F58274093EF583E06010901BA3E004F06E
:1071060070E5901BA2E004F080DD901BA3E004F084
:107116007006901BA2E004F0901BA2E0FEA3E02400
:10712600A3F974093EFA7B01129013901B5E122A92
:107136005C901BA2E0FEA3E024A3F58274093EF551
:1071460083E06010901BA3E004F070E5901BA2E0C2
:1071560004F080DD901BA3E004F07006901BA2E013
:1071660004F0901BA2E0FEA3E024A3F974093EFA02
:107176007B01129013901B62EEF0A3EFF0901BA21E
:10718600E0FEA3E024A3F58274093EF583E06010D7
:10719600901BA3E004F070E5901BA2E004F080DDF4
:1071A600900985740FF0A374FFF0901B5EE0FCA3BA
:1071B600E0FDA3E0FEA3E0F52F8E2E8D2D8C2C7F17
:1071C600007E367D6E7C0112CF1B7E097FA3E4F51F
:1071D6002EFBFD12563F78A57C1B7D017E007F03AA
:1071E6001226D512D832901BA6A3E0FF12D8009023
:1071F6001BA6E0FF12D800901BA474FFF0901BA6FC
:10720600A3E0FD7FFF12D922901BA4EFF0901BA6EE
:10721600E0FD12D922901BA4EFF0E4901BA2F0A38C
:10722600F0901BA6E0FEA3E0FF901BA2E0FCA3E00B
:10723600FDC39FEC9E503E74A32DF58274093CF568
:1072460083E0FF12D800901BA4E0FF901BA2E0FC95
:10725600A3E024A3F58274093CF583E0FD12D9224C
:10726600901BA4EFF0901BA3E004F070B4901BA257
:10727600E004F080AC901BA4E0FF02D80012D356C5
:10728600901B41EEF0A3EFF0E4F527C3E527940346
:1072960074809480501912202EE52725E024D0F51D
:1072A60082E4341BF583EEF0A3EFF0052780DC9033
:1072B6001BD2E0FEA3E0FF901BD1E02FFF901BD076
:1072C600E03EFE901BD5E02FFF901BD4E03EFE7CF7
:1072D600007D031227A8901B37EEF0A3EFF07F1670
:1072E60012C17DEF24C0FDEE34F9FC1223A9E4FBA4
:1072F600FA79C0783F1221FE1223E2901B4BEEF082
:10730600A3EFF07F1712C17DEF24C0FDEE34F9FC28
:107316001223A9E4FBFA79C0783F1221FE1223E278
:10732600901B4DEEF0A3EFF07F1312C17DEE339567
:10733600E0FDFCE47B0BFAF9F81228C4901B39EE49
:10734600F0A3EFF07F1212C17DEE3395E0FDFCE471
:107356007B0BFAF9F81228C4901B3BEEF0A3EFF072
:107366007F1512C17DEE3395E0FDFCE47B0BFAF947
:10737600F81228C4901B3DEEF0A3EFF07F1412C163
:107386007DEE3395E0FDFCE47B0BFAF9F81228C498
:10739600901B3FEEF0A3EFF07F3012C17D901BCE25
:1073A600EEF0A3EFF0FDAC06EC1223A97B337AB323
:1073B600796078C412210D7BB87A1E79557840120F
:1073C60023071223E2901BCEEEF0A3EFF0901BCE24
:1073D600E0FCA3E0FD901B45ECF0A3EDF0EC1223DE
:1073E600A97B3D7A0A793778401221FEE4FBFA79C7
:1073F60042784412210D7B007AF0797F784512217C
:10740600FEE4FBFA791678451223071223E2901B55
:10741600CEEEF0A3EFF0901B43EEF0A3EFF0128F49
:1074260034EF600F128F34EF60097D1FAF16AE1573
:10743600129ACA228B278A2889297B017A1C790C01
:10744600754A00754B0A7F007E487D017C0012BD9F
:10745600BF901C0CE0FFF4700AA3E0F47005A3E0F3
:10746600F46052901BD2EFF0901C0DE0901BD3F00D
:10747600901C0EE0901BD4F0901C0FE0901BD1F0F6
:10748600901C10E0901BCFF0901C11E0901BCEF0EA
:10749600901C14E0FE901C13E0FDED8E2DF52E7E63
:1074A6001B7FCE7534FF7535DE753601AB2EAA2DE2
:1074B6007D231260DDE4F52CC3E52C9440748094A2
:1074C600804003027596E52C75F00AA4FFE42FFFB1
:1074D600E5F03440FEE43401FDE433FC7B017A1C24
:1074E600790C754A00754B0A12BDBF901C0CE0FF63
:1074F600F4700DA3E0F47008A3E0F470030275962F
:10750600901BD2EFF0901C0DE0901BD3F0901C0E58
:10751600E0901BD4F0901C0FE0901BD1F0901C1053
:10752600E0901BCFF0901C11E0901BCEF0901C1445
:10753600E0FE901C13E0FDEEF52DEDF52EE52E4553
:107546002D603C901C12E06420701912D94CAA06DA
:10755600A9077534FF8A3589367E1B7FCE901C12AB
:10756600E0FD80127E1B7FCE901C12E0FD7534FF7D
:107576007535DE753604AB2EAA2D1260DD800C7EC5
:107586001B7FCE901C12E0FD126B10052C0274BE00
:10759600AB27AA28A929754A10754B007F007E30B3
:1075A6007D017C0012BDBFE4F52AF52BAE2AAF2B78
:1075B600E4FCFDFB7A10F9F8D3122A054027AB2725
:1075C600AA28A929852B82852A83122714F4700BF1
:1075D600852B82852A837420122786052BE52B703E
:1075E600CB052A80C722901B47E0FCA3E0FDA3E061
:1075F600FEA3E02401FFE43EFEE43DFDE43CFC90F6
:107606001B47122A5C901BA4122A680000001090E7
:107616000987E070069009B374FFF0E4901BA2F0AE
:10762600A3F0900987E0FF901BA2E0FCA3E0FDC356
:107636009FEC94004003027707901B6775F013EDEB
:10764600122A99EC75F013A42583F583E0FEA3E0D6
:1076560024B3F58274093EAF82F5228F23901B5E18
:1076660075F013ED122A99EC75F013A42583F583B2
:10767600E0FCA3E0FDA3E0FEA3E0F52F8E2E8D2D0A
:107686008C2C7F007E367D6E7C0112CF1B901BA258
:10769600E0FCA3E0FD901B6475F013122A99EC75CB
:1076A600F013A42583F583E0D3940174809480506D
:1076B60050AF23AE2212D09B78A87C1B7D017E00A2
:1076C6007F031226D5901BA4E0F8A3E0F9A3E0FA05
:1076D600A3E0FB901BA9E0FEA3E0FFE4FCFDEB2F7B
:1076E600FFEA3EFEED39FDEC38FC901BA4122A5C45
:1076F600901BA3E004F07006901BA2E004F0027653
:10770600287E097FA3128021E47F3FFEFDFC901BAB
:10771600A4E0F8A3E0F9A3E0FAA3E0FBD3122A055C
:107726007E0040047F7F80027F3F901BAB12D82DE6
:10773600E4901BA2F0A3F0901BABE0FEA3E0FF9049
:107746001BA2E0FCA3E0FDC39FEC9E501F74A32D7B
:10775600F58274093CF583E0FF12D800901BA3E084
:1077660004F070D3901BA2E004F080CB7E097FA3C7
:10777600901BABE0FCA3E0FD12D32C12D800901BAB
:10778600ABE0FEA3E0FF7D007B017A0979A3022E20
:107796005A7F037E0012D132C3E51C9408500302BF
:1077A60078E2E51D7004E51C6408702BAF11AE107D
:1077B600AD0FAC0EF52EF52F1287CBEF6016AA1083
:1077C600AB117527FF7528E87529E97D16AF16AE4A
:1077D600151279330278BA900981E0C39402748055
:1077E60094805069AF11AE10AD0FAC0EE4F52EF5D6
:1077F6002F1287CBEF6016AA10AB117527FF7528DD
:10780600E87529E97D16AF16AE15127933E5112410
:1078160001F511E43510F510E4350FF50FE4350EDA
:10782600F50EAF11AE10AD0FFC75260875270012C8
:107836008AB1EF6016AA10AB117527FF7528E87597
:1078460029E97D16AF16AE151279338067AF11AEF2
:1078560010AD0FAC0EE4F52EF52F1287CBEF6016A8
:10786600AA10AB117527FF7528E87529E97D16AFB3
:1078760016AE15127933E5112401F511E43510F52C
:1078860010E4350FF50FE4350EF50EAF11AE10AD61
:107896000FFC752E08752F001287CBEF6016AA1005
:1078A600AB117527FF7528E87529E97D16AF16AE69
:1078B60015127933E5112401F511E43510F510E4BC
:1078C600350FF50FE4350EF50EE4F51CF51D7E11AA
:1078D6007F94FD7B017A0979A3122E5A12BF06EF17
:1078E60064037008901CE0E004F08005E4901CE05E
:1078F600F0901CE0E0D3940A74809480400C7D1EC6
:10790600AF16AE15129ACA123EC87FFB7E457D1E83
:107916007C00AB11AA10A90FA80EC3122A05400CB1
:107926007D0BAF16AE15129ACA123EC8228E228F52
:10793600238D248A258B26E52464086003027A04B5
:10794600C3E5269498E525943A5003027A047524F3
:107956002312B0888F2D8E2C8D2B8C2A7F007E5083
:107966007D017C00AB2DAA2CA92BA82AC3122A05BF
:107976004003027AB17E007F0A7D007B017A1C7982
:107986000C122E5AE5232404F582E43522F583E011
:10799600901C0CF0E5232405F582E43522F583E0FE
:1079A600901C0DF0E5232406F582E43522F583E0EC
:1079B600901C0EF0852382852283A3A3A3E0901C4E
:1079C6000FF0852382852283A3E0901C10F0852387
:1079D60082852283E0901C11F0A3E524F0E526A31E
:1079E600F0E525A3F0E4A3F0AF2DAE2CAD2BAC2A29
:1079F6007B017A1C790CF54275430A12BE9A12B0C5
:107A0600048F2D8E2C8D2B8C2A7F007E487D017C49
:107A160000AB2DAA2CA92BA82AC3122A05400302C3
:107A26007AB17E007F0A7D007B017A1C790C122ECA
:107A36005AE5232404F582E43522F583E0901C0CF4
:107A4600F0E5232405F582E43522F583E0901C0D4C
:107A5600F0E5232406F582E43522F583E0901C0E3A
:107A6600F0852382852283A3A3A3E0901C0FF085D3
:107A76002382852283A3E0901C10F0852382852231
:107A860083E0901C11F0A3E524F0E526A3F0E5259C
:107A9600A3F0E4A3F0AF2DAE2CAD2BAC2A7B017A7C
:107AA6001C790CF54275430A12BE9A22E4901BA279
:107AB600F0A3F0901BA2E475F001122849FE74A30E
:107AC60025F0F58274093EF583E070E7901BA2E08D
:107AD600FEA3E024A3F974093EA801FC7D017BFF07
:107AE6007ADE7906122C93EF3395E04F70061292E8
:107AF6009D027BD5901BA2E0FEA3E024A3F97409A6
:107B06003EA801FC7D017BFF7ADE790D122C93EFF6
:107B16003395E04F700612C78D027BD5901BA2E00D
:107B2600FEA3E024A3F974093EA801FC7D017BFFB6
:107B36007ADE7913122C93EF3395E04F700612C755
:107B460039027BD5901BA2E0FEA3E024A3F97409B9
:107B56003EA801FC7D017BFF7ADE7919122C93EF9A
:107B66003395E04F7071901BA2E475F0011228491D
:107B7600FE74A325F0F58274093EF583E070E79064
:107B86001BA2E0FEA3E024A3F974093EFA7B0112CE
:107B96009C29901BA4EEF0A3EFF0901BA2E475F0D5
:107BA60001122849FE74A325F0F58274093EF58377
:107BB600E070E7901BA2E0FEA3E024A3F58274091F
:107BC6003EAF82FE901BA4E0FCA3E0FD12AD6090E8
:107BD6001BA6EEF0A3EFF0901BA6E07002A3E060F8
:107BE6003F12D832E4901BA2F0A3F0901BA6E0FE51
:107BF600A3E0FF901BA2E0FCA3E0FDC39FEC9E5018
:107C06002274002DF58274003CF583E0FF12D80043
:107C1600901BA3E004F070D3901BA2E004F080CB8D
:107C260012D77C228F408E3F8D3E8C3D85A74575B1
:107C3600A710AB44AA43A942A841AF40AE3FAD3E10
:107C4600AC3D12294FE47B02FAF9F812294FE47B86
:107C5600FFFAF9F8D3122A05402AAB44AA43A942EF
:107C6600A841AF40AE3FAD3EAC3D12294FE47B028A
:107C7600FAF9F812294F1229E18F8D538EF4438EAB
:107C860008027D6EAB44AA43A942A841AF40AE3F6D
:107C9600AD3EAC3D12294FE47B02FAF9F812294FAA
:107CA600E47B04FAF9F812294FE47BFFFAF9F8D3DA
:107CB600122A054033AB44AA43A942A841AF40AEBD
:107CC6003FAD3EAC3D12294FE47B02FAF9F812298A
:107CD6004FE47B04FAF9F812294F1229E18F8D53EC
:107CE6008EF4438E01027D6EAB44AA43A942A8419D
:107CF600AF40AE3FAD3EAC3D12294FE47B02FAF9F0
:107D0600F812294FE47B0CFAF9F812294FE47BFFAD
:107D1600FAF9F8D3122A05AB44AA43A942A841AFFF
:107D260040AE3FAD3EAC3D401F12294FE47B02FA08
:107D3600F9F812294FE47B0CFAF9F812294F1229A7
:107D4600E18F8D538EF4802012294FE47B02FAF9DD
:107D5600F812294FE47B30FAF9F812294F1229E17B
:107D66008F8D538EF4438E02858D8B53890F4389F5
:107D760020D28ED29DD29C8545A7228E3B8F3C8BEE
:107D86003D8A3E893F7C007D0A1227FD900004ED66
:107D9600122786AE3BAF3C7C007D0A1227FD8E3B48
:107DA6008F3C7C007D0A1227FDAB3DAA3EA93F9081
:107DB6000003ED122786AE3BAF3C7C007D0A1227FE
:107DC600FD8E3B8F3C7C007D0A1227FDAB3DAA3E13
:107DD600A93F900002ED122786AE3BAF3C7C007DAA
:107DE6000A1227FD8E3B8F3C7C007D0A1227FDABD5
:107DF6003DAA3EA93F900001ED122786AE3BAF3C5F
:107E06007C007D0A1227FD8E3B8F3C7C007D0A128A
:107E160027FDAB3DAA3EA93FED122774E4901BD780
:107E2600F0901BD7E0FFC3940574809480501DAB7F
:107E36003DAA3EA93F8F82758300122714FF339512
:107E4600E04F7008901BD7E004F080D5901BD7E078
:107E56006405701BAB3DAA3EA93F7430122774AB74
:107E66003DAA3EA93F900001E41227867F0122E445
:107E7600901BD8F0901BD7E0FFC374059FFEA3E0CC
:107E8600FDC39E5029ED2FF582E433F583AB3DAA61
:107E96003EA93F1227142430FF901BD8E0F58275C7
:107EA6008300EF122786901BD8E004F080C6901B53
:107EB600D7E0FFFDC374059DFDE49400AB3DAA3EEB
:107EC600A93F8D82F583E4122786C374059FFF229E
:107ED60012D8D112D49412D95C12D37F12D7E212DF
:107EE600202612D2D67F0112200612D63512C97E5E
:107EF600C297E490096AF090096CF09009687403DF
:107F0600F09009677409F01283A290096F122A5C37
:107F160090096AE0C3940674809480501475250114
:107F26007526097527647B017A1B79371295B88007
:107F3600DF12728312D7F190096BEFF064017012B1
:107F4600900966E06402600512206E800812BF7216
:107F5600800312BFDC900968E014700302800C14E1
:107F6600601A24FD607624FE7003028015147003E7
:107F760002801B240570DE12B67A80D912AA9812E6
:107F86008C83EF4E60277F0112200612D968752771
:107F9600FF7528E9752921901B53E0FAA3E0FB7DC4
:107FA60008AF16AE15127933E4FF122006901B9C1B
:107FB600E0640170A0F07F0112200612D9687527CF
:107FC600FF7528E97529217B2A7A2B7D08AF16AE25
:107FD60015127933E4FF122006027F5B12943212E7
:107FE6008C83EF4E7003027F5B7527FF7528E9755A
:107FF6002921901B53E0FAA3E0FB7D08AF16AE15CE
:10800600127933027F5B12B5FE128C83027F5B12FC
:10801600BC71027F5B12D3A8027F5B8E278F2890EC
:108026001B47A3A3A3E0852882852783F0901B47DF
:10803600E0FCA3E0FDA3E0FEA3E0FF7808122A1609
:10804600852882852783A3EFF0901B4BE0FEA3E0F3
:10805600852882852783A3A3F0EEFF8528828527BE
:1080660083A3A3A3EFF0901B4DE0FEA3E0FDE5285C
:108076002404F582E43527F583EDF0EEFFE52824A8
:1080860005F582E43527F583EFF0901B51E0FEA35A
:10809600E0FF12B28F901B4FEEF0A3EFF0E4A3F0D7
:1080A600A3F0901B4FE0FEA3E0FDE5282406F58231
:1080B600E43527F583EDF0EEFFE5282407F582E4A5
:1080C6003527F583EFF0901B37E0FEA3E0FDE528AA
:1080D6002408F582E43527F583EDF0EEFFE5282444
:1080E60009F582E43527F583EFF0901B39E0FEA30E
:1080F600E0FDE528240AF582E43527F583EDF0EE68
:10810600FFE528240BF582E43527F583EFF0901B75
:1081160043E0FEA3E0FDE528240CF582E43527F5CF
:1081260083EDF0EEFFE528240DF582E43527F5838F
:10813600EFF0901B3BE0FEA3E0FDE528240EF58260
:10814600E43527F583EDF0EEFFE528240FF582E40C
:108156003527F583EFF022901B47E0FCA3E0FDA353
:10816600E0FEA3E0FFC007900981E0FBE4FAF9F81E
:10817600D00712294F901B47122A5C74A3251DF5C0
:10818600827409351CAF82FE128021901B47E0F8ED
:10819600A3E0F9A3E0FAA3E0FB900981E0FFE4FC89
:1081A600FDFE1228C4901B47122A5C900986E02423
:1081B600EEFF900985E034FFFE74A3251DF5827459
:1081C60009351CF583E5822FF582E5833EAF82FEF5
:1081D60012C117900986E024F6FF900985E034FF66
:1081E600FE74A3251DF5827409351CF583E5822FDF
:1081F600F582E5833EAF82FE12C2A8900985E0FEB5
:10820600A3E0FF7491251DF5827409351CF583E5FD
:10821600822FF582E5833EAF82FE7D107C0012D36D
:108226002C900985E0FCA3E0FD251DFBE51C3CFA2E
:1082360074A12BF58274093AF583EFF074A3251D1A
:10824600F5827409351CAF82FEED24FFFDEC34FF88
:10825600FC12D32C900985E0FCA3E0FD251DFBE56F
:108266001C3CFA74A22BF58274093AF583EFF0ED03
:10827600251DF51DEC351CF51C221297F0E4901B0C
:10828600A2F0A3F0901BA2E475F001122849FE7437
:10829600A325F0F58274093EF583E070E7901BA4F0
:1082A600F0901BA4E0C3940874809480505F901BE8
:1082B600A2E475F001122849FE74A325F0F5827434
:1082C600093EF583E0FF12D599901BA5EFF0E0C4B7
:1082D60054F0F0901BA2E475F001122849FE74A335
:1082E60025F0F58274093EF583E0FF12D599901BBF
:1082F600A5E02FF0E0FF901BA4E02493F582E43480
:108306001BF583EFF0901BA4E004F0809412BA38BA
:10831600EF600B12D8327BFF7ADF79DF807512C4EB
:108326007CEF600B12D8327BFF7ADF79F280641221
:10833600B2107E047F007D007B017A0D79A3122E98
:108346005A78A37C097D017B017A0079007E047F3F
:10835600001226D57E097FA37DFE7C0312D32C90C6
:108366000DA1EFF07B017A0979A37DFF7C0312CF83
:10837600FE900DA2EFF0E4F526F5277F907E08FD2E
:10838600FC128B9AEF700302D76A12D8327BFF7AFF
:10839600E079001243AAE4FF12D80022E4F525F59D
:1083A60024F523F5227F3812D885901BA2EFF07FA3
:1083B6003912D885901BA3EFF07F3A12D885901B0F
:1083C600A4EFF07F3B12D885901BA5EFF07F3C12FF
:1083D600D885901BA6EFF07F3D12D885901BA7EF9E
:1083E600F07F3E12D885901BA8EFF07F3F12D8850C
:1083F600901BA9EFF07E1B7FA27D037C0012D32C7D
:10840600901BA5E0B50731901BA3E0FFE4FCFDFE41
:108416007808122A29A804A905AA06AB07901BA268
:10842600E0FFEB4FFFEAFEE9FDE8FCC004C005C033
:1084360006C007901BA480417E1B7FA67D037C009F
:1084460012D32C901BA9E0B50754901BA7E0FFE4BC
:10845600FCFDFE7808122A29A804A905AA06AB077E
:10846600901BA6E0FFEB4FFFEAFEE9FDE8FCC00427
:10847600C005C006C007901BA8E0FFE4FCFDFE781F
:1084860010122A29D003D002D001D000EF4BF525D7
:10849600EE4AF524ED49F523EC48F5228009E4F58A
:1084A60025F524F523F522AF25AE24AD23AC2222F3
:1084B60012C3C6EF60097D09AF16AE15129ACA7EC1
:1084C600117F947D007B017A0979A3122E5A78A335
:1084D6007C097D017B017A0079007E097F60122686
:1084E600D5E4F52EF52F7F807E08FDFC1287CB7E26
:1084F600117F947D007B017A0979A3122E5A78A305
:108506007C097D017B017A0079007E097F60122655
:10851600D5E4F52EF52F7F907E08FDFC1287CB1251
:10852600D95F8F298E288D278C26E47F517E08FD02
:10853600FCAB29AA28A927A826C3122A0550037F1F
:108546000422E5292470FFE52834F7FEE52734FFE9
:10855600FDE52634FFFCE4FB7A08F9F81228C48FFF
:10856600258E248D238C227E117F947D007B017ABB
:108576000979A3122E5A900A3FE525F0FFAE24ADE5
:1085860023AC227808122A16A3EFF0AF25AE24AD4D
:1085960023AC227810122A16A3EFF0AF25AE24AD35
:1085A60023AC227818122A16A3EFF0E4F52EF52F45
:1085B600FF7E08FDFC1287CB7F00228F4B8E4A8DF3
:1085C600498C4885A74DA2AF920085F54E85EF519F
:1085D60085FF52C2AFE4F5A7FF7E80FDFCAB4BAA38
:1085E6004AA949A848C3122A05500B854A4F854B0C
:1085F6005053F5CF8076E4FFFE7D01FCAB4BAA4AD3
:10860600A949A848C3122A055020E54BF54BE54A6F
:108616004480F54AE549F549E548F548854A4F85D8
:108626004B5053F5CF43F51080427F007E807D018D
:108636007C00AB4BAA4AA949A848C3122A05502078
:10864600E54BF54BE54A4480F54AE549F549E548E9
:10865600F548854A4F854B5053F5CF43F520800C9E
:10866600854A4F854B5053F5CF43F530E4F5EF750A
:10867600FFA0FFEFC394FF7480948050030F80F334
:10868600E5FF30E62975EF0275B7A575B7F1438F9B
:108696000175FFA075EF02855082854F83E54CF08A
:1086A600E4F5EF8552FF8551EF538FFE8006855224
:1086B600FF8551EF854EF5854DA7A20092AF7F014C
:1086C600228F298E288D278C2685A72AA2AF920075
:1086D60085F52B85EF2E85FF2FC2AFE4F5A7FF7E2C
:1086E60080FDFCAB29AA28A927A826C3122A055073
:1086F6000B85282C85292D53F5CF8076E4FFFE7D4A
:1087060001FCAB29AA28A927A826C3122A055020AE
:10871600E529F529E5284480F528E527F527E52606
:10872600F52685282C85292D53F5CF43F510804253
:108736007F007E807D017C00AB29AA28A927A82678
:10874600C3122A055020E529F529E5284480F52895
:10875600E527F527E526F52685282C85292D53F5C9
:10876600CF43F520800C85282C85292D53F5CF4342
:10877600F530E4F5EF75FFA0FFEFC394FF74809426
:108786008050030F80F3E5FF30E62775EF0275B7DB
:10879600A575B7F1438F0375FFA075EF02852D828E
:1087A600852C83E4F0F5EF852FFF852EEF538FFCA4
:1087B6008006852FFF852EEF852BF5852AA7A2003B
:1087C60092AF7F01227536FF7537E475389C8F3C72
:1087D6008E3B8D3A8C397B017A1C79B51243A48F76
:1087E60032753A607539E37538167537007F007E45
:1087F600367D6E7C0112CF55E4F530F53174852552
:1088060031F58274E63530F583E493FF12D78E0591
:1088160031E53170020530C3940AE530940040DD3D
:10882600E4F530F531C3E5319532E5309400501B5F
:1088360074B52531F582741C3530F583E0FF12D707
:108846008E0531E53170DE053080DAE4FF12D78E11
:10885600852E30852F31E4252FFFE52E3408FEC303
:10886600E5319FE5309E501B74A32531F5827409CE
:108876003530F583E0FF12D78E0531E53170D70527
:108886003080D37F647E007D007C0012B950EF708B
:108896002EC3900961E09402900960E09400401CA8
:1088A60078007C007D017BFF7AE479A37E007F025D
:1088B600122E36EF3395E04F7002FF227F01227FA2
:1088C6000122E4901BA2F0A3F0901BA2E475F00134
:1088D600122849FE74A325F0F58274093EF583E05B
:1088E60070E7901BA2E0FEA3E024A3F974093EFA08
:1088F6007B01129013901BA4122A5C901BA2E475B4
:10890600F001122849FE74A325F0F58274093EF59C
:1089160083E070E7901BA2E0FEA3E024A3F97409AC
:108926003EFA7B01129C29901BA8EEF0A3EFF09073
:108936001BA2E475F001122849FE74A325F0F58206
:1089460074093EF583E070E77E097F60FD7B017A5E
:10895600007900122E5AE4901BAAF0A3F0901BA4F3
:10896600E0FCA3E0FDA3E0FEA3E0FF901BA2E0F580
:1089760026A3E0F527901BA8E0F528A3E0F5291229
:1089860090F1EF703812D832901BAAE0FEA3E024D3
:1089960000F58274003EF583E0601D901BAAE47525
:1089A600F001122849FE740025F0F58274003EF5A8
:1089B60083E0FF12D80080D0E4FF12D800228B2378
:1089C6008A248925AB26AA27A9281226FBFFAB23D2
:1089D600AA24A9251226FBFE6F600AEEC39F7F011B
:1089E60050027FFF22AB26AA27A928900001122752
:1089F60014FFAB23AA24A925900001122714FE6FA9
:108A0600600AEEC39F7F0150027FFF22AB26AA2792
:108A1600A928900003122714FFAB23AA24A92590A6
:108A26000003122714FE6F600AEEC39F7F015002F7
:108A36007FFF22AB26AA27A928900004122714FF3D
:108A4600AB23AA24A925900004122714FE6F600AFE
:108A5600EEC39F7F0150027FFF22AB26AA27A928DB
:108A6600900005122714FFAB23AA24A92590000520
:108A7600122714FE6F600AEEC39F7F0150027FFF2C
:108A860022AB26AA27A928900006122714FFAB239B
:108A9600AA24A925900006122714FE6F600AEEC3C9
:108AA6009F7F0150027FFF227F00227536FF7537B8
:108AB600E475389C8F3C8E3B8D3A8C397B017A1C51
:108AC60079B51243A48F2A753A607539E37538165D
:108AD6007537007F007E367D6E7C0112CF55E4F53A
:108AE60028F529748F2529F58274E63528F583E45F
:108AF60093FF12D78E0529E52970020528C3940B2A
:108B0600E528940040DDE4F528F529C3E529952AF2
:108B1600E5289400501B74B52529F582741C352868
:108B2600F583E0FF12D78E0529E52970DE0528803A
:108B3600DAE4FF12D78E852628852729E42527FF24
:108B4600E5263408FEC3E5299FE5289E501B74A33D
:108B56002529F58274093528F583E0FF12D78E059D
:108B660029E52970D7052880D37F967E007D007C75
:108B76000012B950EF701A78007C007D017BFF7AF5
:108B8600E479A3122C93EF3395E04F7F017004FF35
:108B9600227F01227536FF7537E475389C8F3C8E2F
:108BA6003B8D3A8C397B017A1C79B51243A48F2A06
:108BB600753A607539E37538167537007F007E366D
:108BC6007D6E7C0112CF55E4F528F529748525299B
:108BD600F58274E63528F583E493FF12D78E0529CE
:108BE600E52970020528C3940AE528940040DDE4CF
:108BF600F528F529C3E529952AE5289400501B7424
:108C0600B52529F582741C3528F583E0FF12D78E29
:108C16000529E52970DE052880DAE4FF12D78E855E
:108C26002628852729E42527FFE5263408FEC3E5FF
:108C3600299FE5289E501B74A32529F582740935C2
:108C460028F583E0FF12D78E0529E52970D7052878
:108C560080D37FB87E0B7D007C0012B950EF701A6E
:108C660078007C007D017BFF7AE479A3122C93EFD8
:108C76003395E04F7F017004FF227F01227F181297
:108C8600CFC7901BA4EEF0A3EFF07F1912CFC790C9
:108C96001BA6EEF0A3EFF0901BA4E0FCA3E02400DB
:108CA600FDEC34FAFC901BA8F0A3EDF0E42FFFEEE8
:108CB60034FAA3F0A3EFF0C3EC64809480501590CF
:108CC6001BA8E0FEA3E0FFC3E49FFFE49E901BA861
:108CD600F0A3EFF0901BAAE0FEA3E0FFC3EE6480D2
:108CE6009480500DC3E49FFFE49E901BAAF0A3EF6F
:108CF600F0901BAAE0FEA3E0FF901BA8E0FCA3E017
:108D0600FDD39FEE6480F8EC6480984006AE04AF15
:108D1600058000901BA2EEF0A3EFF0C3901B52E07B
:108D26009F901B51E09E500F901BA2E0FFA3E09086
:108D36001B51CFF0A3EFF0901BA2E0FEA3E0FFC310
:108D460094BFEE94014019D3EF94D7EE94035010DC
:108D560012CE1E901B53EEF0A3EFF07E007F012291
:108D6600E4FEFF22E4901BA2F0A3F0901BA2E475A0
:108D7600F001122849FE74A325F0F58274093EF528
:108D860083E070E7901BA2E0FEA3E024A3F9740938
:108D96003EFA7B01129013901BA4122A5C901BA230
:108DA600E475F001122849FE74A325F0F5827409D2
:108DB6003EF583E070E7901BA2E0FEA3E024A3F952
:108DC60074093EFA7B01129C29901BA8EEF0A3EFD2
:108DD600F0901BA2E475F001122849FE74A325F059
:108DE600F58274093EF583E070E77E097F60FD7BBE
:108DF600017A007900122E5AE4901BAAF0A3F09093
:108E06001BA4E0FCA3E0FDA3E0FEA3E0FF901BA2F1
:108E1600E0F52EA3E0F52F1287CBEF700B12D832B8
:108E26007BFF7ADE7988800912D8327BFF7ADE7979
:108E3600A8901BA4E0FCA3E0FDA3E0FEA3E0F539A7
:108E46008E388D378C361243AA22901CE2E004F04D
:108E56007006901CE1E004F0D3901CE2E094E090F0
:108E66001CE1E094015003028F3390096FE0FCA3EC
:108E7600E0FDA3E0FEA3E02401FFE43EFEE43DFDA9
:108E8600E43CFC90096F122A5CE4901CE1F0A3F02C
:108E960090096FE0FCA3E0FDA3E0FEA3E0FF901BBA
:108EA600A2EFF090096FA3A3A3E07808122A169008
:108EB6001BA3EFF090096FE0FCA3E0FDA3E0FEA387
:108EC600E0FF7810122A16E4901BA4EFF07E1B7FB9
:108ED600A27D037C0012D32C901BA5EFF0901BA261
:108EE600E0FD7F3812D892901BA3E0FD7F3912D89F
:108EF60092901BA4E0FD7F3A12D892901BA5E0FD4C
:108F06007F3B12D892901BA2E0FD7F3C12D8929034
:108F16001BA3E0FD7F3D12D892901BA4E0FD7F3E8F
:108F260012D892901BA5E0FD7F3F12D892227E1B9D
:108F36007FD67C1B7DF112ADEB7E1B7FD67C1B7D25
:108F4600F112AE767E1B7FDF7C1B7DFA12ADEB7EC7
:108F56001B7FDF7C1B7DFA12AE767E1B7FE87C1CB6
:108F66007D0312ADEB7E1B7FE87C1C7D0312AE7683
:108F76007E1B7FF17C1B7DFA12A8DFEF700C7FF160
:108F86007C1C7D0312A8DFEF602178917C097D01AE
:108F96007B017A1B79F17E007F091226D578787CD1
:108FA600097D017B017A1B79D6802D7E1B7FFA7C99
:108FB6001C7D0312A8DFEF602878917C097D017B78
:108FC600017A1B79FA7E007F091226D578787C090A
:108FD6007D017B017A1B79DF7E007F091226D58011
:108FE6002978917C097D017B017A1C79037E007FBB
:108FF600091226D578787C097D017B017A1B79E8F0
:109006007E007F091226D57F01227F00228B238ACC
:10901600248925AB23AA24A9251226FBFF12D7579C
:10902600500D74012525F525E43524F52480E4D278
:1090360000AB23AA24A9251226FBFF642B6004EFAC
:10904600B42D1BAB230525E525AA2470020524149F
:10905600F91226FB642D6003D38001C39200E4F568
:1090660029F528F527F526AB23AA24A9251226FBE0
:10907600FF12D85A505CE47F0AFEFDFCAB29AA28F1
:10908600A927A8261228C4C8ECC8EDC0E0EEC0E0A7
:10909600EFC0E0AB23AA24A9251226FBFF3395E0F7
:1090A600FEEF24D0FFEE34FFFEE4FCFDD0E0FBD063
:1090B600E0FAD0E0F9EB2FF529EA3EF528ED39F58F
:1090C60027EC38F52674012525F525E43524F52405
:1090D600809530000AAF29AE28AD27AC26800BAFAD
:1090E60029AE28AD27AC261229E1228F258E248DA4
:1090F600238C227536FF7537E475389C8F3C8E3B82
:109106008D3A8C397B017A1C79B51243A48F2C7564
:109116003A607539E37538167537007F007E367DFF
:109126006E7C0112CF55E4F52AF52B74E0252BF55C
:109136008274E5352AF583E493FF12D78E052BE575
:109146002B7002052AC3940DE52A940040DDAF2555
:1091560012D78EAF25AE24AD23AC227808122A167C
:1091660012D78EAF25AE24AD23AC227810122A1664
:1091760012D78EAF25AE24AD23AC227818122A164C
:1091860012D78E85262A85272BE5292527FFE52850
:109196003526FEC3E52B9FE52A9E501B74A3252B7F
:1091A600F5827409352AF583E0FF12D78E052BE583
:1091B6002B7002052A80D27F647E007D007C00022F
:1091C600B95012AA0690096412D82D7F6412D800ED
:1091D600E4FF12D8007F6412D800E4FF12D8007FA3
:1091E6006412D800E4FF12D800E4901BA2F0A3F0AA
:1091F600E4FF12D800901BA3E004F07006901BA2B7
:10920600E004F0C3901BA3E0940B901BA2E0940033
:1092160040DEE4FF12D8007F1212D8007F7A12D8FF
:1092260000E4FF12D800E4901BA2F0A3F0901BA26A
:10923600E0FEA3E0FFC39407EE9400502074802F55
:10924600F58274E13EF583E493FF12D800901BA3E8
:10925600E004F070D8901BA2E004F080D0E4901BEC
:10926600A2F0A3F0E4FF12D800901BA3E004F07074
:1092760006901BA2E004F0C3901BA3E09410901B81
:10928600A2E0940040DE900964A3E0FF12D80090AB
:109296000964E0FF02D80078A87C1B7D017BFF7A79
:1092A600E579877E007F081226D5E4901BB0F09002
:1092B6001BB0E0C394027480948040030293667EE0
:1092C600097F607D007B017A007900122E5A901B7F
:1092D600B0E025E025E024A8F582E4341BF583E020
:1092E600FCA3E0FDA3E0FEA3E0F53A8E398D388CB1
:1092F600377F007E367D6E7C0112CF55E4F522F570
:1093060023747F2523F58274E53522F583E493FFE4
:1093160012D78E0523E52370020522C39408E522A1
:10932600940040DDE4FF12D78E7F327E007D007C04
:109336000012B950EF7020F522F5230523E523AE80
:109346002270020522142400F58274003EF583E0A3
:1093560070E9AE22AF2322901BB0E004F00292B572
:10936600E4FEFF22753A607539E3753816753700E5
:109376007F007E367D6E7C0112CF55E4F52AF52BF3
:1093860074F6252BF58274E4352AF583E493FF12EF
:10939600D78E052BE52B7002052AC3940FE52A9478
:1093A6000040DD7F987E3A7D007C0012B950EF7058
:1093B6006C900002E0FFE4FCFDFE7810122A29E41E
:1093C600FFFEE4FCA804A905AA06AB07900001E08D
:1093D600FE900000E02400FFEC3EFEE4FDEB2FFFD4
:1093E600EA3EFEED39FDEC38FCC004C005C006C0FF
:1093F60007900003E0FFE4FCFDFE7818122A29E43A
:10940600FFFEFDD003D002D001D000EF2BF52FEEEA
:109416003AF52EED39F52DE83CF52C8006E4FFFEF5
:10942600FDFC22AF2FAE2EAD2DAC2C22E51770031E
:109436000294F4E4F517128E50901CDFE004F0E07D
:10944600D3941E748094804002E4F0901CDFE0C345
:109456001390E8EE9324FF9297901B47E0FCA3E05D
:10946600FDA3E0FEA3E02401FFE43EFEE43DFDE4AF
:109476003CFC901B47122A5C900981E0FBE4FAF958
:10948600F8901B47E0FCA3E0FDA3E0FEA3E0FF127B
:10949600294FAC00AD01AE02AF03E4FBFAF9F8C305
:1094A600122A057014127283125343901B55EFF063
:1094B60012815D127797125BDD7525017526097598
:1094C60027647B017A1B79371295B890096AE0D335
:1094D6009406748094804016E4F0900966E0640275
:1094E600600C7D1DAF16AE15129ACA123EC822E454
:1094F600901BA2F0A3F0901BA2E475F0011228497C
:10950600FE74A325F0F58274093EF583E070E790BA
:109516001BA2E0FEA3E024A3F974093EFA7B011224
:109526009013901BA4122A5CE47B02FAF9F8901BB4
:10953600A4E0FCA3E0FDA3E0FEA3E0FF12294FEFA9
:1095460024FFFFEE34FFFEED34FFFDEC34FFFC900C
:109556001BA8122A5C901BA8E0FCA3E0FDA3E0FE7A
:10956600A3E02470FFE43EFEE43DFDE43CFC901BDA
:10957600A8122A5C901BA2E475F001122849FE7419
:10958600A325F0F58274093EF583E070E7901BA8E9
:10959600E0FCA3E0FDA3E0FEA3E0FF901BA2E0F544
:1095A6002EA3E0F52F1287CBEF700302D76A12D7EE
:1095B6007C228B228A238924AB25AA26A927900000
:1095C6000412271464057008901CE37404F08015D7
:1095D60090000A122714600D90000AE41227869064
:1095E6001CE3E004F0901CE3E0C3940474809480D0
:1095F6005003029679E4F0AB22AA23A92412C88963
:10960600AB22AA23A92490000212285FFFAEF09095
:10961600000412285FFDACF0D39FEC9E4011D3ED01
:109626009470EC94177F0140027F038F28801DAB56
:1096360022AA23A92490000412285FFFAEF090000E
:109646000212285FD39FE5F09E752802AB25AA2655
:10965600A9279000021227146528600F900002E5E2
:1096660028122786900006E40227869000067401D9
:10967600122741228F538E528D518C5085A754A2AA
:10968600AF920085F555C2AFE4F5A7FF7E80FDFCDD
:10969600AB53AA52A951A850C3122A05500B8552A2
:1096A6005685535753F5CF8076E4FFFE7D01FCAB1C
:1096B60053AA52A951A850C3122A055020E553F5C2
:1096C60053E5524480F552E551F551E550F5508584
:1096D600525685535753F5CF43F51080427F007E8F
:1096E600807D017C00AB53AA52A951A850C3122A0F
:1096F600055020E553F553E5524480F552E551F502
:1097060051E550F55085525685535753F5CF43F5DD
:1097160020800C85525685535753F5CF43F5308537
:109726005782855683E493FF8555F58554A7A20095
:1097360092AF227536FF7537E475389C8F3C8E3BA9
:109746008D3A8C397B017A1C79B51243A48F247526
:109756003A607539E37538167537007F007E367DB9
:109766006E7C0112CF55E4F522F52374852523F589
:109776008274E63522F583E493FF12D78E0523E53E
:109786002370020522C3940AE522940040DDE4F525
:1097960022F523C3E5239524E5229400501B74B5D6
:1097A6002523F582741C3522F583E0FF12D78E053A
:1097B60023E52370DE052280DAE4FF12D78E7F646C
:1097C6007E007D007C0012B950EF701978007C0095
:1097D6007D017BFF7AE479A3122C93EF3395E04F5A
:1097E6007003FEFF227E007F01227D0A7FAC12A756
:1097F6000E901B9DE0F526900995E526F0FF12D602
:10980600BF90097CEFF0E48F25F524F523F522AE11
:1098160024AD23AC227810122A298F258E248D237D
:109826008C227D097FAC12A70E901B9DE0F5269039
:109836000996E526F0FF12D6BF90097DEFF0AF2618
:1098460012D6BFEF7F00FE3395E0FDFCEF2525F530
:1098560025E5243EF524E5233DF523E5223CF522C6
:109866007D087FAC12A70E901B9DE0F52690099708
:10987600E526F0FF12D6BF90097EEFF0AF2612D68E
:10988600BFE4FCFDFEE5252FF525EE3524F524ED98
:109896003523F523EC3522F522AF25AE24AD23FC86
:1098A600229000B8E0FF12D6BF900988EFF0900032
:1098B600B9E0FF12D6BF900989EFF09000BAE0FF39
:1098C60012D6BF90098AEFF09000BBE0FF12D6BF18
:1098D60090098BEFF09000BCE0FF12D6BF90098C88
:1098E600EFF09000BDE0FF12D6BF90098DEFF0902B
:1098F60000BEE0FF12D6BF90098EEFF09000C1E0E7
:10990600FF12D6BF90099AEFF09000C2E0FF12D680
:10991600BF90099BEFF09000C3E0FF12D6BF9009FD
:109926009CEFF09000C4E0FF12D6BF90099DEFF0C7
:109936009000C5E0FF12D6BF90099EEFF09000C6DA
:10994600E0FF12D6BF90099FEFF09000C7E0FF122C
:10995600D6BF9009A0EFF0227536FF7537E475384B
:109966009C8F3C8E3B8D3A8C397B017A1C79B512E3
:1099760043A48F24753A607539E375381675370038
:109986007F007E367D6E7C0112CF55E4F522F523ED
:10999600745F2523F58274E53522F583E493FF127F
:1099A600D78E0523E52370020522C39411E5229480
:1099B6000040DDE4F522F523C3E5239524E5229452
:1099C60000501B74B52523F582741C3522F583E0FF
:1099D600FF12D78E0523E52370DE052280DAE4FF29
:1099E60012D78E7F647E007D007C0012B950EF7026
:1099F6001A78007C007D017BFF7AE479C4122C93EF
:109A0600EF3395E04F7F017004FF227F0122E4903F
:109A16001BA2F0A3F0901BA2E475F001122849FEE8
:109A260074A325F0F58274093EF583E070E7901B78
:109A3600A2E0FEA3E024A3F974093EFA7B0112908A
:109A460013901BA4122A5C7E097F607D007B017A3D
:109A5600007900122E5A901BA4E0FCA3E0FDA3E0BF
:109A6600FEA3E0FF12B504EF704D901BA2F0A3F029
:109A7600901BA2E0FEA3E0FFC3EE940850457400DD
:109A86002FF58274003EF583E0FF12D84B50181272
:109A9600D832901BA2E0FEA3E02400F58274003EBB
:109AA600F583E0FF12D800901BA3E004F070C1908C
:109AB6001BA2E004F080B912D8327BFF7ADF79B2BC
:109AC6001243AA228E2A8F2B8D2C12B0048F308E31
:109AD6002F8D2E8C2D7F007E487D017C00AB30AA19
:109AE6002FA92EA82DC3122A054003029B797E00BA
:109AF6007F0A7D007B017A1C790C122E5AE52B24F5
:109B060004F582E4352AF583E0901C0CF0E52B245D
:109B160005F582E4352AF583E0901C0DF0E52B244B
:109B260006F582E4352AF583E0901C0EF0852B823B
:109B3600852A83A3A3A3E0901C0FF0852B82852A98
:109B460083A3E0901C10F0852B82852A83E0901C6D
:109B560011F0A3E52CF0E4A3F0A3F0A3F0AF30AE30
:109B66002FAD2EAC2D7B017A1C790CF54275430A7C
:109B760012BE9A22E4901BA2F0A3F0901BA2E475F9
:109B8600F001122849FE74A325F0F58274093EF50A
:109B960083E070E7901BA2E0FEA3E024A3F974091A
:109BA6003EFA7B01129013901BA4122A5C901BA410
:109BB600E0FCA3E0FDA3E0FEA3E0FF12B581EF7099
:109BC6005512D8327BFF7AE0799B901BA4E0FCA368
:109BD600E0FDA3E0FEA3E0F5398E388D378C361212
:109BE60043AAE4901BA2F0A3F0901BA2E0FEA3E020
:109BF600FFC3EE9408502B74002FF58274003EF5D7
:109C060083E0FF12D800901BA3E004F070DB901BEA
:109C1600A2E004F080D312D8327BFF7AE079AD124D
:109C260043AA228B238A248925AB23AA24A9251299
:109C360026FBFF12D757500D74012525F525E4356F
:109C460024F52480E4D200AB23AA24A9251226FBFE
:109C5600FF642B6004EFB42D1BAB230525E525AA75
:109C6600247002052414F91226FB642D6003D380A8
:109C760001C39200E4F526F527AB23AA24A92512F1
:109C860026FBFF12D85A5036AB23AA24A925122642
:109C9600FBFF3395E0FEEF24D0FBEE34FFFAAE2651
:109CA600AF277C007D0A122E86EF2BF527EE3AF5BC
:109CB6002674012525F525E43524F52480BB3000DE
:109CC60006AE26AF278009C3E49527FFE49526FE56
:109CD60022E4901BA2F0A3F0901BA2E475F00112FF
:109CE6002849FE74A325F0F58274093EF583E070D9
:109CF600E7901BA2E0FEA3E024A3F974093EFA7BD9
:109D060001129013901BA4122A5C7E097F607D00CD
:109D16007B017A007900122E5AE4901BA2F0A3F080
:109D2600A3E0FCA3E0FDA3E0FEA3E0FF12B40AEF6C
:109D3600703F12D832E4901BA2F0A3F0900960E0C5
:109D4600FEA3E0FF901BA2E0FCA3E0FDC39FEC9EF8
:109D5600502B74002DF58274003CF583E0FF12D879
:109D660000901BA3E004F070D3901BA2E004F080E7
:109D7600CB12D8327BFF7ADE79FF1243AA221284F5
:109D8600B6EF600C12D8327BFF7AE07960029E282B
:109D960012CBE5EF600C12D8327BFF7AE0797402C1
:109DA6009E2878007C007D017BFF7AE07995122C55
:109DB60093EF3395E04F60617E117F947D007B01C8
:109DC6007A0979A3122E5A78A37C097D017B017A40
:109DD6000079007E097F601226D5E4901BA2F0A3CD
:109DE600F012D832901BA2E475F001122849FE74D5
:109DF600A325F0F58274093EF583E0602D901BA241
:109E0600E0FEA3E024A3F58274093EF583E0FF1289
:109E1600D800E4FF12D80080CB12D8327BFF7AE05C
:109E260079981243AAE4FF12D800228E228F23E4E7
:109E3600FD7FAC12A70E901B9DE0901BA6F044F789
:109E4600F0FB7A00E4FD7FAC12B8DC8007901BA61D
:109E5600E030E7117D037FAC12A70E901B9DE090CA
:109E66001BA6F080E8AB23AA227D287FAC12B8DCC3
:109E76008007901BA6E030E71412C6E47D037FAC92
:109E860012A70E901B9DE0901BA6F080E5E5227AB6
:109E960000FB7D297FAC12B8DC8007901BA6E03062
:109EA600E71412C6E47D037FAC12A70E901B9DE05B
:109EB600901BA6F080E5E4FD7FAC12A70E901B9DDB
:109EC600E0901BA6F04408F0FB7A00E4FD7FAC02AC
:109ED600B8DC90096F122A680000000090096FE054
:109EE600FCA3E0FDA3E0FEA3E0FF901BA2EFF09031
:109EF600096FA3A3A3E07808122A16901BA3EFF01C
:109F060090096FE0FCA3E0FDA3E0FEA3E0FF78105C
:109F1600122A16E4901BA4EFF07E1B7FA27D037C21
:109F26000012D32C901BA5EFF0901BA2E0FD7F380A
:109F360012D892901BA3E0FD7F3912D892901BA4F1
:109F4600E0FD7F3A12D892901BA5E0FD7F3B12D828
:109F560092901BA2E0FD7F3C12D892901BA3E0FDDD
:109F66007F3D12D892901BA4E0FD7F3E12D89290BE
:109F76001BA5E0FD7F3F02D8921297F0E4901BA24A
:109F8600F0A3F012BA38EF600C12D8327BFF7ADFFA
:109F960079DF02A02212D8327BFF7AE079E61243FB
:109FA600AA12C47CEF60087BFF7ADF79F2806D7BB2
:109FB600FF7AE079FC1243AA12B2107E047F007D7C
:109FC600007B017A0D79A3122E5A78A37C097D01B4
:109FD6007B017A0079007E047F001226D57E097FF8
:109FE600A37DFE7C0312D32C900DA1EFF07B017AAA
:109FF6000979A37DFF7C0312CFFE900DA2EFF0E45A
:10A00600F526F5277F907E08FDFC128B9AEF7BFFE5
:10A0160070067AE1790D80047AE179261243AA2244
:10A026008B228A2389248F288E278D268C2585A727
:10A03600297531007530C2752F01752E007F007E9F
:10A04600367D6E7C0112CEDF75A710C298901BA6D6
:10A05600122A6800000000AF28AE27AD26AC259076
:10A066001BA6E0F8A3E0F9A3E0FAA3E0FBC3122ADB
:10A0760005503B901BA6A3A3E0FEA3E0AB22AA23B8
:10A08600A924F5828E83122714FF12D78E901BA661
:10A09600E0FCA3E0FDA3E0FEA3E02401FFE43EFE16
:10A0A600E43DFDE43CFC901BA6122A5C80A9C29903
:10A0B600C2988529A7901BA6E0FCA3E0FDA3E0FEBD
:10A0C600A3E0FF22900020E064547052A3E06441B4
:10A0D600704CA3E064537046A3E0B44B41E4901B7C
:10A0E600ACF0A3F0901BACE0FEA3E0FF2420F582C9
:10A0F60074003EF583E0FD74A32FF58274093EF5E6
:10A1060083EDF0901BADE004F07006901BACE0040C
:10A11600F0901BACE0B404CCA3E0B400C7229009D5
:10A126006CE064017040901BACF0A3F0901BACE0B7
:10A13600FEA3E0FF2481F58274E83EF583E493FDF7
:10A1460074A32FF58274093EF583EDF0901BADE004
:10A1560004F07006901BACE004F0901BACE07004B9
:10A16600A3E0642070C6228E228F23753A6075396B
:10A17600E37538167537007F007E367D6E7C0112DA
:10A18600CF55E4F524F52574E72525F58274E635E3
:10A1960024F583E493FF12D78E0525E52570020585
:10A1A60024C3940CE524940040DD852224852325D0
:10A1B600E42523FFE5223404FEC3E5259FE5249E1E
:10A1C600501B74A32525F58274093524F583E0FF19
:10A1D60012D78E0525E52570D7052480D37FB07E5E
:10A1E600047D007C0012B950EF701A78007C007D67
:10A1F600017BFF7AE479A3122C93EF3395E04F7F2E
:10A20600017004FF227F01228E268F27753A607522
:10A2160039E37538167537007F007E367D6E7C0112
:10A2260012CF55E4F528F52974032529F58274E73C
:10A236003528F583E493FF12D78E0529E5297002A8
:10A246000528C39413E528940040DD852628852734
:10A2560029E42527FFE5263404FEC3E5299FE528E2
:10A266009E501B74A32529F58274093528F583E0D1
:10A27600FF12D78E0529E52970D7052880D37FB030
:10A286007E047D007C0012B950EF701A78007C00C5
:10A296007D017BFF7AE479A3122C93EF3395E04F8F
:10A2A6007F017004FF227F01228E288F29753A6074
:10A2B6007539E37538167537007F007E367D6E7CFE
:10A2C6000112CF55E4F52AF52B7416252BF5827469
:10A2D600E7352AF583E493FF12D78E052BE52B701D
:10A2E60002052AC3940BE52A940040DD85282A85B9
:10A2F600292BE42529FFE5283404FEC3E52B9FE539
:10A306002A9E501B74A3252BF5827409352AF583E2
:10A31600E0FF12D78E052BE52B70D7052A80D37F59
:10A32600B07E047D007C0012B950EF701A78007C74
:10A33600007D017BFF7AE479A3122C93EF3395E03D
:10A346004F7F017004FF227F0122E4901BA2F0A33D
:10A35600F0901BA2E475F001122849FE74A325F0C3
:10A36600F58274093EF583E070E7901BA2E0FEA338
:10A37600E024A3F974093EFA7B01129013901BA402
:10A38600122A5C7E097F607D007B017A00790012CB
:10A396002E5A901BA4E0FCA3E0FDA3E0FEA3E0FF81
:10A3A60012B504EF703712D832E4901BA2F0A3F076
:10A3B600901BA2E0FEA3E0FFC3EE9404502B7400B2
:10A3C6002FF58274003EF583E0FF12D800901BA3A0
:10A3D600E004F070DB901BA2E004F080D312D832C8
:10A3E6007BFF7ADF79B21243AA22E4901BA2F0A384
:10A3F600F0901BA2E475F001122849FE74A325F023
:10A40600F58274093EF583E070E7901BA2E0FEA397
:10A41600E024A3F974093EFA7B01129013901BA461
:10A42600122A5C7E097F607D007B017A007900122A
:10A436002E5A901BA4E0FCA3E0FDA3E0FEA3E0FFE0
:10A4460012B504EF703712D832E4901BA2F0A3F0D5
:10A45600901BA2E0FEA3E0FFC3EE9404502B740011
:10A466002FF58274043EF583E0FF12D800901BA3FB
:10A47600E004F070DB901BA2E004F080D312D83227
:10A486007BFF7ADF79B21243AA22E4901BA2F0A3E3
:10A49600F0901BA2E475F001122849FE74A325F082
:10A4A600F58274093EF583E070E77B017A0979A3AA
:10A4B600901BA2E0FEA3E0FFE4FCFD12A0267B01B8
:10A4C6007A0979A37F947E117D007C0012D9657E7E
:10A4D60000901BA2EEF0A3EFF0603D12D832E4909C
:10A4E6001BA4F0A3F0901BA2E0FEA3E0FFA3E0FCF8
:10A4F600A3E0FDC39FEC9E502274A32DF582740940
:10A506003CF583E0FF12D800901BA5E004F070D55F
:10A51600901BA4E004F080CD12D77C7E117F947D41
:10A52600007B017A0979A3022E5AE4901BA2F0A3BC
:10A53600F0901BA2E475F001122849FE74A325F0E1
:10A54600F58274093EF583E070E77B017A0979A309
:10A55600901BA2E0FEA3E0FFE4FCFD12A0267B0117
:10A566007A0979A37F947E117D007C0012D9657EDD
:10A5760000901BA2EEF0A3EFF0603D12D832E490FB
:10A586001BA4F0A3F0901BA2E0FEA3E0FFA3E0FC57
:10A59600A3E0FDC39FEC9E502274A32DF58274099F
:10A5A6003CF583E0FF12D800901BA5E004F070D5BF
:10A5B600901BA4E004F080CD12D77C7E117F947DA1
:10A5C600007B017A0979A3022E5A12D832E4901B35
:10A5D600A2F0A3F0901BA2E0FEA3E0FFC3EE94045A
:10A5E600501F74A32FF582740D3EF583E0FF12D839
:10A5F60000901BA3E004F070DB901BA2E004F08047
:10A60600D3E4FF7E08FDFC901BA5E0F8A3E0F9A3C8
:10A61600E0FAA3E0FBC3122A05501CE4FF7E04FD0A
:10A62600FC901BA5E0F8A3A3A3E0122A054008901E
:10A636001BA4E0FF12D800E4901BA2F0A3F0901B2D
:10A64600A2E0FEA3E0FFC3EE9404501C74A32FF512
:10A6560082740D3EF583E4F0901BA3E004F070DEF7
:10A66600901BA2E004F080D62212D832E4901BA2FE
:10A67600F0A3F0901BA2E0FEA3E0FFC3EE9404500B
:10A686001F74A32FF58274113EF583E0FF12D800E4
:10A69600901BA3E004F070DB901BA2E004F080D3D3
:10A6A600E4FF7E0CFDFC901BA4E0F8A3E0F9A3E018
:10A6B600FAA3E0FBC3122A05501CE4FF7E08FDFC4A
:10A6C600901BA4E0F8A3A3A3E0122A054008901B60
:10A6D600A8E0FF12D800E4901BA2F0A3F0901BA202
:10A6E600E0FEA3E0FFC3EE9404501C74A32FF58292
:10A6F60074113EF583E4F0901BA3E004F070DE9045
:10A706001BA2E004F080D6228F2C8D2D85A72E75F6
:10A71600A710E52C64AC703B12D731E4FDAF2C12C8
:10A72600CD59EF7010AF2D12D447EF700512D6D564
:10A7360080067F01227F012212D7317D01AF2C12C4
:10A74600CD59EF700B12D420901B9D12D6CE8003EC
:10A756007F0122E52C6480704612D731E4FDAF2CD0
:10A7660012CD59EF7010AF2D12D447EF700512D6E7
:10A77600D080067F01227F012212D7317D01AF2CC6
:10A7860012CD59EF701612D420901B9DEFF0E4FF06
:10A7960012D4E112D420A312D6CE80037F012285E3
:10A7A6002EA77F00227B017A1C79167E1C7F227DD4
:10A7B600407C008E3F8F408C418D428B438A44897A
:10A7C60045AA06A9077B0112D6A58E468F47E4F552
:10A7D60048F549C3E5479542E54695415061AB4387
:10A7E600AA44A945854982854883122714FF3395D3
:10A7F600E04F603DE5472401FFE43546FEC3EF9593
:10A8060042EE9541502B0549E549AE487002054890
:10A8160014F5828E83122714FF0547E547AC467070
:10A82600020546142540F582E53F3CF583EFF080AE
:10A83600ADE5402547F582E53F3546F583E4F02250
:10A84600E4901BA2F0A3F0901BA2E475F00112287D
:10A8560049FE74A325F0F58274093EF583E070E79E
:10A86600901BA2E0FEA3E024A3F974093EFA7B0143
:10A87600129013901BA4122A5C901BA4E0FCA3E088
:10A88600FDA3E0FEA3E0FF12B487EF703F12D832BB
:10A89600E4901BA2F0A3F0900960E0FEA3E0FF9015
:10A8A6001BA2E0FCA3E0FDC39FEC9E502B74002D81
:10A8B600F58274003CF583E0FF12D800901BA3E0FC
:10A8C60004F070D3901BA2E004F080CB12D8327B48
:10A8D600FF7ADF79531243AA228D828C83E0FB8FA5
:10A8E600828E83E06B600302A9718D828C83A3E064
:10A8F600FB8F828E83A3E06B70718D828C83A3A302
:10A90600E0FB8F828E83A3A3E06B705F8D828C83C6
:10A91600A3A3A3E0FB8F828E83A3A3A3E06B704B5C
:10A92600ED2404F582E43CF583E0FBEF2404F58294
:10A93600E43EF583E06B7033ED2405F582E43CF5E7
:10A9460083E0FBEF2405F582E43EF583E0B5031BC7
:10A95600ED2406F582E43CF583E0FDEF2406F5825E
:10A96600E43EF583E0B505037F01227F002212D97C
:10A9760039787FE4F6D8FD75816D12D60002A9C13B
:10A9860002D92AE493A3F8E493A34003F68001F2E4
:10A9960008DFF48029E493A3F85407240CC8C333D2
:10A9A600C4540F4420C8834004F456800146F6DFA1
:10A9B600E4800B010204081020408090C4D7E47E96
:10A9C600019360BCA3FF543F30E509541FFEE49396
:10A9D600A360010ECF54C025E060A840B8E493A35D
:10A9E600FAE493A3F8E493A3C8C582C8CAC583CA88
:10A9F600F0A3C8C582C8CAC583CADFE9DEE780BE40
:10AA0600E4FD7FAC12A70E901B9DE0901BA8F044BE
:10AA1600F7F0FB7A00E4FD7FAC12B8DC8007901BF0
:10AA2600A8E030E7117D037FAC12A70E901B9DE0D6
:10AA3600901BA8F080E87D287FAC12A70E901B9D86
:10AA4600E0901BA8F07D297FAC12A70E901B9DE01D
:10AA5600FF901BA4E4F0A3EFF0E0FE901BA8E07CBF
:10AA6600002400FFEC3E901BA6F0A3EFF0E4FD7F70
:10AA7600AC12A70E901B9DE0901BA8F04408F0FBBB
:10AA86007A00E4FD7FAC12B8DC901BA6E0FEA3E0E2
:10AA9600FF22E517700302AB28E4F517901CE5E0EA
:10AAA60004F0E0D3941E748094804002E4F0901C7D
:10AAB600E5E0FFC31390E90E9324FF9297E5146433
:10AAC6000170057F1312B9C475250175260975270E
:10AAD600647B017A1B79371295B890096AE0D394A2
:10AAE6000674809480403BE4F0900966E06402605E
:10AAF6003112D5E9900966E06401700F12D37F9098
:10AB060009687407F09009677409F0900966E064B3
:10AB160003700F12D37F9009687401F0900967746F
:10AB260009F022E4901BA2F0A3F0901BA2E475F0BA
:10AB360001122849FE74A325F0F58274093EF583B7
:10AB4600E070E7901BA2E0FEA3E024A3F974093E9F
:10AB5600FA7B01129013901BA4122A5C7E097F6077
:10AB66007D007B017A007900122E5A901BA4E0FC2E
:10AB7600A3E0FDA3E0FEA3E0FF12B50412D832E481
:10AB8600901BA2F0A3F0901BA2E0FEA3E0FFC3EE91
:10AB96009408501F74002FF58274003EF583E0FF81
:10ABA60012D800901BA3E004F070DB901BA2E00417
:10ABB600F080D322E4901BA2F0A3F0901BA2E475D0
:10ABC600F001122849FE74A325F0F58274093EF5BA
:10ABD60083E070E7901BA2E0FEA3E024A3F97409CA
:10ABE6003EFA7B01129C29901BA4EEF0A3EFF01213
:10ABF600C0B0EF703F12D832E4901BA2F0A3F090E1
:10AC06000960E0FEA3E0FF901BA2E0FCA3E0FDC309
:10AC16009FEC9E502B74002DF58274003CF583E06A
:10AC2600FF12D800901BA3E004F070D3901BA2E0A3
:10AC360004F080CB12D8327BFF7ADF792D1243AA3B
:10AC460022E4901BA2F0A3F0901BA2E475F001127F
:10AC56002849FE74A325F0F58274093EF583E07059
:10AC6600E7901BA2E0FEA3E024A3F974093EFA7B59
:10AC760001129C29901BA4EEF0A3EFF07B017A0948
:10AC860079A312743A12D832E4901BA2F0A3F09082
:10AC96001BA2E0FCA3E0FDC3EC94045030901BA57E
:10ACA600E07F0025E025E0FEEF2DFFEC3EFE74A3DD
:10ACB6002FF58274093EF583E0FF12D800901BA39E
:10ACC600E004F070CA901BA2E004F080C222E49077
:10ACD6001BA2F0A3F0901BA2E475F001122849FE16
:10ACE60074A325F0F58274093EF583E070E7901BA6
:10ACF600A2E475F001122849FE74A325F0F58274CA
:10AD0600093EF583E070E7901BA2E475F001122876
:10AD160049FE74A325F0F58274093EF583E070E7D9
:10AD2600901BA2E475F001122849FE74A325F0F5E4
:10AD36008274093EF583E070E7901BA2E0FEA3E073
:10AD460024A3F974093EFA7B01129C29901BA4EEF8
:10AD5600F0A3EFF0129E3102D76A8E228F238C2445
:10AD66008D257E097F607D007B017A007900122E99
:10AD76005A753AE07539937538047537007F007E49
:10AD8600367D6E7C0112CF55E4F526F527C3E527FF
:10AD96009525E5269524501BE5232527F582E522F2
:10ADA6003526F583E0FF12D78E0527E52770DE05E9
:10ADB6002680DA7F327E007D007C0012B950EF706B
:10ADC60020F526F5270527E527AE26700205261469
:10ADD6002400F58274003EF583E070E9AE26AF27C5
:10ADE60022E4FEFF228E288F298C2A8D2B7D0E7F52
:10ADF600AC12A70E12D6BA852982852883EFF09069
:10AE06001B9DE0852B82852A83F07D0D7FAC12A7E2
:10AE16000E12D6BA852982852883A3EFF0901B9D52
:10AE2600E0852B82852A83A3F07D0B7FAC12A70ECB
:10AE360012D6BA852982852883A3A3A3EFF0901B97
:10AE46009DE0852B82852A83A3A3A3F07D0C7FAC8E
:10AE560012A70E12D6BA852982852883A3A3EFF0FE
:10AE6600901B9DE0852B82852A83A3A3F07F002279
:10AE76008E288F298C2A8D2B7D0A7FAC12A70E1265
:10AE8600D6BAE5292404F582E43528F583EFF09057
:10AE96001B9DE0FFE52B2404F582E4352AF583EFBC
:10AEA600F07D097FAC12A70E12D6BAE5292405F566
:10AEB60082E43528F583EFF0901B9DE0FFE52B2417
:10AEC60005F582E4352AF583EFF07D087FAC12A7FD
:10AED6000E12D6BAE5292406F582E43528F583EF65
:10AEE600F0901B9DE0FFE52B2406F582E4352AF55C
:10AEF60083EFF07F00221298A712D96812D95F8FCC
:10AF0600118E108D0F8C0E12BF068F22EF64027009
:10AF160050FFFEFDFCAB11AA10A90FA80EC3122A02
:10AF260005700A12D37F9009687403802190096620
:10AF3600E0640160217F0112D66312D9687D03AFF8
:10AF460016AE15129ACA124BF39009687405F09062
:10AF560009677409F0227D22AF16AE15129ACA80CF
:10AF660006E52264037003023EC89009687403F084
:10AF76009009677409F012D37F227542007541402B
:10AF8600754001753F00753E00753D30753C017595
:10AF96003B007F007E407D017C00AB3EAA3DA93C84
:10AFA600A83BC3122A05504DAF3EAE3DAD3CAC3B6F
:10AFB6007B017A1B79D7754A00754B0312BDBF908A
:10AFC6001BD7E0F47018A3E0F47013A3E0F4700E3E
:10AFD600853E42853D41853C40853B3F8017E53EA9
:10AFE6002440F53EE4353DF53DE4353CF53CE4359D
:10AFF6003BF53B809DAF42AE41AD40AC3F2275383C
:10B006000075374075360175350075340075334067
:10B016007532017531007F007E487D017C00AB34BE
:10B02600AA33A932A831C3122A05504DAF34AE3324
:10B03600AD32AC317B017A1B79D6754A00754B036C
:10B0460012BDBF901BD6E0F47018A3E0F47013A3F2
:10B05600E0F4700E853438853337853236853135E0
:10B066008017E534240AF534E43533F533E4353214
:10B07600F532E43531F531809DAF38AE37AD36ACBB
:10B0860035227535007534407533017532007531DA
:10B0960000753048752F01752E007F007E507D01AA
:10B0A6007C00AB31AA30A92FA82EC3122A05504D19
:10B0B600AF31AE30AD2FAC2E7B017A1B79A2754A2B
:10B0C60000754B0312BDBF901BA2E0F47018A3E0FD
:10B0D600F47013A3E0F4700E853135853034852F76
:10B0E60033852E328017E531240AF531E43530F503
:10B0F60030E4352FF52FE4352EF52E809DAF35AE95
:10B1060034AD33AC322212D9687536FF7537E17526
:10B116003860900978E0753900F53AA3E0753B0090
:10B12600F53C90097BE0753D00F53EA3E0753F00D8
:10B13600F540A3E0754100F542A3E0754300F544F0
:10B146007B017A0979A31243A4901BA212D82DE49D
:10B15600901BA4F0A3F0901BA2E0FEA3E0FFA3E0E7
:10B16600FCA3E0FDC39FEC9E501F74A32DF58274D3
:10B17600093CF583E0FF12D800901BA5E004F070AF
:10B18600D5901BA4E004F080CD227E097F607D006F
:10B196007B017A007900122E5A753A607539E3758B
:10B1A60038167537007F007E367D6E7C0112CF55CE
:10B1B600E4F522F52374702523F58274E53522F52E
:10B1C60083E493FF12D78E0523E52370020522C37D
:10B1D600940FE522940040DD7F647E007D007C00B4
:10B1E60012B950EF7020F522F5230523E523AE2290
:10B1F60070020522142400F58274003EF583E07087
:10B20600E9AE22AF2322E4FEFF229000317401F062
:10B21600901B93E0900025F0901B94E0900026F0A0
:10B22600901B95E0900027F0901B96E0900028F088
:10B23600901B97E0900029F0901B98E090002AF070
:10B24600901B99E090002BF0901B9AE090002CF058
:10B25600900991E09000DCF0900992E09000DDF01A
:10B26600900993E09000DEF0900994E09000DFF002
:10B27600900995E09000E0F0900996E09000E1F0EA
:10B28600900997E09000E2F022E48F2C8E2BF52AAD
:10B29600F529900968E06401702CAD2AAC297B374A
:10B2A600FAF9F81228C48F2C8E2B8D2A8C29E47B70
:10B2B600E87A03F9F81228C48F2C8E2B8D2A8C2954
:10B2C600E4FB7A0C8030AF2CAE2BAD2AAC29E47BA4
:10B2D60037FAF9F81228C48F2C8E2B8D2A8C29E484
:10B2E6007BE87A03F9F81228C48F2C8E2B8D2A8CD2
:10B2F60029E47B997A09F9F812294F8F2C8E2B8D28
:10B306002A8C29AE2BAF2C22E4901BA2F0A3F012BC
:10B31600CA69EF704412D832E4901BA2F0A3F090F1
:10B326000960E0FEA3E0FF901BA2E0FCA3E0FDC3E2
:10B336009FEC9E501F74002DF58274003CF583E04F
:10B34600FF12D800901BA3E004F070D3901BA2E07C
:10B3560004F080CBE4FF02D80012D832E4901BA29E
:10B36600F0A3F0E4FF12D800901BA3E004F07006EF
:10B37600901BA2E004F0C3901BA3E09410901BA2C4
:10B38600E0940040DE22E4901BA2F0A3F012CAB6BD
:10B39600EF704412D832E4901BA2F0A3F09009603B
:10B3A600E0FEA3E0FF901BA2E0FCA3E0FDC39FEC40
:10B3B6009E501F74002DF58274003CF583E0FF1249
:10B3C600D800901BA3E004F070D3901BA2E004F019
:10B3D60080CBE4FF02D80012D832E4901BA2F0A37F
:10B3E600F0E4FF12D800901BA3E004F07006901B57
:10B3F600A2E004F0C3901BA3E09410901BA2E0947B
:10B406000040DE227536FF7537E475389C8F3C8E1A
:10B416003B8D3A8C397B017A1C79B51243A48F2374
:10B42600753A607539E37538167537007F007E36D4
:10B436007D6E7C0112CF55E4F522C3E522940C748F
:10B44600809480500EE52290E5ED93FF12D78E058D
:10B456002280E7E4F522E522C39523501474B5252E
:10B4660022F582E4341CF583E0FF12D78E05228094
:10B47600E5E4FF12D78E7FC87E007D007C0002B90E
:10B48600507536FF7537E475389C8F3C8E3B8D3A88
:10B496008C397B017A1C79B51243A48F23753A60E7
:10B4A6007539E37538167537007F007E367D6E7CFC
:10B4B6000112CF55E4F522C3E522941074809480DE
:10B4C600500EE52290E63193FF12D78E052280E7D3
:10B4D600E4F522E522C39523501474B52522F5829E
:10B4E600E4341CF583E0FF12D78E052280E5E4FFE5
:10B4F60012D78E7F807EEE7DFF7CFF02B9507536B7
:10B50600FF7537E475389C8F3C8E3B8D3A8C397BC2
:10B51600017A1C79B51243A48F24753A607539E314
:10B526007538167537007F007E367D6E7C0112CF2A
:10B5360055E4F523C3E523940974809480500EE501
:10B546002390E64893FF12D78E052380E7E4F52380
:10B55600E523C39524501474B52523F582E4341CE1
:10B56600F583E0FF12D78E052380E5E4FF12D78E20
:10B576007FC87E007D007C0002B9507536FF7537A6
:10B58600E475389C8F3C8E3B8D3A8C397B017A1C56
:10B5960079B51243A48F23753A607539E375381669
:10B5A6007537007F007E367D6E7C0112CF55E4F53F
:10B5B60022C3E522941074809480500EE52290E513
:10B5C6004F93FF12D78E052280E7E4F522E522C3CA
:10B5D6009523501474B52522F582E4341CF583E0D6
:10B5E600FF12D78E052280E5E4FF12D78E7FC87E34
:10B5F600007D007C0002B950900967E06401603369
:10B606007401F012D10012D8D11220267FB07E71BB
:10B616007D0B7C0012C6377F011220967F01122017
:10B62600067F0112D66312AA06900964EEF0A3EF14
:10B63600F0D297E5176006E4F517128E50125E9564
:10B64600EF700C12D8FC122E9812D906127283755E
:10B6560025017526097527647B017A1B79371295B2
:10B66600B890096AE0D39402748094804005E4F0AF
:10B6760012CE6022900967E0640360037403F0E56C
:10B6860017606CE4F517901CE4E004F0E0D3941E18
:10B69600748094804002E4F0901CE4E0FFC31390B1
:10B6A600E8FE9324FF929775250175260975276490
:10B6B6007B017A1B79371295B890096AE0D3940614
:10B6C600748094804029E4F0900966E06402601F6B
:10B6D600A37409F0900966E0640170069009687425
:10B6E60007F0900966E06403700590096804F0228B
:10B6F6007F3812D885901B93EFF07F3912D885904A
:10B706001B94EFF07F3A12D885901B95EFF07F3BA4
:10B7160012D885901B96EFF07F3C12D885901B9728
:10B72600EFF07F3D12D885901B98EFF07F3E12D840
:10B7360085901B99EFF07F3F12D885901B9AEFF00A
:10B746007E1B7F937D047C0012D32C8F227E1B7F71
:10B75600977D047C0012D32CE52270028003EF70E3
:10B7660003FF8003E47F01FEFDFC228B228A2389EE
:10B77600248F288E278D268C25E4F529F52A12D5C7
:10B786007BE47F04FEFDFCAB28AA27A926A8251288
:10B7960028C4AB69AA68A967A866C3122A05500619
:10B7A600E565456460DBE47F08FEFDFCAB69AA68DD
:10B7B600A967A866C3122A0540EC53E7F79009600B
:10B7C600E564F0A3E565F0AE68AF69A3EEF0A3EF1C
:10B7D600F0D3900961E09400900960E094007F0145
:10B7E60040027F0022E4901BA2F0A3F0901BA2E48B
:10B7F60075F001122849FE74A325F0F58274093EFE
:10B80600F583E070E7901BA2E0FEA3E024A3F974A1
:10B81600093EFA7B01129013901BA4122A5C901B1E
:10B82600A4E0FCA3E0FDA3E0FEA3E0FF12995EEF17
:10B83600702012D8327BFF7AE07937901BA4E0FCA7
:10B84600A3E0FDA3E0FEA3E0F5398E388D378C36F4
:10B85600800912D8327BFF7AE079531243AA227EFE
:10B86600097F607D007B017A007900122E5A12C38F
:10B87600C6EF7055901BA2F0A3F0901BA2E0FEA3AA
:10B88600E0FFC3EE9408503974002FF58274003E31
:10B89600F583E0FF12D84B501812D832901BA2E065
:10B8A600FEA3E02400F58274003EF583E0FF12D883
:10B8B60000901BA3E004F070C1901BA2E004F0808E
:10B8C600B97BFF7ADE796A800912D8327BFF7ADF8C
:10B8D600798D1243AA228F268D278A288B2985A740
:10B8E6002A75A710E52664AC702412CD52EF701BA2
:10B8F600AF2712D447EF7010AF2912D447EF700567
:10B9060012D6D580097F01227F01227F0122E526FA
:10B916006480703012CD52EF7027AF2712D447EFF4
:10B92600701CE528FF12D447EF7010AF2912D447D8
:10B93600EF700512D6D5800C7F01227F01227F0190
:10B94600227F0122852AA77F00228F368E358D34ED
:10B956008C33E4F537F53812D57BE47F04FEFDFC25
:10B96600AB36AA35A934A8331228C4AB69AA68A98C
:10B9760067A866C3122A055006E565456460DBE4E0
:10B986007F08FEFDFCAB69AA68A967A866C3122AF0
:10B996000540EC53E7F7900960E564F0A3E565F030
:10B9A600AE68AF69A3EEF0A3EFF0D3900961E0941F
:10B9B60000900960E094007F0140027F00228F2200
:10B9C600E4F51412D10012202612D8D17F011220DC
:10B9D600067F0112D66312D5E912C3C6EF70028044
:10B9E6003C7F2C7E0112D13212C3C6EF7002802D2D
:10B9F6007F2C7E0112D13212C3C6EF7002801E7DEB
:10BA060012AF16AE15129ACA7B017A00790012D4CB
:10BA1600B7EF700E7D1CAF16AE15129ACAAF220292
:10BA2600D22212D37F9009687403F09009677409D3
:10BA3600F022753A607539E37538167537007F0060
:10BA46007E367D6E7C0112CF55E4F527C3E527943B
:10BA56000C74809480500EE52790E53093FF12D742
:10BA66008E052780E77F887E137D007C0012B95003
:10BA7600EF702EC3900961E09402900960E0940093
:10BA8600401C78007C007D017BFF7AE479A37E0070
:10BA96007F02122E36EF3395E04F7002FF227F01B0
:10BAA600227F0122753A607539E3753816753700BD
:10BAB6007F007E367D6E7C0112CF55E4F522C3E50C
:10BAC60022940374809480500EE52290E60493FF3E
:10BAD60012D78E052280E77F0A7E007D007C001249
:10BAE600B950EF702EC3900961E09402900960E0AE
:10BAF6009400401C78007C007D017BFF7AE479A3EA
:10BB06007E007F02122E36EF3395E04F7002FF2241
:10BB16007F01227F0122753A607539E37538167503
:10BB260037007F007E367D6E7C0112CF55E4F5220C
:10BB3600C3E522940974809480500EE52290E4C7F0
:10BB460093FF12D78E052280E77F0A7E007D007C58
:10BB56000012B950EF702EC3900961E0940290096B
:10BB660060E09400401C78007C007D017BFF7AE455
:10BB760079A37E007F02122E36EF3395E04F7002D6
:10BB8600FF227F01227F0122900991E09009AFF008
:10BB9600900992E09009B0F0900993E09009B1F015
:10BBA600900994E09009B2F0900995E09009B3F0FD
:10BBB600900996E09009B4F0900997E09009B5F0E5
:10BBC60012D832E4901BA2F0A3F0901BA2E0FEA3D1
:10BBD600E0FFC39413EE9400501F74A32FF58274F4
:10BBE600093EF583E0FF12D800901BA3E004F07035
:10BBF600D9901BA2E004F080D12212D832E4901B27
:10BC0600A2F0A3F0901BA2E0FEA3E0FFC3EE940413
:10BC1600501F74A32FF58274153EF583E0FF12D8EA
:10BC260000901BA3E004F070DB901BA2E004F08000
:10BC3600D3901BA4E0FF12D800E4901BA2F0A3F05F
:10BC4600901BA2E0FEA3E0FFC3EE9404501C74A375
:10BC56002FF58274153EF583E4F0901BA3E004F003
:10BC660070DE901BA2E004F080D622E4901BA2F0C6
:10BC7600A3F012D8D11220267F011220067FE87E7B
:10BC86000312D132C29712C30AEF7002800E12C39A
:10BC96000AEF7002800612C30AEF700D7F0112D6FA
:10BCA6004D12D8B9C2AF75A70FE4901BA2F0A3F04E
:10BCB600901BA2E0FEA3E0FFE4FCFD7B407A9CF92A
:10BCC600F8D31229EF4010901BA3E004F070E19026
:10BCD6001BA2E004F080D9B29780CEE4901BA2F0BC
:10BCE600A3F012CA1CEF7055901BA2F0A3F0901B94
:10BCF600A2E0FEA3E0FFC3EE9404503974002FF5D2
:10BD06008274003EF583E0FF12D84B501812D832E9
:10BD1600901BA2E0FEA3E02400F58274003EF583AA
:10BD2600E0FF12D800901BA3E004F070C1901BA2A4
:10BD3600E004F080B97BFF7ADE796A800912D83296
:10BD46007BFF7ADE796D1243AA227E097F607D0031
:10BD56007B017A007900122E5A12C92DEF704D9090
:10BD66001BA2F0A3F0901BA2E0FEA3E0FFC3EE949B
:10BD760008504574002FF58274003EF583E0FF12EB
:10BD8600D84B501812D832901BA2E0FEA3E0240034
:10BD9600F58274003EF583E0FF12D800901BA3E005
:10BDA60004F070C1901BA2E004F080B912D8327B77
:10BDB600FF7ADF798D1243AA228F468E458D448CF9
:10BDC600438B478A4889498F4F8E4E8D4D8C4CE563
:10BDD6004B2546FFE54A3545FEE43544FDE435434B
:10BDE600FCAB4FAA4EA94DA84CC3122A055037AF3B
:10BDF6004FAE4EAD4DAC4C12967AAB47AA48A94908
:10BE0600EF12277474012549F549E43548F548E5EC
:10BE16004F2401F54FE4354EF54EE4354DF54DE42E
:10BE2600354CF54C80A9228E228F23753A607539E0
:10BE3600E37538167537007F007E367D6E7C0112FD
:10BE4600CF55E4F524C3E524941174809480500EF4
:10BE5600E52490E69A93FF12D78E052480E7AF2358
:10BE660012D78EE522FF12D78E7F007E537D077C88
:10BE76000012B950EF701A78007C007D017BFF7AC2
:10BE8600E479A3122C93EF3395E04F7F017004FF02
:10BE9600227F01228F3E8E3D8D3C8C3B8B3F8A401C
:10BEA60089418F478E468D458C44E543253EFFE507
:10BEB60042353DFEE4353CFDE4353BFCAB47AA4646
:10BEC600A945A844C3122A055035AF47AE46AD452D
:10BED600AC44AB3F0541E541AA407002054014F968
:10BEE6001226FBF54C1285C1E5472401F547E435DA
:10BEF60046F546E43545F545E43544F54480AB2240
:10BF06007526017527097528787B017A09798812C3
:10BF160089C4EF3395E0C3648094807F0050027F2C
:10BF260001AD077526017527097528787B017A0901
:10BF3600799A1289C4EF3395E0C3648094807F00B8
:10BF460050027F01EDFB7A007006EF70037F01223D
:10BF5600EB64014A7006EF70037F0222ED64017004
:10BF660008EF640170037F03227F002212C3C6EF2D
:10BF76007002801EE4FF1220067FE87E0312D13293
:10BF86007F011220067FE87E0312D13212C3C6EF6C
:10BF960070061298A7E4800D7F2C7E0112D1321212
:10BFA600D068EF7018FDAF16AE15129ACA12D37F7D
:10BFB6009009687402F09009677409F02290096884
:10BFC6007403F07D18AF16AE15129ACA90096774FD
:10BFD60009F012D37F227D19AF16AE15129ACA1236
:10BFE600D679EF603912C3C6EF700280157F2C7EBA
:10BFF6000112D13212C3C6EF7002800612D068EF6A
:10C00600700302AEFC7D18AF16AE15129ACA12D393
:10C016007F9009687403F09009677409F0227D1B0C
:10C02600AF16AE15129ACA9009687403F07D18AF60
:10C0360016AE15129ACA9009677409F012D37F22B8
:10C046007FFE7EFF7D007C0012967AEF901BA2F0A9
:10C05600A3E4F07FFF7EFFFDFC12967A901BA3E01F
:10C066002FF0901BA2E03400F0A3E004F0700690DD
:10C076001BA2E004F07FFE7EFF7D007C001286C7D7
:10C08600901BA2E0F54C7FFE7EFF7D007C001285B2
:10C09600C1901BA2A3E0F54C7FFF7EFF7D007C00D4
:10C0A6001285C1E4F5A775EF10228E228F2375360F
:10C0B600FF7537E47538A085223985233A7B017AE6
:10C0C6001C79B51243A48F25753A607539E3753826
:10C0D600167537007F007E367D6E7C0112CF55E4E3
:10C0E600F524C3E524940B74809480500EE52490C7
:10C0F600E5F993FF12D78E052480E7AF2312D78E7A
:10C10600E522FF12D78E7FC87E007D007C0002B933
:10C1160050900991E08F828E83F0900992E08F8291
:10C126008E83A3F0900993E08F828E83A3A3F09071
:10C136000994E08F828E83A3A3A3F0900995E0FD76
:10C14600EF2404F582E43EF583EDF0900996E0FDD8
:10C15600EF2405F582E43EF583EDF0900997E0FDC6
:10C16600EF2406F582E43EF583EDF0EF2407F58231
:10C17600E43EF583E4F02285A72CE4F5A78FBBD235
:10C18600ECFF20ED0DEFC394647480948050030F90
:10C1960080F0C2EDC3EF9464748094804006AC2DA9
:10C1A600AD2E8030AFBDAEBEE48F328E31F530F5A8
:10C1B6002F7F307E11FDFCAB32AA31A930A82F1299
:10C1C60028C4E47BFF7A0FF9F812294FAC06AD07B5
:10C1D6008C2D8D2E852CA7AF05AE0422753A607581
:10C1E60039E37538167537007F007E367D6E7C0123
:10C1F60012CF55E4F527C3E5279412748094805036
:10C206000EE52790E6AB93FF12D78E052780E7E46D
:10C21600FF12D78E7F887E137D007C0012B950EF07
:10C22600701A78007C007D017BFF7AE479A3122CDA
:10C2360093EF3395E04F7F017004FF227F0122E4E4
:10C24600B51D14E51CB4080FAF11AE10AD0FAC0E42
:10C25600E4F52EF52F8032AF11AE10AD0FAC0EE423
:10C26600F52EF52F1287CBE5112401F511E43510D3
:10C27600F510E4350FF50FE4350EF50EAF11AE10DF
:10C28600AD0FFC752E08752F001287CBE511240122
:10C29600F511E43510F510E4350FF50FE4350EF51C
:10C2A6000E22AB07AA06901B47A3A3A3E08B828AA4
:10C2B60083F0901B47E0FCA3E0FDA3E0FEA3E0FFB4
:10C2C6007808122A168B828A83A3EFF0901B47E028
:10C2D600FCA3E0FDA3E0FEA3E0FF7810122A168B74
:10C2E600828A83A3A3EFF0901B47E0FCA3E0FDA3A3
:10C2F600E0FEA3E0FF7818122A168B828A83A3A396
:10C30600A3EFF022753A607539E375381675370074
:10C316007F007E367D6E7C0112CF55E4F522C3E5A3
:10C3260022940B74809480500EE52290E6BD93FF14
:10C3360012D78E052280E77F647E007D007C001286
:10C34600B950EF701A78007C007D017BFF7AE479A2
:10C35600A3122C93EF3395E04F7F017004FF227FE9
:10C3660001228D26E5266402701A1226FB901BA771
:10C37600F0900001122714901BA6F0E0FEA3E0FF48
:10C38600E4FCFD22E526640470271226FB901BA917
:10C39600F0900001122714901BA8F09000021227BB
:10C3A60014901BA7F0900003122714901BA6F08090
:10C3B60003901BA6E0FCA3E0FDA3E0FEA3E0FF22A2
:10C3C600753A607539E37538167537007F007E3625
:10C3D6007D6E7C0112CF55E4F52AF52B74C8252B0A
:10C3E600F58274E6352AF583E493FF12D78E052B82
:10C3F600E52B7002052AC3940CE52A940040DD7FE4
:10C40600887E137D007C0012B950EF700B7E007F92
:10C41600007DFF7C0302D32C7F0122753A607539BB
:10C42600E37538167537007F007E367D6E7C011207
:10C43600CF55E4F526F52774D42527F58274E6351D
:10C4460026F583E493FF12D78E0527E527700205AC
:10C4560026C39413E526940040DD7F887E137D0075
:10C466007C0012B950EF700B7E007F007DFF7C03CD
:10C4760002D32C7F0122753A607539E3753816753B
:10C4860037007F007E367D6E7C0112CF55E4F523A2
:10C49600F52474182524F58274E53523F583E49391
:10C4A600FF12D78E0524E52470020523C3940BE5FD
:10C4B60023940040DD7F887E137D007C0012B950F6
:10C4C600EF700B7E007F007DFF7C0302D32C7F0183
:10C4D6002201630001620002580000025A000002B5
:10C4E6005C0000015E00441CC400000E10441CC821
:10C4F60000000E10441CCC00000E10441CD000009E
:10C506000E10441CD400000E10441CD8000007086E
:10C51600411CDC00411CDD00411CE000421CE10026
:10C52600000215097802180991008E328F338C3477
:10C536008D35E4F569F568F567F566AF03AE0290EB
:10C546000985E0FCA3E0FD12D58BAE32AF33E4FCE7
:10C55600FDAB69AA68A967A866C3122A055006E555
:10C5660065456460E5AE34AF35E4FCFDAB69AA68A9
:10C57600A967A866C3122A0540EB53E7F7AE64AF76
:10C586006522E4901BA2F0A3F012B190901BA4EEDA
:10C59600F0A3EFF04E603F12D832E4901BA2F0A356
:10C5A600F0901BA4E0FEA3E0FF901BA2E0FCA3E03A
:10C5B600FDC39FEC9E502274002DF58274003CF55D
:10C5C60083E0FF12D800901BA3E004F070D3901B09
:10C5D600A2E004F080CB12D77C228F358E348D33C7
:10C5E6008C32E47F03FEFDFCAB35AA34A933A832B6
:10C5F600C3122A055008E47F01FEFDFC801AAF3500
:10C60600AE34AD33AC32E41223A47B9A7A997939ED
:10C6160078401223071223E28F398E388D378C36F5
:10C62600783674FF122A3EEC4D4E4F60030080F0C0
:10C636002285A722E4F5A775981075A70F122ADBA5
:10C64600C67F00002580C6770001C200C672000BB7
:10C6560071B0C66D000F4240C6680016E360000068
:10C66600C68575ACF8800D75ACF4800875ACF080A5
:10C676000375AC9875ADFF800675AC1E75ADFB7580
:10C68600AB43D2AC8522A722C0E0C083C082C0D013
:10C6960075D000C00630983BC298C3E565956DE538
:10C6A60064956C502B856B82856A830565E565AE5E
:10C6B6006470020564142582F582E5833EF583E500
:10C6C60099F07569007568007567007566008003E6
:10C6D60053E7F7D006D0D0D082D083D0E0327F0A9D
:10C6E6007E007D007C008F278E268D258C24E4F528
:10C6F6002BF52AF529F528AF27AE26AD25AC24ABB8
:10C706002BAA2AA929A828C3122A055025E4FFFE28
:10C716000FBF00010EBE04F8BF38F5E52B2401F566
:10C726002BE4352AF52AE43529F529E43528F528B8
:10C7360080C5227E097F607D007B017A0079001228
:10C746002E5A753AE07539937538047537007F00AF
:10C756007E367D6E7C0112CF557F3112D78E7F32A9
:10C766007E007D007C0012B950EF7017FFFE0FEFC0
:10C77600AC0670010E142400F58274003CF583E0CB
:10C7860070EC22E4FEFF227E097F607D007B017A49
:10C79600007900122E5A753AE0753993753804758A
:10C7A60037007F007E367D6E7C0112CF557F3212B8
:10C7B600D78E7F327E007D007C0012B950EF701755
:10C7C600FFFE0FEFAC0670010E142400F582740014
:10C7D6003CF583E070EC22E4FEFF22E4901BA2F01D
:10C7E600A3F0901BA2E475F001122849FE74A3255C
:10C7F600F0F58274093EF583E070E712D832901B9B
:10C80600A2E0FEA3E024A3F58274093EF583E0606E
:10C816001D901BA2E475F001122849FE74A325F0B1
:10C82600F58274093EF583E0FF12D80080D022E439
:10C83600901BA2F0A3F0901BA2E475F00112284908
:10C84600FE74A325F0F58274093EF583E070E712C5
:10C85600D832901BA2E0FEA3E024A3F58274093E21
:10C86600F583E0601D901BA2E475F001122849FED5
:10C8760074A325F0F58274093EF583E0FF12D80013
:10C8860080D0228B298A2A892BE94A4B60467F135E
:10C8960012C17DEE3395E0FDFCE47B0BFAF9F8124C
:10C8A60028C4AB29AA2AA92B900002EE8FF01228E1
:10C8B600977F1212C17DEE3395E0FDFCE47B0BFA07
:10C8C600F9F81228C4AB29AA2AA92B900004EE8FE6
:10C8D600F01228972212C3C6EF703F12D832E490A6
:10C8E6001BA2F0A3F0900960E0FEA3E0FF901BA25C
:10C8F600E0FCA3E0FDC39FEC9E502B74002DF58257
:10C9060074003CF583E0FF12D800901BA3E004F00E
:10C9160070D3901BA2E004F080CB12D8327BFF7A52
:10C92600DE79D81243AA22753A607539E37538164E
:10C936007537007F007E367D6E7C0112CF55E4F59B
:10C9460022F52374F32523F58274E63522F583E474
:10C9560093FF12D78E0523E52370020522C3941098
:10C96600E5226480948040DBE4FF12D78E7FF47E5C
:10C97600017D007C0002B95085A722E4F5A775FF6A
:10C9860080F582F583A3E58264FE458370F7E4F5BE
:10C9960083F582E5FF30E613AF82AE83E4FCFD7BD0
:10C9A600607AEAF9F8D31229EF4003A380E5E5FFA0
:10C9B60030E60575EF02800CE4F5EF7D25AF16AE87
:10C9C60015129ACA8522A7227B2E7E1C7F227D40C5
:10C9D6007C008E3B8F3C8C3D8D3E8B3FAA06A90783
:10C9E6007B0112D6A5EF2401FDE43EFCC3ED953E86
:10C9F600EC953D5020E53C2FF582E53B3EF583E581
:10CA06003FF0EF2401FFE43EFEE53C2FF582E53BD7
:10CA16003EF583E4F0227E097F607D007B017A008B
:10CA26007900122E5A753A607539E37538167537DE
:10CA3600007F007E367D6E7C0112CF55E4F522C361
:10CA4600E522940974809480500EE52290E60793BF
:10CA5600FF12D78E052280E77F327E007D007C00A4
:10CA660002B9507E097F607D007B017A0079001251
:10CA76002E5A753A607539E37538167537007F009A
:10CA86007E367D6E7C0112CF55E4F522C3E52294F5
:10CA96001174809480500EE52290E61093FF12D711
:10CAA6008E052280E77F647E007D007C0002B950FF
:10CAB6007E097F607D007B017A007900122E5A750F
:10CAC6003A607539E37538167537007F007E367D16
:10CAD6006E7C0112CF55E4F522C3E52294107480D2
:10CAE6009480500EE52290E62193FF12D78E052200
:10CAF60080E77F647E007D007C0002B950856582F8
:10CB0600856483E47F0AFEFDFCAB69AA68A967A871
:10CB160066D3122A05402FE5829402E583940040ED
:10CB26002578627C1C7D017BFF7AE9791E7E007F79
:10CB360002122E36EF3395E04F700553E7F7FF22CA
:10CB460053E7F77F01227F01227E017FBE7D007BB6
:10CB5600017A0979A3122E5AE4900B61F0900B65C5
:10CB6600740BF0900B697404F0E4A3F0A3F0A3F047
:10CB7600A3F0A37409F0A3743DF0E4A3F07E04FFD0
:10CB8600FD7B017A0B7971122E5A900BA17455F028
:10CB9600A374AAF022753A607539E37538167537AD
:10CBA600007F007E367D6E7C0112CF55E4F528F5B8
:10CBB6002974A22529F58274E53528F583E493FFC7
:10CBC60012D78E0529E52970020528C3940DE5289C
:10CBD600940040DD7FE87E037D007C0002B950753D
:10CBE6003A607539E37538167537007F007E367DF5
:10CBF6006E7C0112CF55E4F522F52374D32523F577
:10CC06008274E53522F583E493FF12D78E0523E57A
:10CC16002370020522C3940DE522940040DD7FE0D7
:10CC26007E937DFF7CFF02B9508D238B2412D71E85
:10CC36007A00EF4480FB7D167FAC12B8DCAF23127E
:10CC4600D71E7A00EF4480FB7D157FAC12B8DCAFAF
:10CC56002412D71E7A00EF4480FB7D137FAC12B8F6
:10CC6600DCAF2512D71E7A00EF5401FB7D147FAC92
:10CC760002B8DCE4901BA2F0A3F0901BA2E475F0CE
:10CC860001122849FE74A325F0F58274093EF58346
:10CC9600E070E7901BA2E0FEA3E0FF12A16DEF702B
:10CCA6000512D76A800312D77C901BA2E0FEA3E090
:10CCB60024A3F974093EFA7B0102D79F8E228F23A3
:10CCC600753A607539E37538167537007F007E361C
:10CCD6007D6E7C0112CF55E4F524C3E524941174CE
:10CCE600809480500EE52490E69A93FF12D78E0525
:10CCF6002480E7AF2312D78EE522FF12D78E12D8F3
:10CD0600E77F0022E4901BA2F0A3F012CA1CEF708A
:10CD16003712D832E4901BA2F0A3F0901BA2E0FEDB
:10CD2600A3E0FFC3EE9404502274002FF582740032
:10CD36003EF583E0FF12D800901BA3E004F070DB01
:10CD4600901BA2E004F080D312D77C2212D731E4E4
:10CD5600FDAF2685A72F75A710AE07ED4206E5C8DD
:10CD660030E7FB12D73112D8F2E4FDEDC394087414
:10CD7600809480500A12D4D9EE25E0FE0D80EC1284
:10CD8600D5B58F30E530600312D6D0852FA7AF30EA
:10CD9600227525007524307523017522007F007EDB
:10CDA600607D017C00AB25AA24A923A822C3122AF0
:10CDB600055022AF25AE24AD23AC221286C7E4254A
:10CDC60025F525E5243402F524E43523F523E43559
:10CDD60022F52280C8228D238B2412D71EEFFB7AE0
:10CDE600007D0E7FAC12B8DCAF2312D71EEFFB7AA4
:10CDF600007D0D7FAC12B8DCAF2412D71EEFFB7A94
:10CE0600007D0B7FAC12B8DCAF2512D71EEFFB7A84
:10CE1600007D0C7FAC02B8DCE48F258E24F523F56B
:10CE260022AD23AC227B37FAF9F81228C48F258E5F
:10CE3600248D238C22E47BE87A03F9F81228C48F28
:10CE4600258E248D238C22E47B997A09F9F8122900
:10CE56004F8F258E248D238C2222900966E0640351
:10CE66006038C29712D7F190096BEFF0E4A3F09007
:10CE76000966E06402701A90096BE06014E4F51428
:10CE86007D21AF16AE15129ACA9009687402F08019
:10CE9600069009687403F012D37F227B017A097920
:10CEA600A312743AE4901BA2F0A3F0901BA2E0FE3A
:10CEB600A3E0FFC3EE9404501F74A32FF5827409F8
:10CEC6003EF583E0FF12D800901BA3E004F070DB70
:10CED600901BA2E004F080D322ABA775A70FC28EE9
:10CEE60053C7FD75A710859932C298C29975A70FC9
:10CEF60075D4CF75D50F43C7028BA78531448530CE
:10CF060043852F42852E41127C2A7E007F007D605C
:10CF16007C0902D58B85A73075A70F53E7F7C28E1C
:10CF260053C7FD75A710859931C298C29975A70F89
:10CF360075D4CF75D50343C702852F44852E438507
:10CF46002D42852C41127C2A43E7088530A722858D
:10CF5600A73B75A70F53E7F7C28E53C7FD75A710FA
:10CF660085993CC298C29975A70F75D4CFE4F5D5BB
:10CF760043C702853A44853943853842853741128D
:10CF86007C2A43E708853BA7228D228B2312D71ED6
:10CF96007A00EF4480FB7D127FAC12B8DCAF221220
:10CFA600D71E7A00EF4480FB7D117FAC12B8DCAF50
:10CFB6002312D71E7A00EF4480FB7D107FAC02B8A7
:10CFC600DCAEA7E4F5A78FBBD2ECFF20ED0DEFC3D7
:10CFD60094647480948050030F80F0C2EDEFC39484
:10CFE600647480948040067C067D008004ACBEADEF
:10CFF600BD8EA7AF05AE04228B288A29892A8C2BE1
:10D006008D2CE4FFE52C152CAC2B7002152B4C60F7
:10D0160015AB28052AE52AAA297002052914F91252
:10D0260026FB2FFF80DEEF75F0FFA4FF2212936A26
:10D036008F258E248D238C22EC4D4E4F601712D8EF
:10D04600327BFF7AE0790F852539852438852337A9
:10D05600852236800912D8327BFF7AE07924124382
:10D06600AA227D09AF16AE15129ACA7B017A0079FB
:10D076000012D4B7EF700F1298A77D1CAF16AE152D
:10D08600129ACA7F002212D9687D12AF16AE151207
:10D096009ACA7F01228E288F29EF2401FFE43EFEE3
:10D0A6008D2E7B01E4FD12563F78AD7C1B7D017E03
:10D0B600007F031226D5901BADE085298285288343
:10D0C600F07B017A1B79AD228D228B2312D71EEFBE
:10D0D600FB7A007D0A7FAC12B8DCAF2212D71EEFB6
:10D0E600FB7A007D097FAC12B8DCAF2312D71EEFA6
:10D0F600FB7A007D087FAC02B8DCAFA775A70F7579
:10D10600F1FE75F30375F4F875A41275A59575A669
:10D116000375AE7875AF0375D4CF75E10175C74257
:10D12600E4F5B575B00775A0FC8FA7228F828E83B4
:10D1360012D6E212D95112D744AF82AE83E4FCFD77
:10D14600AB0DAA0CA90BA80AD3122A0540EB12D8DC
:10D15600DC12D955E4F50DF50CF50BF50A228F22F4
:10D166008D237F6F12D8007F6B12D800AF2212D8A2
:10D1760000AF2312D800752404C3E52494407480BC
:10D1860094805009E4FF12D800052480EC228F22F7
:10D196008D237F6E12D8007F6F12D800AF2212D86F
:10D1A60000AF2312D800752404C3E524944074808C
:10D1B60094805009E4FF12D800052480EC227E00FA
:10D1C6007F007DFF7C0312D32C901BACEFF0600B2D
:10D1D60012C47C901BADE4F0A3EFF078A37C097D2C
:10D1E600017B017A0079007E047F000226D5C0E02B
:10D1F600C083C082C0D075D000C007309813C298D3
:10D20600AF63056374002FF582E43400F583E59976
:10D21600F0D007D0D0D082D083D0E0328F231298BE
:10D22600A712D95F8F118E108D0F8C0E12D968AD93
:10D2360023AF16AE15129ACA124BF39009687405FD
:10D24600F07D01AF16AE15029ACA9009A374EBF0F1
:10D25600A37458F0A37490F0A37445F0A3744CF033
:10D26600A37449F0A37443F0A3744FF0A3744DF074
:10D27600E4A3F0A37430F0228F2212D8327F6F120B
:10D28600D8007F6B12D800AF2212D800752303C3D3
:10D29600E5239440748094805009E4FF12D8000579
:10D2A6002380EC228F2212D8327F6E12D8007F6F35
:10D2B60012D800AF2212D800752303C3E523944089
:10D2C600748094805009E4FF12D800052380EC2274
:10D2D600AFA7E4F5A743BC0175BE0475BD7C75BE5A
:10D2E60007F5BD75BE0875BD0153BCFE75BB30752F
:10D2F600BC3875E8C075D1178FA72212D5E9E4901E
:10D30600096CF012CD977527FF7528E1752988906D
:10D316000964E0FAA3E0FB7D20AF16AE151279335F
:10D32600E4FFFE02CCC28E328F337FFFED1DAA04CE
:10D3360070011C4A60190533E533AA3270020532C2
:10D3460014F5828A83E06FFE90E72193FF80DD2249
:10D356007D027F8012A70E901B9DE0FEA3E02400B5
:10D36600FFE43EFEEF7803CEC313CE13D8F978025E
:10D37600C333CE33CED8F9FF22AFA775A70F8FA739
:10D38600E4FF12D64DE4FF122006E4FF122096E4D5
:10D39600FF12D663E4FF12D94012D90612D81E0234
:10D3A600D8C5E5176006E4F517128E50125E95EFA4
:10D3B600700C12D8FC122E9812D906127283E5143C
:10D3C60064017005F51412D5E922E4901BA2F0A3BE
:10D3D600F0901BA2E475F001122849FE74A325F013
:10D3E600F58274093EF583E070E790096C04F0025B
:10D3F600D76AC29712C30AEF70137F0112D64D1275
:10D40600D8B912D8327BFF7AE1793C800912D8323A
:10D416007BFF7AE1794C1243AA22AEA775A710E4E6
:10D42600FDFCECC39408748094805010ED25E0FD5B
:10D436005305FE12D5B5EF42050C80E68EA7AF0563
:10D4460022AE07E4FDEDC3940874809480500A125E
:10D45600D4D9EE25E0FE0D80EC12D5B58F2FE52F41
:10D46600600312D6D0AF2F2212D8327BFF7AE17931
:10D476005C90096FE0FCA3E0FDA3E0FEA3E0F539B4
:10D486008E388D378C361243AAE4FF02D800AFA738
:10D4960075A70F759F3075A7107592FF7593FE756A
:10D4A60094FF7595FE4396104391048FA743E7803A
:10D4B600228B238A248925754A04754B007F007EBA
:10D4C600507D017C0012BDBFAE24AF257D007C04DB
:10D4D60002D32CEEC41313135401FFC287EF24FFAB
:10D4E6009286E5C830E7FB12D731D287E5C830E728
:10D4F600FB02D731C0E0C0D053917FE50D2401F582
:10D506000DE4350CF50CE4350BF50BE4350AF50A9C
:10D51600D0D0D0E032E4FFFE12BE2DEF700B12D851
:10D52600327BFF7ADE793A800912D8327BFF7ADEC7
:10D5360079501243AA22C0E0C0D0C2CFE5692401C7
:10D54600F569E43568F568E43567F567E43566F549
:10D5560066D0D0D0E0328F298E288D278C26AF2931
:10D56600AE28AD27AC26AB0DAA0CA90BA80AD31280
:10D576002A0540EA22F569F568F567F5667E007FBB
:10D58600007D607C098E6A8F6BE4F564F5658C6CB2
:10D596008D6D22EFFD3395E0FCD3ED9439EC64807C
:10D5A60094805006C3EF9430FF22EF24C9FF22D2A5
:10D5B60086C287E5C830E7FB12D731D287A286E458
:10D5C60033FFE5C830E7FB02D7317B017A007D01E6
:10D5D6007FAC12B8DC7B017A007D027FAC12B8DC2E
:10D5E60002D7E2E4FBFA7D017FAC12B8DCE4FBFA79
:0ED5F6007D027FAC12B8DC02D9595390F322AB
:07D6080043900C5390F72240
:07D6100043900C5390FB2234
:10D6180043900C22C0E0C083C08253917F751701EC
:10D6280090096E7401F0D082D083D0E032AFA7E4C5
:10D63800F5A775CBFE75CA0B85CBCD85CACCD2CAEA
:10D64800D2AD8FA7228F277F327E0012D132E527F5
:10D6580024FF92B37F647E0002D1328F277F327E0F
:10D668000012D132E52724FF92B67FF47E0102D161
:10D67800327F907E087D007C0012B5047E007F001A
:10D688007DFF7C0302D32C12D7F1EF6401700D12D9
:10D69800D8327F0112D8007FEB12D80022E4FFFEB7
:10D6A8001226FB600C0FEF70010E09E970F20A8078
:10D6B800EF22901B9DE0FFEFC4540F75F00AA4FE03
:10D6C800EF540F2EFF22EFF07F0112D4E1E4FF1296
:10D6D800D4E1E4F5C8D286D28722AFA7E4F5A775CE
:10D6E80093F875922F8593958592948FA722900928
:10D6F80068E0640870087F0112D94002D76A12D71F
:10D708007C2212D832129ED87BFF7AE07998124395
:10D71800AAE4FF02D800EF75F00A84C454F0FEEFC3
:10D7280075F00A84E5F04EFF22E4F5C875CBFF7565
:10D73800CAE675CDFF75CCE675C80422ABA7E4F53B
:10D748000DF50CF50BF50AF5A74391048BA722EF0D
:10D75800C394094005EF940E4003BF2003D3800112
:10D76800C32212D8327F6F12D8007F6B12D800E420
:10D77800FF02D80012D8327F6E12D8007F6F12D8FD
:10D7880000E4FF02D800AEA775A710C2998F9930A0
:10D7980099FDC2998EA7227542047543007F007EC9
:10D7A800507D017C0002BE9AE4FF12200612D83296
:10D7B8007BFF7AE079B90243AA7F0112200612D8CA
:10D7C800327BFF7AE079D00243AA7BFF7ADE791FA9
:10D7D8001243AAE4F5A775EF1022AFA775A70F7536
:10D7E800E4068FA7D296D2A8227D017FAC12A70E9D
:10D7F800901B9DE05401FF22AEA7E4F5A78F993056
:10D8080099FDC2998EA722AEA7E4F5A78F99309902
:10D81800FDC2998EA7227F047E007D007C0012C580
:10D82800E053B5FD22EEF0A3EFF07F0A12D8007F97
:10D838003E02D800123A4712D8327BFF7ADE79C806
:10D848000243AAEFC394204007EF947F500280015F
:10D85800C322EFC394304007EF943A50028001C3CB
:10D868002243B5027F027E007D007C0002C5E09065
:10D8780009687401F0E4FF12D94002D76AAD077F46
:10D88800AC12A70E901B9DE0FF22AE05AD07EEFB84
:10D898007A007FAC02B8DC12CB03EF700302D76AC0
:10D8A80012D77C2212BB1CEF700302D76A12D77CF6
:10D8B80022C2A07FC87E0012D132D2A02285A7271B
:10D8C80075A70F53ABBFC2AC22AFA775A70F75A141
:10D8D800C78FA722AFA7E4F5A75391FB8FA7227E96
:10D8E8001C7F627D3F7C0002D58BC286E5C830E78D
:10D8F800FB02D73143B5017F017E0002D13253B517
:10D90800FE7F017E0002D1329009687408F002D7C8
:10D918006A9009687401F002D76AEF6D90E7219365
:10D92800FF2212D100D297027ED675140112D9595E
:10D9380032E4F5A753D9BF22EF24FF92A12212D5D2
:10D94800E902D76A7EE17F882243E6402253E6BF98
:10D9580022C2A822D2AF2202936A02D76A02B77102
:10D96800028F34202D204177616974696E672072B7
:10D978006567697374726174696F6E2E2E2E00204C
:10D988002D20526567697374726174696F6E206DBA
:10D998006F6465206163746976652E00202D2052BE
:10D9A8006567697374726174696F6E206D6F646501
:10D9B80020636F6E636C756465642E00202D2052A1
:10D9C8006573746F72696E672072656769737472C4
:10D9D8006174696F6E206D6F64652E2E2E00202D88
:10D9E800204E6F20726573706F6E73652066726F5C
:10D9F8006D206465766963652E00202D2053686F5D
:10DA080072742063697263756974206465746563F0
:10DA18007465643A2000202D205A65726F20706F5B
:10DA280077657220636F6E73756D7074696F6E3A87
:10DA38002000202D204572726F722072656365691F
:10DA480076696E6720646174612066726F6D206408
:10DA580065766963652E00202D20494D5041435459
:10DA680020657863656564696E67206465746563BD
:10DA7800743A2000202D20275461736B2720666993
:10DA88006C65206D697373696E6720696E204E41FD
:10DA98004E442E00202D20566F6C7461676520520D
:10DAA8006567756C61746F722044726F706F7574FE
:10DAB8002064657465637465642E00202D20705F92
:10DAC80061646472657373206F766572666C6F77D4
:10DAD8003A2000202D2048525A5F73697A653A200F
:10DAE80000202D205761726E696E672C20536D617E
:10DAF800727420737769746368206F75743A2000B4
:10DB0800202D205761726E696E672C20746865201D
:10DB1800667573652069732063726173682E0020CF
:10DB28002D205761726E696E672C205562617420D2
:10DB380044726F706F7574206465746563743A20FD
:10DB480000202D205761726E696E673A2052656712
:10DB580020537461727420776974682054656D70FD
:10DB68002E00202D20275461736B272066696C6571
:10DB7800206D697373696E6720696E20466C6173E6
:10DB8800682E00202D2052544320416C61726D2074
:10DB98007472696767657265642E00202D2053745E
:10DBA80061727420526567697374726174696F6E0B
:10DBB8002044756520746F2074696D65206D6174EB
:10DBC80063682E00202D2045565420666F72204130
:10DBD8005220746F2053657269616C206E756D6296
:10DBE80065723A2000202D204572726F722077727C
:10DBF8006974696E6720746F20666C61736820733E
:10DC0800746F726167652E2000202D205761746340
:10DC180068646F672054696D657220526573657416
:10DC2800207472696767657265642E00202D205321
:10DC3800797374656D2073757370656E646564209F
:10DC480064756520746F20706F77657220697373CF
:10DC58007565732E00202D20416C61726D206E6FEA
:10DC680074207365742E00202D20417761697469D2
:10DC78006E67206D6F646520286E6F206261747412
:10DC880065727920706F7765722900202D204865AC
:10DC9800616465722048525A2073756363657373B3
:10DCA80066756C6C7920726561642E00202D2027C2
:10DCB8005461736B272066696C65206765742069F9
:10DCC8006E20466C6173682E00202D2052656720F7
:10DCD8006D6F6465206D6573736167653A206E6F5B
:10DCE800204261747465727920706F7765720020C4
:10DCF8002D20526567206D6F6465206D65737361B3
:10DD080067653A2054696D6520656E6400202D2092
:10DD18005254432072656164206D616A6F72697440
:10DD280079206661756C742E00202D205365726908
:10DD3800616C206E756D6265722026206669726D51
:10DD4800776172652076657273696F6E3A2000207C
:10DD58002D204177616974696E67206D6F64652055
:10DD68006166746572204C494E4B2073746174650A
:10DD78002E00202D20526567206D6F6465206D652B
:10DD880073736167653A2055534220706F776572E7
:10DD980020636F6E6E656374656400202D20494DA5
:10DDA80050414354206F766572203135673A200020
:10DDB800202D205461736B20706172736520657229
:10DDC800726F722E00202D20564444204D6F6E69CC
:10DDD800746F72204661696C65642064657465635C
:10DDE8007465642E00202D20556E6B6E6F776E2043
:10DDF8006576656E742E0030006D470020006C6FEC
:10DE0800616465720072657365740065726173653B
:10DE1800007772697465005265736574205379736D
:10DE280074656D0A0D004D61722032342032303233
:10DE3800360046696C652073797374656D2063726A
:10DE480065617465640A0D0046696C6520737973B1
:10DE580074656D206E6F7420637265617465640A01
:10DE68000D000A0D004572726F7220726561646957
:10DE78006E67204F6E66692061727261790A0D00C3
:10DE880057726974654C6F676963616C5061676547
:10DE9800204F4B2C2070616765203D20256C640065
:10DEA80057726974654C6F676963616C5061676527
:10DEB800204E4F2C2070616765203D20256C640042
:10DEC8005365744B6174616C6F67204F4B0A0D008A
:10DED8006E6F7420726573706F6E73696E672066FB
:10DEE8006F7220636F6D6D616E64204E616E644762
:10DEF80065745461736B006E6F7420726573706F14
:10DF08006E73696720666F7220636F6D6D616E64F2
:10DF18002052656164506879736963616C41646417
:10DF280072657373006E6F7420526573706F6E73D1
:10DF3800696E6720666F7220636F6D6D616E642015
:10DF48004572617365426C6F636B006E6F7420522B
:10DF58006573706F6E73696E6720666F7220636F8A
:10DF68006D6D616E6420536574446174610A0D00BF
:10DF7800467265652041646472657373203D20258F
:10DF88006C640A0D006E6F7420726573706F6E7327
:10DF9800696E6720666F7220636F6D6D616E6420B5
:10DFA8004765745461736B0A0D006E6F7420726557
:10DFB80073706F6E73696E6720666F7220636F6D22
:10DFC8006D616E64205465726D696E616C4765742D
:10DFD800506167650A0D004E6F74206D6F7665207D
:10DFE8004B6174616C6F670A0D004E6F7420676532
:10DFF800742048727A0A0D004E6F74207772697423
:10E008006520706167650066726565206164647289
:10E01800657373203D20256C640A0D006E6F7420B3
:10E028006672656520616464726573730A0D0077B2
:10E038007269746520256C64206164647265737309
:10E04800203D207375636365737300777269746527
:10E05800206661696C6564004572726F7250726502
:10E0680070617265526573746F7265004572726F84
:10E0780072526573706F6E7365526573746F7265F3
:10E088004661743332636F6D6D616E64004F4B008F
:10E098006F6B007265616420616464726573733DBF
:10E0A800256C64200072656164206661696C656432
:10E0B80000526567697374726174696F6E20706F5E
:10E0C800776572204F4646005265676973746172BE
:10E0D80074696F6E20706F776572204F4E004D6FB8
:10E0E80076654B6174616C6F6720737563636573E4
:10E0F800730A0D0047657448727A20737563636507
:10E1080073730A0D0057726974652048525A204289
:10E118006F647920737563636573730A0D005772B2
:10E128006974652048525A20426F64792066616993
:10E138006C0A0D005365745573624D6F6465204F0A
:10E148004B0A0D005365745573624D6F6465204E1C
:10E158004F0A0D00256C6400253032642F253032BB
:10E16800642F2530326420253032643A25303264F9
:10E178003A253032640A0D0041525F3135300000D3
:10E188005F332E300000000030372E30322E32350B
:10E19800004572726F725072657061726552657374
:10E1A800746F7265006C6F61646572006669726D88
:10E1B800776172655F766572007465737400726367
:10E1C800616C007763616C0067657474696D6500E4
:10E1D800636C660067616C0063686172676572658D
:10E1E800670073657474696D6500617574680073A0
:10E1F800657461736D0067640067645F6130006710
:10E20800645F61310067645F61320067645F613336
:10E21800007365745F706172616D00666173745F2D
:10E22800636C656172007772697465706167650017
:10E238006261636B75705F7461736B0063686563BB
:10E248006B0063686B6F66660063686B6F6E006374
:10E258006F6E00636F666600706F737473796E63B8
:10E2680000636C65617200436C6561720072656180
:10E2780064007265616470616765006372656174EA
:10E288006566696C650043726561746546696C65AD
:10E2980000626174746572795F6F6B006261747497
:10E2A8006572795F696E660077726974655F706818
:10E2B80079736963616C5F70616765007265616439
:10E2C8005F706879736963616C5F70616765006529
:10E2D800726173655F626C6F636B00746573745F02
:10E2E80072657175657374006E616E645F696E69DD
:10E2F80074006E616E645F6F6E66695F72656164FB
:10E308000065726173655F656E6400577269746554
:10E318004164647265737354657374005265616413
:10E3280041646472657373546573740070656769DA
:10E338007374726174696F6E5F706F7765725F6412
:10E348006F776E00726567697374726174696F6E56
:10E358005F706F7765725F7570006E616E645F6C79
:10E368006F61646572004765744E616E64436F6DDA
:10E3780070696C65566572004E616E6447657454C9
:10E3880061736B00526573746F72654661743332E2
:10E398000057726974654C6F676963616C50616797
:10E3A8006500526561644C6F676963616C506167B1
:10E3B80065004765744576656E74506167650072DF
:10E3C800656661740072656661745F737461747503
:10E3D800730047657452756E6E696E6754696D6532
:10E3E80000526573657452756E6E696E6754696D17
:10E3F80065004765744576744D657373616765009C
:10E408004765744F6E6669004765745061676500BB
:10E418004765745061676531004765745061676589
:10E428003200536574466174333200526573657403
:10E43800004765745461736B005365745461736B62
:10E44800005365744B6174616C6F67005365745059
:10E458006F737473796E63004765744672656541BE
:10E46800646472657373005365745573624D6F64A9
:10E478006500536574446174610047657454696D3F
:10E488006500556E6B6E6F776E20636F6D6D616E94
:10E49800640A0D00256C64002564004F4B0025308C
:10E4A80032642F253032642F2530326420253032F3
:10E4B800643A253032643A25303264006F6B004E7E
:10E4C800616E64496E69740041545F575F315F48FB
:10E4D800414C460041545F575F325F48414C46000B
:10E4E80045726173655461736B426F647900476567
:10E4F8007446726565416464726573730052656140
:10E508006450616765466F7250687950616765004D
:10E5180047657448727A426F647900457261736521
:10E5280048727A426F6479004D6F76654B61746109
:10E538006C6F67004765744672656541646472650F
:10E5480073735465737400526561644164647265E1
:10E5580073735465737400577269746541646472A7
:10E568006573735465737400476574436F6D7069A0
:10E578006C6544617461005F6C6F61646572000072
:10E5880016E360001E8480536574526573746F725D
:10E59800655461736B426F647900536574457665A1
:10E5A8006E74426F647900536574526573746F7248
:10E5B8006548525A426F64790053657452657374A2
:10E5C8006F72654B6174616C6F6700526573746F2D
:10E5D80072654661743332005772697465506879A0
:10E5E800506167650052656164506879506167657C
:10E5F800004572617365426C6F636B004154005251
:10E608006561644F6E666900537461727452656225
:10E6180075696C644E616E640052656275696C64FC
:10E6280050726F6772657373005465726D696E61BD
:10E638006C53657444617461005365744576740065
:10E648005265616450616765004765744576744238
:10E658006F6479466972737448616C6600476574C3
:10E66800457674426F64795365636F6E6448616C74
:10E678006600536574457674496E666F0057726913
:10E6880074655061676500577269746532506167D7
:10E69800650043726561746546696C655379737486
:10E6A800656D0052657365744576656E744C6F6769
:10E6B80046696C65005365745573624D6F646500F7
:10E6C8004765745461736B426F6479004765744899
:10E6D800727A426F6479576974684461746500534B
:10E6E80065745461736B426F6479005465726D6927
:10E6F8006E616C5365745461736B00536574487232
:10E708007A426F6479576974684461746500536527
:10E718007448727A426F647900005EBCE2613FDD42
:10E7280083C29C7E20A3FD1F419DC3217FFCA24084
:10E738001E5F01E3BD3E6082DC237D9FC1421CFE5B
:10E74800A0E1BF5D0380DE3C62BEE0025CDF816366
:10E758003D7C22C09E1D43A1FF4618FAA427799B41
:10E76800C584DA3866E5BB5907DB856739BAE4063C
:10E77800581947A5FB7826C49A653BD987045AB827
:10E78800E6A7F91B45C6987A24F8A6441A99C7251E
:10E798007B3A6486D85B05E7B98CD2306EEDB3510D
:10E7A8000F4E10F2AC2F7193CD114FADF3702ECCEC
:10E7B80092D38D6F31B2EC0E50AFF1134DCE9072F3
:10E7C8002C6D33D18F0C52B0EE326C8ED0530DEFCE
:10E7D800B1F0AE4C1291CF2D73CA947628ABF517D1
:10E7E800490856B4EA6937D58B5709EBB536688AB4
:10E7F800D495CB2977F4AA4816E9B7550B88D634AF
:10E808006A2B7597C94A14F6A8742AC896154BA995
:10E81800F7B6E80A54D7896B3542200049006E00E4
:10E8280066006F000F007272006D0061007400696D
:10E83800006F0000006E00000001530079007300B3
:10E84800740065000F00726D00200056006F006CA8
:10E8580000750000006D00650053595354454D7E06
:10E868003120202016009F13918F558F55000014DA
:10E87800918F550300000000005441534B20202085
:10E888002020202020000126918F558F5500008AD6
:10E898005E8F550A00000400004556454E544C4F03
:10E8A8004754585420006C5C8952575257000070E6
:10E8B8008752570600001000004147474320202098
:10E8C8002048525A2000B333918F558F550000A429
:10E8D800788F550B0000E06CF76D412E006D562EB9
:10E8E8000070616765000000010001000100000080
:10E8F800000000000000000001000000000000000F
:10E9080000000000000000000100010000000000FD
:0FE918000000000000004F4B006D4700000000A2
:00000001FF
